:020000040000FA
:10000000B8780020D5230000DD640000A92300009B
:10001000A9230000A9230000A9230000A9230000B0
:10002000000000000000000000000000491F000068
:10003000A923000000000000A9230000A92300005C
:10004000A51F0000A51F0000A51F0000A51F0000A0
:10005000A51F0000A51F0000A51F0000A51F000090
:10006000A51F0000A51F0000A51F0000A51F000080
:10007000A51F0000A51F0000A51F0000A51F000070
:10008000A51F0000A51F0000A51F0000A51F000060
:10009000A51F0000A51F0000A51F0000A51F000050
:1000A000A51F0000A51F0000A51F0000A51F000040
:1000B000A51F0000A51F0000A51F0000A51F000030
:1000C000A51F0000A51F0000A51F0000A51F000020
:1000D000A51F0000A51F0000A51F0000A51F000010
:1000E000A51F0000A51F0000A51F0000A51F000000
:1000F000A51F0000A51F0000A51F0000A51F0000F0
:10010000A51F0000A51F0000A51F0000A51F0000DF
:10011000A51F0000A51F0000A51F0000A51F0000CF
:10012000A51F0000A51F0000A51F0000A51F0000BF
:10013000A51F0000A51F0000A51F0000A51F0000AF
:10014000A51F0000A51F0000A51F0000A51F00009F
:10015000A51F000053B94AB9002908BF00281CBFD9
:100160004FF0FF314FF0FF3000F00CB8ADF1080C4C
:100170006DE904CE00F008F8DDF804E0DDE90223C3
:1001800004B07047704700BF2DE9F04786468C46A3
:100190000846089E154674461946002B40F0C1805B
:1001A0008542B2FA82F245D94AB1C2F1200300FA7F
:1001B00002FC954094402EFA03F343EA0C0C4FEAFC
:1001C000154EA8B2230CBCFBFEF80EFB18CC08FBA6
:1001D00000F943EA0C43994528D9EB1808F1FF3799
:1001E00004D2994502D9A8F102072B44A3EB0903D5
:1001F000A4B2B3FBFEFC0EFB1C330CFB00F044EA84
:100200000344A04214D92C190CF1FF3304D2A042AC
:1002100002D9ACF102032C44241A43EA07401EB170
:10022000D440002334607360BDE8F0874746DDE7C3
:100230006346F1E792BB431B01214FEA154EAFB273
:10024000200CB3FBFEFC0EFB1C330CFB07F840EA52
:100250000343984561D9EB180CF1FF3004D298455F
:1002600002D9ACF102002B44A3EB0803A4B2B3FB08
:10027000FEFC0EFB1C330CFB07F744EA0344A742C9
:100280004DD92C190CF1FF3304D2A74202D9ACF19D
:1002900002032C44E41B43EA0040C0E7C2F1200300
:1002A0009540944020FA03F12EFA03F34FEA154EDD
:1002B0009040AFB20343B1FBFEFC0EFB1C10190CC7
:1002C0000CFB07F841EA0041884522D969180CF176
:1002D000FF3004D2884502D9ACF102002944A1EBD9
:1002E00008019BB2B1FBFEFC0EFB1C110CFB07F7D7
:1002F00043EA01439F420ED9EB180CF1FF3104D2BF
:100300009F4202D9ACF102012B44DB1B41EA0041C0
:1003100093E76046E3E76146F7E76046A4E7634694
:10032000B8E7834206D916B9002108467CE7C6E93A
:1003300000E0F9E7B3FA83F78FB9834201D372453E
:1003400008D8BEEB020460EB030301209C461EB9F3
:10035000002169E73846FAE7C6E9004CF8E7C7F13B
:10036000200CBB400EFA07F522FA0CF42EFA0CF121
:10037000BA401C4320FA0CF3B8404FEA1449014339
:100380001FFA84FEB3FBF9F809FB18300B0C08FBCD
:100390000EFA43EA00439A4540D9E31808F1FF30CA
:1003A00004D29A4502D9A8F102002344A3EB0A0320
:1003B00089B2B3FBF9F809FB183308FB0EFE41EADA
:1003C00003418E452CD9611808F1FF3304D28E45C4
:1003D00002D9A8F10203214443EA0040A1EB0E0137
:1003E000A0FB02984145CE46434602D306D14D4577
:1003F00004D20138B9EB020E68EB0403002EA7D03B
:10040000B5EB0E0261EB030101FA0CFC22FA07F3D3
:10041000F9404CEA0303C6E9003199E74046C5E7D5
:100420004346D9E7F0B5394B394A4921C2F800367D
:10043000C2F80436C2F80836C2F80C36C2F81036D4
:10044000C2F81436C2F81836C2F81C3602F58052CB
:10045000C2F800362F48C2F8043685B0C2F8083614
:10046000C2F80C36C2F81036C2F81436C2F8183684
:10047000C2F81C3605F0A9FF00F07AF801A800F0D8
:1004800023FD254B1B68834204D04521234805F0FA
:100490009CFFFEE7039A4921214805F096FF492178
:1004A000204805F092FF4FF44041002003F024FC67
:1004B000044620B145211C4805F087FFFEE703F004
:1004C000B1FC69469DF8080000F032F8009B039DDE
:1004D0001D44019B1E8900F0C7FFAF1900F0A8FF63
:1004E00001F0BAFF84F30B8884F30A88AB5983F3D5
:1004F000088884F31488BFF36F8FBFF36F8F7B6816
:1005000098474521094805F060FFFEE73546526EE1
:10051000008001501A8E0000E0210020338E000080
:10052000568E0000858E0000AA8E0000DD8E000031
:10053000024608B538B105480023452105F045FFBE
:100540006FF0150008BD0860FCE700BF008F0000D9
:100550001FB50C46014601AA044806F072F918B905
:10056000019B2360029B636004B010BDF086000015
:100570004FF4C051014803F0A3BE00BFAC2F0020D0
:100580002DE9F04FDFF8E4A1F9B038A8DDE984489F
:1005900017461D46DAF8006007F0C5FD002138A8AF
:1005A00003F0A2FF3CB1B8F1000F04DD4246214642
:1005B00038A807F0BCFD4FF000097B89B7F8088028
:1005C0009844FB689844C84521D80DA938A807F07D
:1005D000E7FD869B23B1202218460DA905F0BCFF3C
:1005E00000232A46009339464FF6FF7307A805F00B
:1005F0009DFB044638B928460C9F00F0DDF9874280
:100600001BD94FF0FF34204679B0BDE8F08F839BB3
:10061000A8EB090B9B4528BF9B4649465B462846ED
:10062000829A05F0E0FE04460028ECD15A468299F1
:1006300038A807F07CFDD944C5E74FF0FF37DFF855
:1006400030910DF1160305AA06A907A805F0BCFB19
:10065000B0F10008C0F288807BD1BDF816B0BBF1C4
:10066000100F18D1BDF81440202CCAD123462846BB
:10067000069938AA05F0B7FE8046002874D12246B4
:1006800038A90DA805F0ECFB04463A4B1B688342E1
:10069000B9D10124D5E7BBF1010F37D1BDF8143032
:1006A000202BAED82846069938AA05F09CFE804635
:1006B000002859D19DF814B0BBF1200F03D94FF099
:1006C000FF384746BDE7D9F800302B4F0393039B13
:1006D0009845F4DA1DA807F026FD00211DA803F0B7
:1006E00003FF7A681DA8126857F8081B07F01FFD62
:1006F00015A91DA807F054FD5A4638A915A805F0FC
:1007000004FF0028DDD008F10108E0E7BBF1200F6D
:1007100097D17B1C95D0D9F80030BB4216DDBDF8CF
:100720001430B3F5807F7FF46CAF2846069938AA61
:1007300005F059FE8046B8B9FFB25946BDF81430ED
:10074000009738AA0DA800F019F806464FF0FF37B9
:1007500077E73CB1074B1B68B34218BFDAF800607B
:10076000344650E74FF0010844464CE70020002093
:10077000F8890000E0210020FC8900002DE9F04FFD
:100780001F46ADF54B7D6A4B804627A89DF8506308
:100790008A4691461D6807F083FC664B8AAA53F887
:1007A000364003EBC6035B6802941B6802A81C4436
:1007B0002146302306F008FA68BB029B8A9A13444C
:1007C0009C4228D1214629AA02A806F011FA10BBA2
:1007D0000DF1B00B5A46214602A806F009FA06466A
:1007E000C8B929A806F024FD029B28909C4212D18A
:1007F00033463246CDE9006B29A927A807F00DFC46
:1008000048B927A803F002FE28B929A806F010FD70
:10081000874228900AD027A807F04CFC27A807F0A9
:1008200049FC28460DF54B7DBDE8F08FB7F5807F7C
:1008300002D04FF0FF35F1E7BAF1200FF9D1494668
:100840008AAA27A803F008FE04460028F1D19DF8E3
:100850002733BC2BEDD152AFDF263D4603900CA8C9
:1008600007F061FC00210CA803F03EFE20220DF2EF
:1008700007310CA807F05BFC042203A90CA807F0C1
:1008800056FC04A90CA807F08BFC202EB146A8BF8B
:100890004FF020099DF80F30384601334A4604A92D
:1008A000A6EB09068DF80F3005F056FE002E4F44DA
:1008B000D5DC2F46294600228AAB087813F8016B55
:1008C00001327040DF2A01F8010BF6D12B7803F0DA
:1008D0007F032B7017F8016B002EAAD10134BE2CB8
:1008E000F8D195F8BE30012BA3D10CA807F01BFC62
:1008F00031460CA803F0F8FD08220F490CA807F0B8
:1009000016FC414620220CA807F011FC20220DF213
:1009100007210CA807F00BFC04A90CA807F040FC69
:1009200020220DF2073104A805F09AFA054682E765
:1009300000200020FC890000268F00002DE9F041F6
:10094000022386B00D466F460026DFF86880ADF8BA
:10095000003017F8010B01A901F0D8F90446A0B93D
:1009600001981023816802AA103905F03CFD044665
:10097000019805F037FD44B91022414602A805F060
:10098000C4FD40B12EB14FF0FF34204606B0BDE8A3
:10099000F0810126DDE7019806F01DF80423A0F19F
:1009A00008012A46019805F01EFD0446019805F04D
:1009B00019FDEAE70A8E000007B505F065FA6946F9
:1009C000FFF7C6FD38B10548452105F0FEFC0020C3
:1009D00003B05DF804FB0098FAE700BF2E8F00001B
:1009E0002DE9F041354B88B0064600200C461D68C5
:1009F00005F091F906A9C0B201F088F9002857D195
:100A0000214605F088F92C2507A9C0B205FB04652D
:100A100001F07CF9002833D02C27674306EB070848
:100A2000D8F81010069B11F0100138D14FF48072E5
:100A30000192234A08460092CDE903112A46029109
:100A4000FFF79EFD05461F4BF25906989A420CD1BE
:100A5000D8F80C20B8F808309B1806D28268934268
:100A600003D2194B1B68AB421FD02CB38268002104
:100A700005F0E3FC154A4521154805F0A6FC13E0F6
:100A8000079805F0F5FC0746079805F0ABFC6B1ED0
:100A9000EA1C13F8011FB942BED19342F9D11CB12F
:100AA0003046069905F0D4FA0125069805F09AFC1F
:100AB000284608B0BDE8F081064ADCE700200020A7
:100AC000AC4700203DB8F396E0210020718F000074
:100AD0007B8F0000698F000073B50D46002104462E
:100AE0002846CDE9001105F072FA30B3164E23689E
:100AF000B34203D1204601AA05F0FEF9E36AB342EE
:100B000004D16A460121204605F0F6F9DDE90032FC
:100B1000934288BF0193019BAB60019A294620460E
:100B200000F07CFB094B1A68002A03DD57210848B6
:100B300005F04BFC002002B070BD05F10801FFF785
:100B4000FDFEAB680193E8E73DB8F396442E002024
:100B5000A38F00002DE9F84F884691469A4600265B
:100B6000DFF88CB0234D244C0B9B9E4201D3002018
:100B70000FE00B9B40469F1BB7F5806F28BF4FF4DB
:100B800080671B4A3B4606EB0A0105F02CFC10B1BE
:100B90000120BDE8F88F0A993B465A46484671182D
:100BA00005F036FC0028F3D1144BC5F800463E444E
:100BB000C5F80446C5F80846C5F80C46C5F8104601
:100BC000C5F81446C5F81846C5F81C46C3F80046D3
:100BD000C3F80446C3F80846C3F80C46C3F81046E9
:100BE000C3F81446C3F81846C3F81C46BCE700BF58
:100BF000E4290020008001503546526E00900150DB
:100C00002DE9F0430F460021A54B87B04362A54B69
:100C100004460365084605F07EF804F12001C0B2E1
:100C200001F074F80121002005F075F804F14C0181
:100C3000C0B201F06BF80546204605F09EF9064665
:100C400068B900222046114605F040F9064600B377
:100C500000225721944805F0B8FB0123BCE0802214
:100C60005721924805F0B1FB01239E4284F8583089
:100C7000E7D194F85830042B8DF80F3000F2AF8094
:100C8000012B00F2B38000F0CA80FF2384F85830B3
:100C9000C5E0204600F0DAF90028DED002A805F011
:100CA0008DF90146204605F028FA18B13246572141
:100CB0007F48D0E702A805F08AF980F0010102AA76
:100CC0002046C9B205F002F902460028C0D102A8A8
:100CD00005F07DF9064660BB204602A9FFF7FCFE41
:100CE0009DF80F3084F85830033B012B06D830466E
:100CF00005F051FA10B1FF2384F858309DF80F30F9
:100D0000023B022B0BD8002005F033FA38B1FF2349
:100D100084F858304521674805F057FBFEE794F802
:100D20005830FF2BF6D00021204602AA05F0CEF85D
:100D300093E79DF80F30012B43D15F4B0192E26A9C
:100D4000D4F84C809A420CD10423A18E40460DEB7E
:100D50000302194405F047FB18B1052684F85860D2
:100D600087E7002003F0DCF8831E022B0646F5D847
:100D700001212046FFF734FE504B1B68984203D0F8
:100D80000128EAD10126E9E7019BB3F1807FE5D98B
:100D9000D8F8043049211E89D3F80C9048481E44E5
:100DA00005F013FB4946304603F032F80028D4D151
:100DB0004921444805F009FB4146204605F048F921
:100DC000E0E701212046FFF70BFE3C4B1B689842F1
:100DD00014BF05239DF80F3084F8583049E7052BE0
:100DE0007FF453AF002005F0D6F913E0204602A9A6
:100DF000FFF772FE94F858300546DA1E012A0CD827
:100E0000002005F0C8F9054600287FF43EAF002019
:100E100005F0AFF9054610B137E7022BF7D094F88B
:100E20005830FF2B04D14521224805F0CEFAFEE7C9
:100E3000012B10D00021204602AA05F047F80546F4
:100E400048B1E06C05F0CEFA206A05F0CBFA2846EE
:100E500007B0BDE8F08300212046FFF7C1FD06463C
:100E6000DFF85880D8F8003098420FD110220021C6
:100E700002A805F07CFB206A04F056FF3871236A53
:100E80005B683C60D8F80050BB60DAE7E06C05F0C6
:100E9000A9FA206A05F0A6FA002D08BF3546D6E764
:100EA000E4250020E421002014900000D28F0000EF
:100EB000409000006A9000003DB8F396E0210020C9
:100EC000769000009890000038B5064D04466022E8
:100ED0000021284605F04BFB21462846FFF790FEEF
:100EE00038BD00BFE42D002073B516461D4643B142
:100EF0005B79012B07D121B9204B2A681B689A42E4
:100F000017D8002418E0022BFBD12B68012B07D93E
:100F10001A4A12689342F4D8B1FA81F14909F0E70C
:100F2000EFD131B10129ECD12979023918BF012162
:100F3000E7E70021436A5C68002004F0ECFE01A9A9
:100F4000C0B200F0E3FE30B10124019805F04AFA86
:100F5000204602B070BD214620233246019805F09C
:100F600042FA04460028EFD1002DEED03468044B3D
:100F7000E41A18BF4FF0FF34E7E700BF0420002059
:100F80003DB8F3962DE9F04F07460C4685B0014673
:100F90000020164604F06BFF051E50DB3846E46D5A
:100FA00004F072FF5FFA84F94FF0000A4FF0010B72
:100FB0004FF0FF346B1E09FB03089DB9BAF1010F16
:100FC00003DD4521204805F000FA631C06D07F2C84
:100FD0002ADC40F2011301343460B380284605B0A6
:100FE000BDE8F08F6B1E00934146012338460DF19A
:100FF0000F0205F0F8F9031E019322DB01223846A7
:101000000DF10F0105F0FBFC019B40B15B4501D0E8
:101010000AF1010A9B46009DA8EB0908CDE7B4F14F
:10102000FF3F08BF2C46F5E70223803C7371631035
:1010300004F001040133013433603471CEE7072535
:10104000CCE70125CAE700BFB890000038B5816A37
:10105000426D914208D0531C8B4205D05721134852
:1010600005F0B3F9002038BD80291CD9572110485C
:10107000F6E7446A056D04EBC30405EBC305646839
:101080006D68AC4202D057210A48E9E701339A4221
:10109000EFD1914205D9436A03EBC2035B68A342D7
:1010A000F1D10120DFE700231C46F0E7DB900000D0
:1010B000139100004291000000B589B0022004A9FC
:1010C00005F00FFD9DF81020012A41D0254B26493F
:1010D000032A08BF0B469DF81320492102929DF870
:1010E0001220224801929DF811200092204A05F01A
:1010F0006CF9052006A905F0F4FC9DF81820012ADA
:1011000028D0184B1849032A08BF0B469DF81B200E
:10111000492102929DF81A20144801929DF8192045
:101120000092144A05F051F99DF81030012B13D1AB
:101130009DF81230032B0FD19DF81830012B0BD0E6
:101140000D48492105F041F9022009B05DF804FB82
:101150000A4BC0E7094BD9E70948492105F035F9A1
:101160000020F2E76E910000779100008B91000063
:101170007D910000CC910000DC9100007291000094
:10118000FB91000070B54B6814461E4A03F0FF2324
:10119000934206460D4686B02FD10B68012B2CD109
:1011A000204604A902F066FE9DF81020012A26D0F0
:1011B000154B1649032A08BF0B469DF813204921F9
:1011C00002929DF81220124801929DF8112000927F
:1011D000104A05F0FAF89DF81030032B0DD1214686
:1011E000304604F035FF204605F06EFC2046A96825
:1011F00004F05DFE204602F01DFE06B070BD064BF9
:10120000DBE700BF000100046E9100007791000051
:101210008B910000CC910000729100002DE9F04FFD
:1012200005460C467D48492189B0174605F0CDF8A2
:101230006B6A01225E6800233344BB42114602F10F
:101240000102F9D3764F2046396004F0C0FE08B39E
:10125000E86D04F007FEAB6A03F1FF380023334466
:10126000834202D208F1FF38F9E73B68434511D3C6
:1012700057216C4805F0A9F83A6808FB06F3572196
:1012800002FB0662684805F0A0F80123E37109B08B
:10129000BDE8F08F06A9022000F038FD07A905205F
:1012A00000F034FD21462846079AFFF76BFF63796B
:1012B000012B0BD1D7F80080DFF870B13B68DDF867
:1012C0001890B8F1000F11D10123236002234FF0D1
:1012D000010863713B68DDF818A0984549D950466C
:1012E00005F080F8079805F07DF8D0E72268013313
:1012F0009B1A98453AD86B6A012A196853F8380046
:1013000003EBC80353F8083CA0EB010AA3EB01036D
:10131000049311D1079B0393E368022B08D049463D
:10132000284604F095FE22464946284604F0C6FEAB
:101330002846039904F08CFE32465146484604F094
:1013400085FE049B4A4649462846CDE900A6FFF79C
:1013500001FC2146284604F047FE23680133236040
:1013600020B1DBF800300133CBF8003008F1FF3852
:10137000A4E7236898454ED36A6A4FEAC80352F837
:101380003810083B04911168DDF81CB00391D15866
:101390002A6DD0581368A0EB03092379012B38D1AB
:1013A000039B3246C91A5046059104F04FFE059939
:1013B0004B4652460091284659460196FFF7CAFB14
:1013C0002146284604F010FE0223237118B1174A63
:1013D00013680133136032464946584604F036FE1E
:1013E000DDE9032351469B1A28465A46CDE900966B
:1013F000FFF7B0FB2146284604F0F6FD23680133D1
:1014000023600123237130B1084A1368013313604C
:1014100001E0022BDFD008F101085BE71292000027
:10142000042000203B9200006A920000442E00201D
:10143000BFF36F8F72B600234FF0FF30094A03F1FC
:1014400020010133102B42F82100F8D100234FF086
:10145000FF30044A03F160010133102B42F82100F0
:10146000F8D1704700E100E038B501224FF0FF34B9
:1014700000251A4B29465A60C3F84843C3F808436D
:1014800003F580535A60C3F84843C3F80843A3F5F3
:101490005043C3F800558022C3F80843104805F0B4
:1014A00066F8802229460F4805F061F80E4B80222D
:1014B000C3F800552946C3F808430C4805F057F80F
:1014C000802229460A4805F052F80A4BC3F808451D
:1014D0004FF05023C3F8084338BD00BF004001500F
:1014E000808000508081005000900050809000501B
:1014F0008091005000700150014B1B68184700BFDD
:1015000008200020014B1860704700BF0820002011
:1015100007B50B46002102460091034800F014F97C
:1015200003B05DF804FB00BFF91400002DE9F0479B
:10153000058B04462807904611D4022905F00705BB
:1015400040F0CD80204604F066FE78B10138218B52
:10155000042811D8DFE800F0C3106D85950001293B
:101560000CBF45F0100545F02005258388F3118850
:10157000BFF36F8FBDE8F08701F0070AAA4500F0BE
:10158000A6800027B9463E46A368002B00F0BD8028
:1015900041F00801218388F31188BFF36F8FA168A0
:1015A000002900F0BB800D68002900F0B7803346A9
:1015B00052462046D1F80480C047002D76D02B68D3
:1015C00029461D46F0E701F007035A1F012A1BD8E0
:1015D000002221F00701062B276889B2C4E9002206
:1015E00009D13B4603E0628B013262831B68002B0A
:1015F000F9D141F002012046218304F00CFE0028BD
:101600007BD041F0200177E0042B0AD121F00701C3
:1016100089B22046218304F0FEFD10B141F0200183
:101620002183218B01F0070AAA4550D00027B94633
:10163000AAE7236921F0070141F00601062DD3F83E
:10164000009021832DD1B9F1000F40D041F0080165
:10165000218388F31188BFF36F8F20463949C8472B
:1016600029E021F00701236941F0040189B2042D2A
:10167000D3F804902183E6D000274FF0040A3E46B9
:1016800082E721F00701236941F0050189B2052DA8
:10169000D3F808902183D6D000274FF0050A3E46A4
:1016A00072E700274FF0060A3E466DE72B4687E7B4
:1016B000B9F1000FD1D14FF02003EFF3118883F37C
:1016C0001288BFF36F8F238B23F008032383258BAE
:1016D000EA062ED525F01003238305F00705666979
:1016E000218B002EBFF66FAF00232768C4E90033BB
:1016F00021F0070141F001012183218B4FF0000906
:1017000001F0070AAA457FF43FAF002F9BD041F0BC
:101710000801218388F31188BFF36F8F002FC7D092
:101720003D68394633465246204604F0A0FD2F4618
:10173000F4E7AB067FF51AAF25F02003238305F00D
:101740000705FFE69B6200002DE9F04F82464FF04F
:1017500000098DB01D46531E01910393039B5878D9
:101760005C1C252819D100204FF0FF381E46444646
:1017700003460236029031780396392955D81F293D
:1017800014D8002900F0F18101992520D047019952
:101790003078D04709F10209E0E7002800F0E58140
:1017A0000199D04709F101090394D7E7A1F120027B
:1017B000192AE9D801A757F822F000BF2518000020
:1017C00089170000891700002518000089170000FC
:1017D000A51800008917000089170000891700006C
:1017E00089170000F1180000251800008917000073
:1017F00005190000B118000089170000BF1800008B
:10180000DF180000DF180000DF180000DF180000FC
:10181000DF180000DF180000DF180000DF180000EC
:10182000DF18000008460136A5E7582900F0EE80D1
:10183000A1F16302D7B2172FA6D8172AA4D801A7FF
:1018400057F822F0B31A00002B1900008917000086
:1018500089170000891700000B1900002B190000E0
:1018600089170000891700000B1900008917000074
:101870008917000089170000E71900008917000088
:1018800089170000871A0000891700002B19000033
:101890008917000089170000E71900008917000068
:1018A0000B19000025200199D04709F1010955E7DE
:1018B000029A4FF0000802F0FE020292B3E7002CF9
:1018C0000DDAB8F1000F0DDA029A002A00F0458116
:1018D0000A2224EAE47402FB0414303CA3E7B8F1C2
:1018E000000FF5DB0A2202FB0812A2F130089AE78A
:1018F000B8F1000F55F8042B80F23181002A80F2F4
:1019000030815442022202928DE7682903D1682B6C
:1019100006D1482387E76C2902D16C2B00F0238184
:10192000002B7FF431AF0B467DE77A2B06D175296A
:1019300055F8046B14D14FF0000B0CE06C2BF6D073
:101940004C2BF4D1073525F00703752903F1080561
:10195000D3E9006B06D120283ED1864F013C09E037
:101960004FEAE67BBBF1000FF5DA7642824F6BEB74
:101970004B0B013C0DF12D030593002304933046DE
:1019800059460A220023FEF7E5FB049B303203F19F
:10199000FF3CCDF810C0DDF814C00CF8012DCDF8D7
:1019A00014C0B4465A46BCF10A0F72F10002064652
:1019B0008B46E4D2C3F1010B30330DEB0306B8F1D3
:1019C000000FA6F104066DDA029BD9077CD4A8EBC0
:1019D0000B03A4EB0B0413E02B280ABF674F684FDF
:1019E00004F1FF34C6E770290FD155F8042B00230A
:1019F000FAB96FF004034FF0050B624E053C604FDF
:101A0000029A92076FD4A04665E078216C2B03D12F
:101A1000002355F8042B08E04C2BF9D1073525F0AD
:101A200007031D465B6855F8082B232825D1880637
:101A300021D5554F023C002601F06001A1F1390B80
:101A40000DF12D0E02F00F01092988BF59443031E4
:101A50000EF8011D102A4FEA121141EA03714FEAF4
:101A6000131073F1000306F1FF3C08D2C6F1010B1D
:101A700006F13003A1E7454FDCE7414FDBE766465F
:101A80000A460346DEE755F8046B304604F036FD9F
:101A9000B8F1000F834602DB4045A8BFC3464FF0B4
:101AA0000008374FA8EB0B03002B92DDA4EB0804D2
:101AB000A6E755F8043B4FF0010B8DF81830013CB8
:101AC0004FF0FF3306AE9AE7A046EBE702932020E3
:101AD0000199D047029BB8F10108F7D524EAE472D6
:101AE000013C9144A41AB84606E00493029201997D
:101AF000D047029A049B9046424612F8010B0028F8
:101B0000F3D11A46013A15D5002BACBFC7EB03073A
:101B10007F425B46013B15D5BBF1000FA8BF5F4478
:101B200026464F44013E14D5002CA8BF3F1907EBB1
:101B3000080913E60493029230200199D047049BD0
:101B4000029ADFE70293019916F8010BD047029B36
:101B5000E0E701992020D047E4E70122D3E6904650
:101B600061E614465FE64C235DE648460DB0BDE8ED
:101B7000F08F00BFC0970000BA930000BC93000034
:101B80002B9E0000C4930000BE930000C193000090
:101B900008B54FF02002EFF3118382F31288BFF3F0
:101BA0006F8F00F047FC034804F028FB00F012F9A7
:101BB000FCE700BFCA930000054B03EB8000D0F8A0
:101BC000003223F0E04343F04053C0F80032704746
:101BD0000025845038B54FF02003EFF3118583F3CF
:101BE0001288BFF36F8F01211A4B1B4AC3F80015EF
:101BF00002230020C2F8D036FFF7DEFF0846FFF7C9
:101C0000DBFF7E237F20C2F80C37C2F83C39134B30
:101C1000134CC3F818010020C4F8040EC4F8080ED1
:101C200004F54824C4F81001C3F82401C3F82C01BA
:101C300003F5FF1303F58053C3F8A002C2F804179D
:101C4000C2F80419C2F8001B85F31188BFF36F8F27
:101C500038BD00BF00100050004000500020005070
:101C600000900350F8B50523194D1A4F2C781A4EE1
:101C70000134B4FBF3F303EB8303E41A04F089FEAD
:101C8000164A137873B157F82430C01A072809D8B8
:101C900033782BB95721124804F097FB0123337096
:101CA0000020F8BD00214FF050233170D3F814010B
:101CB00038B1C3F81411D3F814312C700CB90123C6
:101CC00013702C7804F065FE47F824000120E8E743
:101CD000AE480020482E0020AC480020AD4800202F
:101CE000F393000048B1054B054A1B68B3FBF2F3C0
:101CF0005843044B43F00103184770473C20002031
:101D000040420F00F089000002F016BD70B5114B83
:101D10000D461C68DCB1104B196800238B4202DBB6
:101D20006FF0010070BD224612F8106B864202D09F
:101D300014460133F2E7E06810B96FF01200F1E7E2
:101D400006F058FC0028F8D000202C60EAE76FF07D
:101D50000C00E7E70C200020088A000070B588B06E
:101D600005460C46C0B269461646FFF7CFFF00286D
:101D70001BDB0098C8B14368226802938368019511
:101D8000CDE903360023CDE906230593C56804F0A9
:101D900029FB6DB12846084901AA04F056FD0798B1
:101DA00008B9059B236008B070BD6FF01500FAE715
:101DB0006FF01200F7E700BF7F640000014803F0F6
:101DC00099BE00BF8C8A0000014910220A6070474A
:101DD00010ED00E072B6404080F31188BFF36F8FC2
:101DE00001B5FFF73FFF002802D0BFF34F8F30BF90
:101DF000BDE8014062B6BFF36F8F704772B64940CD
:101E000081F3118801B5FFF72DFF002802D0BFF341
:101E10004F8F20BFBDE8014080F3118862B6704744
:101E200037B505460C46C9B18B6810480093D1E917
:101E30000023452104F0C9FA636945210093D4E9E0
:101E400003230B4804F0C1FA4521E269094804F074
:101E5000BCFA4521A269084804F0B7FA2146284691
:101E600003B0BDE8304003F073BC00BF2594000010
:101E7000599400008D940000A194000040B2002805
:101E800007DB01234109034A00F01F00834042F8A9
:101E90002130704700E100E040B200280CDB012255
:101EA0000649430900F01F008240203341F82320F7
:101EB000BFF34F8FBFF36F8F704700BF00E100E0AB
:101EC000054B420953F82220012300F01F0003FABA
:101ED00000F01040704700BF00E100E040B2002871
:101EE00001F10101ACBF00F16040064B4FEA411126
:101EF000C9B2ABBF00F5614000F00F0080F80013DD
:101F00001954704714ED00E030BFFFF7FDBF00BF6C
:101F10000B4A08B50B4B22F07F029A60BFF34F8F3C
:101F2000BFF36F8FD3F8882022F47002C3F88820A3
:101F300003F086FC03F0CCFC00F040FA03F08CFCCC
:101F40000000000000ED00E01EF0040F0CBFEFF3F6
:101F50000880EFF30980816911F8021C0229FFD083
:101F600001B504F0B3FA01BD0446084611461A460D
:101F7000002383F30B880A4B2025A3F5205686F314
:101F80000B8883F3098863B64FF0000383F311884D
:101F9000BFF36F8FA04785F31188BFF36F8FFEE704
:101FA000B878002001B5EFF30580A0F110004FEAEA
:101FB000C0000449014409C99847BDE801400249ED
:101FC0000847000020870000CD1F0000704700BFB9
:101FD00038B5214C4521214804F0F7F9A36A9D0149
:101FE00003D545211E4804F0F0F9A36ADC0103D5AE
:101FF00045211C4804F0E9F9174DAC6A14F480142B
:1020000004D04521184804F0E0F90224AB6A180313
:1020100003D54521154804F0D8F90F4DAB6A590393
:1020200003D54521124804F0D0F9AB6A9A0303D5D1
:102030004521104804F0C9F9074DAB6ADB0303D50D
:1020400045210D4804F0C1F9AB6A20466FEA03430D
:102050006FEA1343AB6238BD00ED00E0D49400009A
:10206000F1940000099500002895000057950000A4
:102070007A950000A4950000C395000070B5234C2C
:1020800006460D462248452104F09FF9A36AD9046B
:1020900003D545211F4804F098F9A36A1A0503D512
:1020A00045211D4804F091F9184CA36A9B0510D5F1
:1020B0001A48452104F089F9A26BA36A180408D5CF
:1020C0004521174804F081F91EB1A36A23F40043A7
:1020D000A3620E4CA36A590503D54521114804F0AB
:1020E00074F9A36ADA050BD545210F4804F06DF9A0
:1020F0000020064A936A43F47F439362287070BDC0
:10210000A36A9B04F4D545210848EFE700ED00E001
:10211000F39500000E960000249600003C96000007
:102120005A9600007496000094960000B196000044
:1021300070B5264C06460D462548452104F045F964
:10214000A36AD80603D54521224804F03EF9A36AC4
:10215000190703D54521204804F037F91B4CA36A21
:102160009A0710D545211D4804F02FF9626BA36A28
:102170001B0608D545211A4804F027F91EB1A36AA9
:1021800023F08003A362114CA36ADE0703D5452127
:10219000144804F01AF9A36A980603D54521124899
:1021A00004F013F90020094B9A6AD10658BF9A6AC5
:1021B0009A6A920642BF5A6A22F400525A629A6A96
:1021C00042F0FF029A62287070BD00BF00ED00E08F
:1021D000E596000000970000249600003897000064
:1021E0005597000070970000B19600002DE9F0416E
:1021F0005C4B05465F6800268AB0C7F3080486F387
:102200001188BFF36F8F02F07F43B3F17F4F07D187
:1022100002F00C03082B14D14521534804F0D5F8E3
:10222000002635464FF00008E31E8DF80780092B85
:1022300000F28680DFE803F00A797D758484848467
:10224000848110074CBF0D460126EBE74521474826
:10225000444C04F0BAF88DF80780E36A9A0705D574
:102260004521434804F0B1F8002432E0E36A002B32
:1022700002DA45213F48F5E7E36A5B00F4D54521E2
:102280003D4804F0A2F86369AA6943F4807363616E
:10229000BFF34F8FBFF36F8F636932F8022C23F4C3
:1022A00080736361BFF34F8FBFF36F8F4DF602737F
:1022B0009A4208D0A36ADBB22BB301200DF10701CB
:1022C000FFF736FF2FE045212A682C4804F07DF8FF
:1022D0002C689DF807309BB92022294602A804F0FB
:1022E0003BF9099B002E38D0C3F3080222B96FEAEC
:1022F00053236FEA43230993204602A9FFF790FD79
:102300000AB0BDE8F081A36A13F47F4F05D0012025
:102310000DF10701FFF7B2FE05E0A36AB3F5803FB8
:10232000A2D3FFF755FE0446D3E700200DF10701C5
:10233000C6E700200DF10701ECE74521104891E7C1
:10234000104917F4F87F104A104808BF0A46A4F154
:102350001003452104F039F886E723F4FF7323F0D6
:102360000103C8E700ED00E0C2970000F29700000B
:102370000E98000034980000479800006B98000009
:102380008C98000094970000A9970000B598000071
:10239000044B5A6942F010025A615A6942F4806251
:1023A0005A61704700ED00E0EFF30880EFF3098118
:1023B00001B57246FFF71AFF01BD00BF00232021BF
:1023C0000348C2180133452B82F80013F9D1704736
:1023D00000E100E0002080F31488BFF36F8F00203D
:1023E00080F30A8880F30B88FFF78EFC00200E49EB
:1023F0000860BFF34F8F0D4880F3088800F03EF867
:10240000202080F311880A484FF40061401880F3BF
:102410000988EFF314800221084380F31488BFF386
:102420006F8FFFF775FD000094ED00E0B878002095
:10243000B8480020BFF34F8F0549064BCA6802F425
:10244000E0621343CB60BFF34F8F00BFFDE700BFD7
:1024500000ED00E00400FA05002318460649D1F813
:102460009020C2F30722934200DB7047C1F89830F6
:10247000C1F8A0000133F6E700ED00E010B572B638
:10248000002484F31388FFF7E7FF23464FF0FF3063
:102490000C4A03F120010133102B42F82100F8D13E
:1024A00000234FF0FF30074A03F160010133102B86
:1024B00042F82100F8D162B6BFF34F8FBFF36F8FA0
:1024C00010BD00BF00E100E00121024B024A0348B9
:1024D00000F016B90000072000200020948A0000B8
:1024E00010B50C7A0B6804F01F0223F01F031A4387
:1024F000CB68640923F01F03054943EA440343F012
:102500000103C1F89800C1F89C20C1F8A03010BDAB
:1025100000ED00E030B50C684B6885B00A894D8944
:102520000094013B24F01F04234402F01F0242EAFE
:10253000451223F01F03072804468DF80820039353
:1025400009D902464521064803F03FFF6FF0150404
:10255000204605B030BD6946FFF7C2FFF8E700BF6F
:10256000D19800002DE9F04F8946144606464FF0F9
:102570000008544D85B0C84527DAD6F804A0BAF152
:10258000000F44D0BAF11F0F18D91AF01F0F15D140
:10259000D6F800B01BF01F0F10D1584603F0A5FF6E
:1025A00007460AEB0B00013803F09FFF874210D06B
:1025B0006FF015073A464521434802E0424645215F
:1025C000424803F002FF6FF01504204605B0BDE855
:1025D000F08F17F1160FEDD0BC42EBDDC5F8987007
:1025E000D5F89C10C5F89870D5F8A03021F01F01DF
:1025F00043F01F0BD6E900321A44994202F1FF3A28
:102600001DD1D34507D13146F8B2FFF783FF08F15A
:1026100001080C36AFE73146C5F89870D5F89C3004
:1026200022F01F0203F01F031343C5F89C30E0B2F1
:10263000FFF770FF10F1160FC5D0441CE7E7C5F88F
:102640009870D5F8A020013B23F01F0302F01F0271
:102650001343D3453146E0B2C5F8A030E8D0FFF7C8
:1026600059FF10F1160FAED0C5F89870D5F89C2020
:102670009DF808300BF1FF3B62F304038DF808303E
:10268000D5F8A0309DF808205B0863F34712D6E91F
:1026900000310B44009323F01F0301305B44A3EB94
:1026A0000A03C0B223F01F0307288DF80820039304
:1026B00003D902464521064883E76946FFF710FF24
:1026C000BBE700BF00ED00E024990000FC9800008B
:1026D000D19800000522044BC3F89420BFF34F8F1C
:1026E000BFF36F8F704700BF00ED00E0BFF35F8F57
:1026F0000022024BC3F89420704700BF00ED00E0B9
:1027000010B5034C2278FFF72DFF207010BD00BFDD
:10271000AF48002038B50E4D2C68082C15D8002085
:10272000FFF7E4FF0B4B0C4AC3F8C020844205D1ED
:102730000A4B00201C70FFF7CDFF38BD696801EB24
:102740000011FFF7CDFE0130F0E74FF0FF30F4E766
:10275000A08A000000ED00E0AAFF4400AF4800207E
:10276000014B1860704700BF10200020084B70B567
:10277000C31A0D4607499B10044659434022064898
:1027800003F01DFF2B4601462046BDE87040184768
:10279000702E0020B76DDBB690860000402373B525
:1027A0000B4C0093041B0B460D460A49A4106143D1
:1027B0000646094A094803F02EFF011E05DA304695
:1027C0002B4602B0BDE87040184702B070BD00BF94
:1027D000702E0020B76DDBB6876600009086000083
:1027E00010B54FF02003EFF3118483F31288BFF389
:1027F0006F8F074A136823F00201DB07116002D4D0
:10280000012005F086FE84F31188BFF36F8F10BDA1
:10281000102F00202DE9F843002201210646052053
:10282000FFF75CFB114802F073F8114B984219D185
:1028300005F0FEFD00244FF01C090C27DFF8348062
:102840003569414609FB045003F035FD002807DBDC
:10285000012307FB04551C44042CAB67F0D1002076
:10286000BDE8F8836FF00400FAE700BFAD28000070
:102870000000AD0BC88A000001460C23002270B591
:102880004B430848C4187833D4E91C5618442267CF
:1028900003F082FE2DB132462B46BDE8704002485F
:1028A000184770BD702E002090860000052811D8B2
:1028B000DFE800F0030E10100C0A074B986F10F0C1
:1028C000070007D1FFF7D8BF0220FBE70320F9E795
:1028D0000120F7E7704700BF702E002008B54FF0C9
:1028E0002003EFF3118183F31288BFF36F8F124A35
:1028F000136843F002001060DA0708D481F31188EE
:10290000BFF36F8FBDE80840012005F0A3BD4FF075
:102910005023D3F80C24D3F80C34D307EED5074852
:1029200003F03AFE81F31188BFF36F8FBDE80840D2
:102930000020FFF7A1BF00BF102F0020E82E0020CD
:102940002DE9F843012207463449D1E8EF3FC1E8B9
:10295000E02F0028F9D133B9314932484B60CB60C0
:102960008A6003F0BBFC7B1E012B2DD8012F07D101
:102970004FF05023D3F81C3403F00303022B23D071
:1029800005F047FE054608BB274B1B78F3B14FF017
:10299000502302220646C3F808234FF050244FF07C
:1029A0000008DFF88890D4F81834D4F81824D2033B
:1029B00016D503F00303022B01D0012F10D13DB334
:1029C00086F31188BFF36F8FBDE8F8834FF02003C3
:1029D000EFF3118683F31288BFF36F8F0125DCE7D5
:1029E0003046FFF70BFAD4F81835DBB2012BDAD1F9
:1029F000D4F80421002AD6D0C4F80481D4F80421E4
:102A00000222C4F818252022C9F88021A360CAE751
:102A10004FF050230222C3F80423D5E76C2E002088
:102A20005C2E00208C2E0020B548002000E100E044
:102A300008B5074805F0DEFD38B10648FFF790FEFF
:102A40000448FEF75FFD002008BD6FF01200FBE7B1
:102A5000D8860000592A00000A2838B50446074DD8
:102A600004D1AB680D2128465B689847AB680348E2
:102A70005B68E1B29847204638BD00BFD8860000A9
:102A800030B5406801F01F04057BB2F5001F85B02A
:102A900044EA451405D1204602F0EAF9002005B0C9
:102AA00030BD0025B2F5800FCDE9025514D1B3F148
:102AB000007F0CBF042305238DF808300023204637
:102AC000194602AA02F012F81F4B984238D1012190
:102AD000204602F087F9E1E7B3F1C06F25D0B3F1EA
:102AE000007F14BF012302238DF808308368CB4098
:102AF000D907E3D4B2F1A07FE0D1144A14486109A8
:102B0000012908BF024604F01F03803352F8233026
:102B1000DB07D3D40DF107052946204602F00EF954
:102B20000C4B984203D00395C8E70323DCE7284603
:102B300002F052F9044B9842F5D06FF00B00AEE76B
:102B40006FF01500ABE700BF0000AD0B002584500F
:102B5000002884500400AD0B10B502F02DF9044696
:102B600068B902F001F9084B98420AD1214607489A
:102B700002F0DEF8224605210D20FFF7AFF9002014
:102B800010BD6FF00400FBE70000AD0B912B0000BF
:102B90004209034670B502D0012A17D070BD0D4E10
:102BA000326951680029F9D0012503F01F030C6830
:102BB0009D400029F2D08A682A4002D030464B68F6
:102BC00098472CB1236821461C46F2E7024EE7E7FE
:102BD0002346F8E7C0860000A88600002DE9FF41E3
:102BE000476801F01F053B7B144645EA43150E4636
:102BF00028460DF1030102F0A1F814F4403F80468D
:102C00000BD1284602F05CF93C4B984503D19DF866
:102C1000030002F0DBF800200CE0002328461946F0
:102C200002AACDE9023301F061FF344B984204D08F
:102C30006FF0150004B0BDE8F081804503D19DF828
:102C4000030002F0C3F8A30349D540F20633234042
:102C5000B3F5837F19D00CD8062B17D004D8ABB1AD
:102C6000022BE5D1042311E0B3F5807FE0D10123ED
:102C70000CE040F20222934226D0B3F5407F25D0EB
:102C8000B3F5007FD4D1022300E007238DF8043090
:102C900084F48033C3F30043E0068DF805304CBF65
:102CA0000323C4F3401321038DF8063010D501230C
:102CB0007A68B34093600022284601A901F0C4FF5E
:102CC0000E4B9842A7D0B3E70523DFE70323DDE7E8
:102CD000620341BF01237A68B340D360EBE7E306A8
:102CE0004FF000034CBF0324C4F340141A46284697
:102CF00001A98DF8044001F0F9FEE1E70000AD0BF9
:102D000000F1744000F5A6000A289ABF024B33F97F
:102D100010006FF00F007047F48D0000024B0B6045
:102D200001231360704700BFD08B0000004870473C
:102D3000648B000010B5084C23785BB90269074921
:102D4000406802F015FBFFF7DBFFB0FA80F35B0988
:102D5000237010BD0020FCE7B24800205767000038
:102D600037B50D464168B1B1D1E900138468A4B10B
:102D7000D4E9002494B18BB19C4208D10133092BD2
:102D800000780ED902465721104803F01EFB6FF061
:102D9000150003B030BD0B46E8E72246013323445B
:102DA000EDE78DF8013040F20113ADF80230002359
:102DB0008DF8000068468DF804308DF8055002F05B
:102DC000B1FB03B0BDE83040FFF79ABFAD990000FA
:102DD00010B5084C02F0E6FBA04205D102F004FC5D
:102DE0000022054B1A7010BD4CF2503005F017FC54
:102DF000F0E700BF0000AD0BB24800200C4B10B54F
:102E0000994204460FD14FF02003EFF3118083F372
:102E10001288BFF36F8F237833B10023237080F3C0
:102E20001188BFF36F8F10BDFEF7E8FFEBE700BF1F
:102E30000000AD0B2DE9F04F81460E461C46904632
:102E400085B07AB1002B00F092800029426803DB44
:102E50009269CB1893420BD9234632464521454807
:102E600003F0B3FA6FF01505284605B0BDE8F08F02
:102E7000FFF760FF0546002876D1754205F003058F
:102E8000A54228BF2546D8F1000303F0030308F04C
:102E9000030758BF5F427F4207F00307A74228BFDE
:102EA0002746631BE41B24F0030423F0030AA24516
:102EB000C8BFA24603F0030BC8BFA3EB040BBAF1D3
:102EC000000F19D008EB07037219514618460193F9
:102ED00005F088FB04460146D9F81000FFF78EFF85
:102EE000254A94423CD1BD4206D0019B5246194628
:102EF00008EB050003F019FBBDB1C5F1040704217F
:102F0000F21B02A805F06EFB04460146D9F810003A
:102F1000FFF774FF184B9C4222D107F108032A46A1
:102F200040460DEB030103F017FBBBF1000F16D079
:102F30000821721952440DEB010005F053FB0446C1
:102F40000146D9F81000FFF759FF0B4B9C4207D1FF
:102F50000AEB05005A4602A9404403F0FDFA064C6C
:102F60002046FFF7CDFE0546FFF732FF7CE71D4602
:102F70007AE700BFD59900000000AD0B2DE9F347BB
:102F800006460F461D4690469AB193B1042B01D9CF
:102F90009A070ED1BB070CD1002F726803DB926930
:102FA0007B1993420BD92B463A464521354803F00D
:102FB0000CFA6FF01504204602B0BDE8F0873046E9
:102FC000FFF7B8FE044650B903F0E4FB044648B1ED
:102FD000012003F0DFFB2046FFF792FE0446FFF7D7
:102FE000F7FEE8E7032D1ED804213A460DEB010059
:102FF00005F0F8FA044601463069FFF7FFFE224B60
:103000009C4233D12A46414601A803F0A5FA042187
:103010003A460DEB010005F0E2FA0446014630693C
:10302000FFF7ECFE22E008F06043B3F1005F24D02C
:10303000DFF854A0042DA94628BF4FF004094146EB
:103040004A4601A803F088FA04213A460DEB010034
:1030500005F0C5FA044601463069FFF7CFFE544536
:1030600004D1B5EB0905C8444F44E3D1012003F076
:1030700091FB002C08BF0446ADE73A46294640467E
:10308000C9E700BF239A00000000AD0B2DE9F84FFF
:1030900015460A1E8046D0F8049005DBD9F8183092
:1030A00051199942174609D92B464521334803F057
:1030B0008CF96FF015042046BDE8F88FC2F30B02BF
:1030C000002DF6D0C5F30B031343F2D1FFF732FE08
:1030D0000446F0B903F05EFB0446D0B9DFF8A0A0C7
:1030E000D9F81830AB4217D105F07FFAAB46064647
:1030F0003146D8F81000FFF781FE564532D1B5EBC6
:103100000B055F44ECD1012003F044FB002C08BF09
:103110000446FFF75DFECEE7B5F5803F09D3BBB2AD
:1031200053B93946012002F0ADFA4FF4803B064610
:10313000DEE7B5F5805F09D3C7F30B0030B9394638
:1031400002F0A0FA4FF4805B0646D1E72B463A46E0
:1031500045210C4803F039F90B49D8F81000FFF766
:103160004DFE094E2B4609483A46452103F02DF9FC
:103170003046FFF7C5FD0446C5E700BF729A000060
:103180000000AD0BC19A00000400AD0BE49A0000F2
:103190004FF0502302222DE9F041C3F8B8254368CF
:1031A0008AB01E6A05460021304607AA03F0F5FBE7
:1031B000041E2EDB079B32681979186800F0DCFCCE
:1031C000041E26DB002201212B20FEF787FE6E68FD
:1031D0002A693046474902F0CBF8FFF791FD041EFB
:1031E00017DBF37A023B012B17D996F80A80A8F176
:1031F0000308B8F1010F8CBF4FF000084FF0010831
:1032000003F0ADFA041E0BDA224645213A4803F0DA
:10321000DCF820460AB0BDE8F0814FF00108EFE786
:10322000E2B2C4F38014A04504AE05AF26D000235B
:10323000012182F0400207A8CDE90613ADF8103055
:1032400005968DF8102009938DF81C100897FFF74C
:1032500087FD041E0CD0DCDA2849294A2346B8F140
:10326000000F08BF0A462748452103F0AEF8D0E713
:1032700003F075FA041EEFDBE307F9D4FFF7A8FDAE
:103280004FF003080023CDE9068308939F232846C7
:1032900005968DF81C300997FFF74CFD014620B1CB
:1032A000FFF796FD6FF01204B3E707A8FFF758FD8C
:1032B0000446FFF78DFD002CF4D16D68424631467F
:1032C00005F11C0003F021F904460028A1D0AB7FD2
:1032D000452103936B7F9DF8102002932B7F0A48B2
:1032E00001939DF8123000939DF8113003F06DF8B2
:1032F000D8E700BF576700000D9B0000079B000048
:1033000079910000229B0000389B0000024B0B606B
:1033100001231360704700BF2C2F00200048704726
:10332000EC8B000010B505F054F9034C206005F05B
:103330004DF96060002010BD2C2F0020F8B50E461E
:10334000144605F043F921460546304603F037FAA6
:10335000374600B3B6FBF5F305FB136323B9B4FBA3
:10336000F5F305FB134343B12346324645210C4890
:1033700003F02BF86FF0150002E0A54201D9002000
:10338000F8BD05F023F90546384601F0AFFE641B91
:103390002F44F9D1F3E72346324645210148E7E7B8
:1033A000859B0000A99B0000F8B50E4619463046E3
:1033B00017461D4603F003FA40B92B463246452115
:1033C000114803F002F86FF01500F8BD46EA050455
:1033D00014F0030404D02B46324645210B48F0E795
:1033E0004DB12B19032BA6EB040006D8084AD2F8DE
:1033F0000034DB07FBD50020E7E73B1B196801F031
:1034000093FE043CEDE700BFA99B0000CB9B0000AE
:103410000090035070B50D461946284616461C46C6
:1034200003F0CDF940B9084823462A46452102F069
:10343000CCFF6FF0150070BD24B1224629463046FE
:1034400003F08AF80020F6E7A99B0000F8B50446CF
:103450000D46076905F0DDF890B92C4B1B787BB160
:103460006426606803F040FAE0B9012004F01BFF15
:10347000013EF6D1F4E786F31188BFF36F8FEFE7D3
:103480004FF02003EFF3118683F31288BFF36F8FA1
:103490006068314603F028FA90B986F31188BFF3CB
:1034A0006F8FEDE74FF02003EFF3118683F312885F
:1034B000BFF36F8F6068314603F016FA0028DAD048
:1034C0003B691D70626838691368C3F844050120C0
:1034D000C3F848050020C3F82001D3F82051C3F8F1
:1034E00058015268D3F85801D20608D508206268FE
:1034F0001268C2F800054FF48002C3F804230122C9
:103500009A6081F31188BFF36F8FF8BDB548002032
:10351000F0B54B79012B29D0032B24D110278B79BF
:10352000032B20D1CE790EB1012E1CD10A79012AAC
:103530001ED0022A20D0B2B914460B684568B3F5F4
:10354000164FD5F800C06ED033D8B3F5165F6DD0E6
:103550001CD8B3F5966F6BD010D8B3F5967F6AD0B0
:10356000B3F5167F6AD06FF085005BE00027D6E7E1
:103570004FF480740E22E0E70024FBE7B3F5166FEA
:103580005FD0B3F5965FEED1384B3CE0B3F5E14F39
:103590005AD007D8B3F5615F58D0B3F5964FE2D152
:1035A000334B30E047F61225AB42DCD14FF4000339
:1035B00029E0B3F5613F4BD013D8B3F5963F4AD01D
:1035C00009D84DF6C025AB4247D0B3F5614FCAD1FB
:1035D0004FF46B0317E0B3F5E13FC4D14FF0EB7349
:1035E00011E0B3F5612F3BD008D8224DAB423AD061
:1035F000B3F5E12FB7D14FF0E86304E01E4DAB42C5
:10360000B1D14FF080530569CCF8243543683A4373
:103610001B6834432243C3F86C252B1D03C983E880
:1036200003000020F0BD4FF41D03ECE7134BEAE765
:103630004FF49E23E7E74FF4A033E4E74FF41C3345
:10364000E1E74FF41D23DEE70D4BDCE70D4BDAE736
:103650004FF06C73D7E70C4BD5E74FF46503D2E717
:103660004FF07063CFE74FF08063CCE700B01300FA
:1036700000A04E0090D0030040420F0000502700F1
:1036800000C0750000F03A0000903A012DE9F743C0
:103690008046002201210820FEF720FC0820FEF7CA
:1036A000EDFB0021D8F80470D8F810603C6801AA3E
:1036B000C4F80015C6F80080D7F80C90484603F00F
:1036C0006CF9051E1EDB019BD9F8002019791868DA
:1036D00000F052FA051E15DB4046311DFFF718FFBA
:1036E000054678B97B6899071DD506F1180001F0E9
:1036F00077F9214B984209D04521204802F065FE18
:103700006FF00405284603B0BDE8F083337E43F034
:103710000043C4F8A031C4F88C300123327E9340BA
:10372000174AC2F804350823C4F800353B7A53B968
:10373000C4F81031D4F810317369C4F8343501235A
:10374000C4F8383523607B689A075CBF4FF48073F8
:10375000C4F804337B68DB0644BF4FF48003C4F82D
:1037600004333369C4F844350023C4F848350123D1
:10377000A360E360C6E700BF0000AD0B0F9C000034
:10378000007001500123834070B5DC430B4AD2E83E
:10379000EF1F01EA0405C2E8E65F002EF7D14FF4FF
:1037A000803282400648C0F80823BFF35F8FBFF322
:1037B0006F8F0B4214BF0120002070BD382F0020F6
:1037C0000050015070B40E4922F07F46D1E9003418
:1037D000D01AC31844F10004C1E90034A6F500135F
:1037E000B3F5400F09D2074B1B681A0A1B069C1938
:1037F000054B42F10005C3E9004570BC02F0C8B8B2
:10380000482100203C2F002050210020D9B1012365
:103810000D4A8340D2E8EFCF4CEA030CC2E8E1CF77
:103820000029F7D14FF48033084A8340C2F80433AB
:10383000074BD3E8AF3FC340DB0742BF4FF4001252
:10384000044BC3F800217047382F0020005001506E
:10385000342F002000E100E00D4B1868010A00063B
:10386000BFF35F8F0B4BD3F80435181841F10001FB
:10387000B3F5801F0AD2084BD3E90023904271EBC5
:10388000030303D210F1807041F10001704700BFC3
:103890003C2F002000500150502100202DE9F74F0F
:1038A00016461F460446FFF76DFF0090FFF7D4FF52
:1038B000B04271EB070350D2384B301A67EB01016D
:1038C000984271F1000165D2354B03EB0413D3E943
:1038D00002239F4208BF964249D04FF480393149B4
:1038E00009FA04F9204626F07F4BC1F8489303F00B
:1038F00044F84FF0030A584604F15005AD00ADB24C
:1039000005F1502504F5A873274A05F58035019384
:10391000DDF804C020F07F4341F82C30C1F8449317
:10392000D1F80485A0EB0800033820F07F409042D6
:103930001DD9286860B1D1F80485A8EB0B0020F0F0
:103940007F40B0F5000F12D9204603F016F8164A52
:103950000AEB08000AF1010ADAE70123134AA3403F
:10396000D2E8EF0F1843C2E8E10F0029F8D1002593
:103970000B490C98230101EB0412C850C2E90267FD
:103980000D9B536020460099FFF740FF284603B087
:10399000BDE8F08F6FF01505F4E700BF010080006F
:1039A0003821002000500150FDFF7F00342F0020FF
:1039B00073B500244FF0FF304FF0FF31164D174B19
:1039C000C5F80845C3E902014FF4803302264FF4DD
:1039D0000012C5F80433124B0121C5F80463152009
:1039E000C3F880212246FEF779FA1520FEF746FA41
:1039F00001230C4AAB602B6013600B4B0B4A009306
:103A0000204600230194FFF749FF3046FEF798FF58
:103A1000204602B070BD00BF005001503821002088
:103A200000E100E0382F0020C5370000FFFF7F00D5
:103A30002DE9F7432E4BD3F8042390070BD5D3F889
:103A4000042142B10022C3F804212A4AD3F80431E8
:103A5000136801331360264AD2F80433D90327D5FB
:103A6000254BD3E8EF1F21F00100C3E8E40F002C41
:103A7000F7D1CB0702D4D2F84031CBB100251C4C92
:103A8000C4F84051D4F84031FFF7E6FE4FF0200370
:103A9000EFF3118283F31288BFF36F8F174BD3E9D3
:103AA0000267B042B94106D282F31188BFF36F8F2B
:103AB00003B0BDE8F0834FF0FF38D3E900104FF0BA
:103AC000FF391D60C3E902894FF48033C4F84833DD
:103AD000C4F84051D4F8403182F31188BFF36F8F9E
:103AE0000029E5D0009032463B4628468847DFE76C
:103AF000005001503C2F0020342F0020382100209E
:103B0000431C13B521D0012821DD124A124B9042EB
:103B1000D4BF04461C46FFF79FFE104B0E49D3E965
:103B20000023801AB0F5000F28BF002404448C4203
:103B300028BF0C4600200A49A2180190009143F1C9
:103B40000003FFF7ABFE02B010BD034CE3E7012416
:103B5000E1E700BFFEFF7F00FFFF7F00482100205C
:103B6000C537000008B5FFF777FE024B1B68C01A87
:103B700008BD00BF482100204FF0010C2DE9F0479F
:103B80005B4E5C4F00EB8101814202D10020BDE819
:103B9000F087046804F07F03C4F343257F2B4FEACA
:103BA000144408BF4FF0FF33222C00F29D80DFE861
:103BB00004F0122328422B3E429B9B9B9B45729B09
:103BC0009B9B9B9B9B9B9B9B757D80839B9B9B86D1
:103BD0008C8F92959800C2F80C354FEA5318B8F1C3
:103BE000010F14BFB646BE4603F01F040CFA04F4DE
:103BF000CEF80840012402E0C2F814350024A6469D
:103C000023E0C2F80835E8E70024C2F808354FEA97
:103C10005319B9F1010F14BFB046B84603F01F0E97
:103C20000CFA0EFEC8F80CE04FF0010E0DE0C2F8E1
:103C30000C350124EBE7C2F81035DFE7C2F8083590
:103C4000002DDBD100240625A64650F804AB03F076
:103C50001F090AF40058B8F1000F4FEA53131CBFB4
:103C600001244FF0000E012B0CBFB846B04608EB04
:103C70008908D8F80032CAF3C11A03F0E0492B02D0
:103C800043EA8A0343EA0E0343EA440343EA09038F
:103C9000C8F8003278E7C2F80C35D1E7C2F86035D1
:103CA0000468C4F38034002CC3D096E7C2F86435AE
:103CB000F6E7C2F86835F3E7C2F86C35F0E7C2F80A
:103CC000243501244FF0000EBFE7C2F8283584E701
:103CD000C2F83035F5E7C2F83435F2E7C2F83835C6
:103CE000EFE7C2F83C35ECE76FF085004FE700BF27
:103CF000002584500028845040EA0103C3F30D03DB
:103D000030B58BB940F21515094C890BC0F38730DB
:103D1000994201D1002030BDC218D2B202F5C07262
:103D200044F822500133F3E76FF01500F3E700BFCA
:103D3000003000500348452108B502F046FB002042
:103D4000FEF778FB4D9C00004FF000531868054BC0
:103D5000984205D0044B98420CBF012002207047C6
:103D600000207047B6B3B4B55DCE03F138B5144644
:103D700001234FF05022C2F8143608B301B34FF0BC
:103D8000005399604FF408411A4DD960C3E90050BF
:103D9000002349211848C2F8143602F016FB34B348
:103DA000164D284604F03BFCFFF7CEFF04460028E2
:103DB000F7D002280ED14521114802F006FB07E09A
:103DC0006FF0150249210F4802F0FFFA6FF0150459
:103DD000204638BD4FF0502301224921C3F8142654
:103DE000094802F0F2FA0022084BC3F840240024EC
:103DF000EEE700BFB6B3B4B56F9C000040420F00C1
:103E0000B09C00008B9C0000D09C00000030005053
:103E10001022034BC3F840240122FFF7A7BF00BFC5
:103E2000003000504FF48272014BC3F800277047F6
:103E30000030005030B5816885B0103921F007049A
:103E4000054602F015FB10220146684602F08FFB82
:103E500010226846064902F07FFB10236A4621467D
:103E6000284602F0D5FA003818BF012005B030BD51
:103E70000A8E000030B50D46816887B0102302AA73
:103E80001039044602F0AFFA002802DA012007B028
:103E900030BD1022204602A902F0B1FD00283AD11F
:103EA00010221E4902A802F030FB00280CBF01239B
:103EB00002232B70204602F08EFD012301460DF1F6
:103EC0000702204602F08FFA0028DFDB9DF807305A
:103ED000204603F00F021B096A702B7101220DF1BD
:103EE000070102F08CFD10B96B78042B03D9012374
:103EF0006B7000232B71A2682046183A22F007024B
:103F0000083AA91C02F08EFD0028BFD12046E91C0A
:103F100002F0E1FDBBE70323CBE700BF0A8E000000
:103F20007FB505466946022002F0DBFD044610B16C
:103F3000FF2004B070BD052002A902F0D2FD0128C7
:103F400036D12A464921284802F03FFA274B8DF8FE
:103F50000C40029300229DF800509DF80860244C0C
:103F60002946207802F03DFD48B33146607802F0E2
:103F700038FD20B3A378042B03D09DF80310994299
:103F80001DD1E378042B03D09DF80B10994216D174
:103F90002379042B0FD16379022B1BD1154A1648C4
:103FA000492102F012FA6079831E022BC1D9BFE7C2
:103FB0000028CFD0BCE79DF802109942EBD0013227
:103FC000032A04F10604CBD10C48492102F0FDF983
:103FD0000120AEE7032B05D0094A0A49042B08BF8C
:103FE0000A46DCE7084ADAE7149D000003010303F0
:103FF000879D0000F69C00005F9D0000729D000000
:10400000FB9C00000D9D0000F19C000001680E4A21
:104010000346914215D1C169A2F11022A2F1EF121B
:1040200091420ED18268012A0BD8C26812B101698F
:104030008A4206D0586928B19B691B1A58425841D8
:1040400070470120704700BF55AA00FF70B50D4BA7
:104050009E68A6B13046FFF7D9FF044678B9F368E9
:104060006BB935690DB9204670BD2846FFF7CEFF04
:1040700028B9EB68B34202D12E462D69F2E701243C
:10408000F1E700BF402F00202DE9F8433F4F3C6887
:10409000D4B1BC68C4B100284AD0002948D001FB83
:1040A00000F5B5FBF0F0884242D1281D40D8A907A1
:1040B0000DD025F003060436FC6803E06368B342C4
:1040C00038D2A469002CF9D12046BDE8F8832E46E9
:1040D000F2E7FB6041E006F120016318203A5A60E4
:1040E0000022C3E902242A4822691A616050294942
:1040F000D96102B1D36062695A61A1699961AAB1BB
:1041000093619A6902B153614FF001092361002361
:10411000C4E90169C4E905333B69DB072ED5FFF724
:1041200095FF58B31C4B48461B6826E0FB60E8E748
:104130000024C9E7A3681BB1174B01201B689847EF
:10414000626804F12008921B232AC4D80123A360CB
:10415000D4E90523002ABCD09361A3690BB162693D
:104160005A610023C4E905333B69DA0706D5FFF736
:104170006DFF18B10120084B1B6898472A460021A3
:104180004046444602F0F3F99EE700BF402F00206E
:1041900055AA00FF669911EE3020002070B5054643
:1041A000002800F08880444E3368002B00F08380A4
:1041B000B268002A7FD0834203D8726813449842C1
:1041C00003D33E4B01201B689847A5F120042046ED
:1041D000FFF71CFF18B1394B01201B68984755F8B1
:1041E000183C012B03D0354B01201B689847002356
:1041F00045F8183C55F8143C3BB39A682ABB55F86F
:104200001C2C02F120015A680A445A6055E9053213
:104210001A6155F8145C2B6903B1DD60202200217E
:10422000204602F0A4F9286910B18368002B2ED033
:1042300033699B073FD5FFF709FF00283BD0BDE856
:1042400070401E4B01201B68184755F8100C0028C1
:104250002AD0836843BB4268636813442033636099
:1042600003692361D4E905239AB9CBB94369636132
:104270008269A261B3B19C61A36903B15C612369E6
:1042800003B1DC602022002102F071F9D0E72C4656
:10429000E1E79361A369002BE8D062695A61E5E721
:1042A000F360F7E7F460E7E7F36845F8083C03B12B
:1042B0005C61F460BCE770BD402F0020302000201E
:1042C00038B50C46142200210546134802F04FF978
:1042D0001249134800F034F8232C1CD915F00303BD
:1042E0001FBF043CE418C3F10403ED18224600216B
:1042F000284602F03CF9084B0A49C3E90054203C27
:104300009D606C609A6811609A68A1F11021A1F11A
:10431000EF11D161DA6038BD402F00209D410000CF
:104320008940000055AA00FF014B1B68184700BFD9
:1043300038200020014B1B68184700BF34200020A4
:10434000024B1860024B0020196070473820002093
:1043500034200020F8B500F10806476804463046CE
:104360000D4602F065FF87424BD16368B3F5807F4D
:1043700047D80021304603F0C6F8002841DD00216F
:10438000304602F027FFE0B345B9294604F1140096
:1043900003F0B9F8002834DD0020F8BD04F12C0545
:1043A0000021284603F0AFF800282ADD0021284626
:1043B00002F010FF28B304F138050021284603F06D
:1043C000A2F800281DDD0021284602F003FFC0B13D
:1043D000002104F1140003F096F8002811DD0021FB
:1043E00004F1440003F08FF800280ADD002104F1F5
:1043F000500003F088F8002803DD002104F15C0080
:10440000C6E70148C9E700BF80BFFFFF70B50021C4
:104410000446FFF79FFF054610B10E4D284670BDBC
:1044200004F10806304602F0E5FE7F28F5D9143481
:104430002946204602F0CEFE0028EED0204602F0AB
:10444000D9FE0128E9D93146204603F01BF800289F
:10445000E4DBE2E700BEFFFFF0B50C4687B00021C9
:1044600005461646FFF776FF002839D103A802F06B
:1044700007FE21466A6803A802F0E0FE044618B170
:1044800003A802F003FE0CE005F10804214603A88E
:1044900002F0F8FF002807DB03A802F0F7FD6FF039
:1044A0000304A4F5854418E005F1680303A96F68C7
:1044B0000846009305F11402234603F03EFB044630
:1044C0000028DDD13A46314603A802F0D8FE044662
:1044D00003A802F0DBFD002CE3D1204607B0F0BDBD
:1044E000004CFAE780BFFFFF234A2DE9F041B1F10C
:1044F000000818BF9646214A214918BF944602F188
:10450000794208BF8E4602F574021E4902F5016227
:1045100008BF8C461C4918BF11461C4A1C4F18BFC7
:1045200017461C4A1C4E18BF164602F1D14202F52E
:10453000C01202F51E62194D18BF1546184A0346EF
:10454000184C194818BF1446A2F11162A2F50C22AA
:10455000A2F28E2218BF02460020C3E902ECC3E992
:104560000000C3E90417C3E90665C3E90842C3F8BC
:104570006880BDE8F08100BFD89E05C107D57C36B4
:1045800067E6096A85AE67BB72F36E3C39590EF770
:104590003AF54FA5310BC0FF7F520E518C68059B39
:1045A000A78FF964ABD9831FA44FFABE2DE9F04F52
:1045B000D1B00DF58E7B5A46031D019300F1240303
:1045C0000393019B53F8040F42F8040F0398984299
:1045D000F8D1DDE948074FF000094F9B4CAD02933D
:1045E000DDE94AE30493424B06AA059395E82011BE
:1045F000B9F10F0F63D84C780B78240444EA0364B4
:10460000CB7823438C7843EA04234FEAF52A8CEADB
:104610000804059E8AEAB51A2C408AEA756A84EA7B
:104620000C04544456F804AB936054442344029C55
:104630004FEA703A234440EA070405968AEAB00A32
:1046400004EA0E0400EA07068AEAB05A34435444E6
:1046500009F10109DDF810A0B9F1400F9A4402F107
:104660000402234401F10401CDF808C0CDF810E0A4
:104670001ED1CDE90634CDE94E8CCDE94CA5CDE96E
:104680004A7ECDE94830019A52F8043F01925BF826
:10469000042F1344019A1360039B9342F3D106A89D
:1046A0004FF4947101F02EFA002051B0BDE8F08F64
:1046B000BE46C4460746A8461846554698E71368BE
:1046C00052F8384C4FEAF34A8AEA734A8AEA932A44
:1046D00052F8143C52F8346C234452F8344C53448E
:1046E0004FEAB44484EAF61484EAD60423448CE7FF
:1046F0003C8C00004FF47F03D3F83021D3F83431E1
:10470000072A05D1023B032B02D8024AD05C70472E
:10471000002070479D9D00004FF05023D3F858258E
:10472000034B02F00302D340024A1360704700BFFC
:104730000020A1073C20002008B5FFF7DBFF58B19F
:104740004F4BD3F8202A3AB90D21C3F8201A012182
:10475000C3F81C19C3F81C290022D30003F57F03FA
:10476000D3F80013013107D0D3F800130132D3F886
:104770000433202A0B60F0D1FFF7BCFF002876D16C
:10478000FFF7B8FF40B13F4B3F4AC3F830254FF029
:1047900050230122C3F858254FF47F03D3F830216A
:1047A000D3F83431072A09D1023B032B06D8374A04
:1047B000D35C1BB10022364BC3F84C25FFF79AFFA0
:1047C00050B14FF05023D3F80024D10742BF00224C
:1047D000C3F81421C3F818214FF47F03D3F8302114
:1047E000D3F83431072A09D14FF05023D3F80024ED
:1047F000D20744BF6FF00102C3F80024FFF77AFF2D
:1048000018B165221E4BC3F80C274FF47F03D3F871
:104810003021D3F83431072A16D11D4BD3F8203478
:10482000002B11DA4FF050230322C3F81825012280
:104830009A60D3F80421002AFBD00022C3F8042197
:104840000122DA60C3F81825124AD2F88C3043F4FA
:104850004063C2F88C30104A104B1168C3F84415FD
:10486000D269C3F84C25BDE80840FFF755BF29229F
:10487000034BC3F80C270322C3F83C2780E700BF93
:1048800000400050009003504400EFBE999D00008E
:104890000020035000ED00E00080FF0000600050A9
:1048A00070B501250268B2FA82F3C3F11F03DBB2CF
:1048B00005FA03F422EA0404D0E8EF6F964204D12B
:1048C000C0E8EC4FBCF1000FF6D1EBD101480B7002
:1048D00070BD00BF0000AD0B10B50368CB40DB0717
:1048E00010D401238B40026843EA0201D0E8EF4F65
:1048F000944204D1C0E8EC1FBCF1000FF6D1F2D114
:10490000014810BD0148FCE70000AD0B0400AD0BF1
:10491000044B1A7922B9012218601A7102487047B3
:1049200002487047542F00200000AD0B0C00AD0B67
:104930004FF0502310B5D3F8002152B10020C3F836
:104940000001D3F800210122C3F80823234B1B6880
:1049500098474FF05023D3F804218AB10022C3F8BE
:104960000421D3F80421D3F81824D3F8181402F042
:104970000302012A4FF0020128D1C3F818159A60EA
:104980004FF05023D3F8202162B10022C3F8202138
:10499000D3F820214FF48072C3F808230F4B042072
:1049A0001B6898474FF05023D3F82421AAB1002266
:1049B000C3F82421D3F824214FF40072C3F808234C
:1049C000064B0520BDE810401B681847C3F80813C4
:1049D000024B01201B689847D2E710BD542F0020DE
:1049E00001460148FFF75CBF40200020036803F048
:1049F0001F020260034A04485B09012B18BF1046DE
:104A0000704700BF0025845000288450034B0830B5
:104A100033F81000C0F34010704700BF442000205E
:104A200070B50D4C00F1080334F813300546DA0573
:104A30000E4607D5C3F3432304EBC302526854F870
:104A400033309847A3682BB131462846E268BDE869
:104A50007040184770BD00BF4420002010B4124AB7
:104A6000083032F81030D9051BD5C3F3432123F4A5
:104A7000F85322F81030002002F10E0434F8023FFF
:104A800013F4807F03D0C3F34323994209D001304C
:104A90003028F3D1002342F83130044810BCFFF72E
:104AA0001BBF10BC704700BF44200020B82000206E
:104AB00038B50246FFF7AAFF0B4C02F1080560B1BA
:104AC000002134F815305B0B9B0003F1A04303F584
:104AD0005043C3F81015C3F810151046FFF7BEFF7A
:104AE000002324F8153038BD442000202DE9FF4173
:104AF000044690461D4601B34F4E00F1080736F8B4
:104B000017309B0702D5FFF781FF28BB0023204603
:104B1000CDE900338DF80E308DF80F300DF10F0216
:104B20000B460DF10E0103F0F6FC36F8173023F0BA
:104B3000020343F0010326F81730B8F1000F2DD01F
:104B40003D4E04F1080736F8171098F800008A0760
:104B5000D8F8043002D5CBB1384821E021F020014B
:104B6000C904C90C26F8171083B10328F4D8D8F863
:104B7000043093F800C06246920002F1A04202F5B0
:104B8000504280B9C2F81005C2F8100536F8173047
:104B900023F01C0343EA800326F817301DBB284886
:104BA00004B0BDE8F081D2F8103541EA4C3123F071
:104BB0000303C2F81035D2F8103541F0200123F478
:104BC0004F3323F44073C2F810352302D2F810E5B6
:104BD00003F47C5343EA004343EA0E03C2F8103562
:104BE00026F81710D2E72046D5E90067FFF736FF11
:104BF000002ED4D0104DD5E90023964201D19F421A
:104C000018D010480DF10F01FFF74AFE0C4B9842E7
:104C1000C6D19DF80F2005EBC20308345F6035F85C
:104C2000143045F8326043EA422343F4807325F898
:104C30001430B4E70022EEE7442000200400AD0B5E
:104C40000000AD0BB8200020F0B50446154685B035
:104C500019B3344E00F1080736F81720930703D430
:104C6000FFF7D4FE00285AD112F01C0F02D04B7867
:104C7000012B54D001238DF80F3000234A1CCDE9BD
:104C8000001320468B1C0DF10F0103F044FC36F895
:104C9000173043F0030326F8173015B9224805B042
:104CA000F0BD204E04F1080736F81700830736D50B
:104CB00095F800C00023614620F02000890001F132
:104CC000A041C00401F55041C00CC1F8103526F8D0
:104CD0001700C1F810356A78002ADFD0D1F81035F6
:104CE000AD7823F4991323F4F853C1F81035D1F8B3
:104CF00010E5230203F47C53120402F4403243EA29
:104D00000E0313432A0502F4801240EA4C30134389
:104D100040F02000C1F8103526F81700BEE7034820
:104D2000BDE700BF442000200000AD0B0400AD0B28
:104D3000014BC3E9020170474420002008B5024638
:104D4000FFF764FE38B1054B083233F812300448DF
:104D50005B0B0B7008BD0348FCE700BF442000203C
:104D60000000AD0B0400AD0B38B50F4C94F8785033
:104D7000BDB96022294604F1100001F0F8FB0D20B6
:104D8000FDF77CF8094B0A48C3F87C51D3F87C2125
:104D90004FF00042C3F80423012384F8783063679E
:104DA00038BD0448FCE700BF4420002000D000507C
:104DB0000000AD0B0500AD0B034B93F878000038F5
:104DC00018BF0120704700BF442000200146014861
:104DD000FFF782BDB420002001460148FFF760BD07
:104DE000B420002037B50446FFF710FE1E4B04F137
:104DF000080233F81230E8B113F002051AD15B0B48
:104E00009A0002F1A04000F5514002F1A042056075
:104E100002F550420068D2F8100540F00100C2F8D7
:104E2000100529B1012202FA03F3104AC2F8043333
:104E300003B030BDC3F38203042B11D0052B11D076
:104E400001A80194FFF7D2FD019B0169D94001F04F
:104E500001010231204603B0BDE8304003F0A4BB9D
:104E60000321F7E70221F5E74420002000D000509D
:104E700008B50246FFF7CAFDC0B10F4B02F10801A9
:104E800033F81130990711D401225B0B9A400B497A
:104E90009B0003F1A043C1F8082303F55043D3F866
:104EA000102522F00302C3F8102508BD0021BDE83B
:104EB0000840104603F078BB4420002000D000508A
:104EC00013B5104B00F1080233F812300446DB072B
:104ED00016D5FFF7CDFF2046FFF7EAFD01A80194A4
:104EE000FFF784FD019B00EB8300D0F8003203F054
:104EF000E04343F00203C0F80032034802B010BDA3
:104F00000248FBE7442000200000AD0B0400AD0B7D
:104F10002DE9F04F002601223446634B6348644973
:104F200087B01D6835B1D0F8045315421EBF1C6010
:104F30001D68164304338B424FEA4202F1D1DFF879
:104F40006CA1DAF87C31002B00F09180DFF86481ED
:104F5000D8F820300493C8F82030574B1A6A0592CD
:104F60001A624FF000090DF1100B4FEA491300933C
:104F700048E094FAA4F4B4FA84F4009B4F4A1C4429
:104F800004F1080332F813700123E00804F007026B
:104F900003FA02F21BF80030039423EA02030BF831
:104FA000003003A8FFF722FD039BB908803350F8B7
:104FB0002330C7F382054A072F46C3F301432BD59D
:104FC00020463946DDB2FFF72BFD03A80394FFF717
:104FD0000DFD039B803350F82330C3F301439D4202
:104FE00007D10021204603F0DFFA2946204603F0CE
:104FF000DBFA03A80394FFF7F9FC0122039B02FAF2
:1050000003F303625BF82940002CB2D1B9F1000F21
:105010001DD14FF00109A8E7022B0CD10321204636
:1050200003F0C2FA05F00503012BE2D13946204610
:10503000FFF7F6FCDDE702212046019303F0B4FA06
:10504000032DF3D0019B032BD3D1022DEDE7CAF83A
:105050007C41DAF87C31D8F8203017490493C8F83D
:1050600020300A6A134305920A627FF47AAF012462
:1050700016B907B0BDE8F08F96FAA6F3B3FA83F33A
:1050800004FA03F29B0003F1A04303F55043D3F865
:105090001005D3F81015C0F30520C1F3014126EA2D
:1050A0000206FFF7BDFCE3E700D1005000D000503E
:1050B00020D1005000258450002884504420002036
:1050C0000022034BC3F88425C3F80425704700BFB2
:1050D00000900350044AD2F80034DB07FBD501608E
:1050E000BFF35F8F704700BF0090035008B5C0F357
:1050F0000B0383B90222094BC3F88425C3F80425A6
:105100004FF0FF320260D3F80024D207FBD5FFF73F
:10511000D7FF034808BD0348FCE700BF00900350D9
:105120000000AD0B0A00AD0B012208B5054BC3F81A
:105130008425C3F80425FFF7CDFFBDE80840FFF73D
:10514000BFBF00BF0090035070B500F06044B4F1E1
:10515000005F68D1840766D1354D95F83040012C49
:1051600001D09C4261D12C6804BB022B314B0BBF98
:10517000C3F81025C3F80425C3F81405C3F80805BF
:105180000BBFC3F81815C3F80C1508220422002120
:10519000C3F8001102F1A043012203F52C331A6079
:1051A000244AD2F80031002BFBD00DE0AE68214C30
:1051B00066B1022BE8606961EA612DD1C4F810255F
:1051C000C4F81405C4F818151B4870BD022B85F8E7
:1051D00030302961AA61A8600CBFC4F81025C4F85A
:1051E00004254FF000020BBFC4F81405C4F80805ED
:1051F000C4F81815C4F80C1508BF08230D4918BFCA
:105200000423C1F80021012203F1A04303F52C334C
:10521000C1F804231A60D7E7C4F80425C4F80805C8
:10522000C4F80C15D0E70548CFE70548CDE700BF27
:105230005C2F002000B002500000AD0B0A00AD0B47
:105240000B00AD0B38B56424064DD5F8003133B9E9
:105250000A2003F028F8013CF7D1034838BD034881
:10526000FCE700BF00B002500700AD0B0000AD0B23
:10527000084B9A685A621A699A629A69DA62DA681D
:105280009A6032B15A691A61DA699A610022DA6069
:10529000704770475C2F002010B50A4A0A4C00F096
:1052A0001F034009012818BF224602EB8302D2F8EF
:1052B000003203F0E04343EA012343F00203C2F863
:1052C000003210BD002884500025845010B50E4BCC
:1052D0000238D3F83C26D3F83836072813D8DFE84D
:1052E00000F0110F0D0B0A080604100EC871100C07
:1052F0008871100A48710A711A0ECA701A0C8A70E5
:105300001A0A4A700B7010BD00B00250023807280C
:105310001FD8DFE800F02927251123211F04CB79AE
:105320001B068A7943EA02434A7943EA02230A794F
:1053300013430E4AC2F83C36CB781B068A7843EA00
:1053400002434A7843EA02230A781343074AC2F821
:10535000383670470023E4E70023E5E70023E6E75B
:105360000023EBE70023ECE70023EDE700B0025059
:10537000F8B5674F044697F830300D461646002BB7
:1053800040F0C280C27C12B1037D002B6CD1207929
:10539000FF2800F0BB806379FF2B00F0B780A37972
:1053A000FF2B00F0B380E179FF2900F0AF80636844
:1053B000DFF860C123F07F43634540F0A7800E29EA
:1053C00040F0A480237AFF2B02D00F2B40F09E8068
:1053D000637AFF2B02D0102B40F09880B2B90321E2
:1053E000FFF75AFF6079FFF757FFA079FFF754FFE7
:1053F000E079FFF751FF207AFF2801D0FFF74CFF3B
:10540000607AFF2802D00321FFF746FF237D5BBBB4
:105410002379FF2B14BF1A464FF0FF323E4BC3F8DF
:1054200024256279FF2A08BF4FF0FF32C3F82825F0
:10543000A279FF2A08BF4FF0FF32C3F83025E27986
:10544000FF2A08BF4FF0FF32C3F83425227AFF2A23
:1054500008BF4FF0FF32C3F83825627AFF2A08BF31
:105460004FF0FF32C3F83C2523682B4AC2F8403581
:10547000237BE07AA17A9B0143EAC0030B43617B63
:1054800043EAC113C2F84435617CD2F84435B1BB5C
:1054900043F44033C2F844354FF4C063C2F8403699
:1054A000D2F80016A37B21F07F4121F0FF010B43CE
:1054B000E17B43EA0163217C43EA4163617C43EA87
:1054C0000173C2F80036E37CC7E9005687F8313033
:1054D0000123C2F8083315B12B20FCF7CFFC0021C3
:1054E0000122C7E902110C4B87F83020C3F80025D0
:1054F000C3F800111A60BDE8F840FFF7A3BE23F41B
:10550000003343F48033C5E70448F8BD0448FCE7A2
:105510005C2F002011120D0000B002500500AD0BF1
:105520000400AD0B70B51446194A054692F83020B8
:10553000012A2BD10022174EC6F8002111B1407864
:10554000FFF7E4FE0123C6F80833AB786A781B0343
:1055500043EA02232A781343EA7843EA42332A795A
:1055600043EA82336A7943EAC233C6F83436FFF736
:1055700069FE094B984208D00023C6F800311CB1DF
:1055800021466878FFF7A2FE044870BD0448FCE796
:105590005C2F002000B002500700AD0B0000AD0BE7
:1055A0000B00AD0B1FB500230C4A02A802920DF1AF
:1055B000070211468DF80730ADF80C30FFF7B2FF47
:1055C000074B984206D19DF8073013F0010F054BA9
:1055D00018BF184605B05DF804FB00BF05020001C6
:1055E0000000AD0B0B00AD0B2DE9F8432B20FCF7B1
:1055F00053FC214B214ED3F8342602F44032B2F54D
:10560000803F04BF1E4AC3F834260122C3F8082392
:105610001A610022C3F80025C3F8002196F8312052
:1056200022BBD3F82405D3F82895C0B2D3F830852F
:10563000D3F83475D3F83855D3F83C4502F0CCFF95
:105640005FFA89F002F0C8FF5FFA88F002F0C4FF49
:10565000F8B202F0C1FFE8B2FF28E4B201D002F0D4
:10566000BBFFFF2C02D0204602F0B6FF002386F8D5
:105670003030BDE8F88300BF00B002505C2F00203E
:10568000000103008B0721D1124A13681BB192F865
:105690003030012B1CD1042382F830300E4BC3F87C
:1056A0001C150021C3F82005C3F800110121D960A1
:1056B000106840B9D3F800110029FBD0012382F80B
:1056C000303006487047C3F80413FAE704487047BF
:1056D000044870475C2F002000B002500000AD0B62
:1056E0000A00AD0B0B00AD0B10B5174BD3F8002122
:1056F000E2B10022154CC3F8002194F83020032AAF
:1057000015D0042A15D0022A04D1012384F82030B0
:10571000FFF7AEFDA36813B9012384F83030D4E954
:10572000003100209847002384F8203010BD022368
:10573000ECE7032284F82020D3F81C256262D3F81A
:10574000203584F82830E5E700B002505C2F0020B7
:1057500073B504460D464FF02003EFF3118683F333
:105760001288BFF36F8F0022042896BF114B124B93
:1057700053F82030009245210246104800F025FEE3
:105780003DB1EB69C3F308031BB145210C4800F0A0
:105790001CFE00220B4B45210B4800F016FE29464B
:1057A0002046FEF7C7FA86F31188BFF36F8F02B069
:1057B00070BD00BF3C8D0000CB9D0000D99D000056
:1057C000069E00002C9E0000349E00000F4B70B51A
:1057D00053F82040013053F82060A64200D870BD35
:1057E000D4E90035284698476DB138B10028B8BFD4
:1057F0004042FF28A8BFFF20EB681870EA68537882
:1058000043F0010353700834E7E700BF508D0000F8
:10581000012208B5084B03201A70FFF7D7FF00F0EC
:1058200013F90420FFF7D2FFFAF7FCFD034A137BBC
:1058300023F00103137308BDB54800205821002050
:1058400008B50348034A0021121A02F0DEFE08BD23
:1058500038210020B848002008B50020FFF7B6FF27
:10586000184B03F5006282F3088883F30A88002549
:10587000E023154C84F82230E57725766576A57609
:1058800084F82050636A43F4E023636284F8235071
:10589000FCF77EFDFCF798FA4FF0FF33A362E3625A
:1058A000FCF738FFFCF710FE02F0A3FE0120FFF723
:1058B0008DFF0220FFF78AFF2B462A462946034820
:1058C000FCF752FBB848002000ED00E01158000042
:1058D00008B50648064A0749121A02F098FEBDE8C4
:1058E0000840054A0549064802F091BE0020002004
:1058F00034210020CC9E000000000000CC9E00005F
:1059000000200020034B1B680BB9FEF72BB90020C9
:10591000704700BF902F002010B50E4B1C689C42B2
:1059200004D1FFF7EFFF6FF0004010BDFFF7EAFF73
:10593000002CF8D0D4E904321B1A62EBE072B3F108
:10594000004F72F10001EEDA002AACBF18460020C9
:10595000EBE700BFC020002030B570B10B4B5B6897
:1059600098420AD0036843B1D3E90421D0E9044541
:10597000121941EB0501C3E90421D0E9003213609B
:105980005A600023C0E9003330BD00BFC0200020B2
:105990002DE9F84303464FF02002EFF3118482F320
:1059A0001288BFF36F8F254FDFF89490D9F800006D
:1059B000DFF890C048453B604FEAE375DCE9001E24
:1059C0000CD058B1D0E90486434575EB060217DACE
:1059D000B8EB030266EB0506C0E9042659184EEB46
:1059E0000505CCE9001500253D60FFF795FF294628
:1059F000FEF786F884F31188BFF36F8FBDE8F88354
:105A000018EB01014EEBE8730022CCE900130023F0
:105A1000C0E90423FFF7A0FF84F31188BFF36F8F61
:105A2000836898474FF02003EFF3118483F31288C3
:105A3000BFF36F8F3B68A3EB0803B7E7902F0020FD
:105A4000C0200020D8210020014800F0D7BB00BFB3
:105A50009E9E000010B50A4C23681BB10123002054
:105A6000236010BD00F058F80028F7D0013807284F
:105A700003D8044B53F8200010BD034810BD00BFED
:105A8000942F0020688D0000FE8FFFFFBFF34F8F23
:105A90000549064BCA6802F4E0621343CB60BFF3CA
:105AA0004F8F00BFFDE700BF00ED00E00400FA05E6
:105AB00030B44FF0FE3200250B4B0C4C0C494968BA
:105AC000C3F80024C3F80424C3F80824C3F80C2442
:105AD000C3F81024C3F81424C3F81824C3F81C24F2
:105AE000C4F8005530BC0847005084500040845032
:105AF000C8200020024BD0E90012C3E90012704711
:105B0000C820002038B131B10022014403460130E1
:105B100088421A70FAD1704708B500F011F830B910
:105B200000F010F838B9054AC2F80C0A08BD00F0B8
:105B300037F8032008BD042008BD00BF0050845082
:105B40000020704710B5114800F048F800B110BDB2
:105B50000F4800F043F80028F9D10E4C204600F021
:105B60003DF80028F3D10C4B0C481C6000F036F8CF
:105B700001460028EBD100F02DF8044608B120467C
:105B800010BD00F03FF82046FAE700BFDC200020FF
:105B9000D0200020D8200020E0200020D4200020A9
:105BA00008B5084800F024F8074800F021F8074835
:105BB00000F01EF8064800F01BF8BDE8084000F0B1
:105BC0000BB800BFDC200020D0200020D82000200F
:105BD000D420002000207047704700BF08B5034B59
:105BE00002681B6810689847002008BDEC20002060
:105BF00008B5034B02685B6810689847002008BD31
:105C0000EC20002070B5094C094D2069AB6898471D
:105C100018B1084B08485B6898470021074AEB68B1
:105C200011602069BDE87040184700BFFC200020CB
:105C3000EC200020C8200020888D0000982F002034
:105C400010B5044650B1636813F0685F05D0064A8A
:105C5000934202D000236260236010BD034B0448CE
:105C60005B689847EFE700BF2C5F5CA9C820002065
:105C7000A88D0000C8B143680D4A934213D013F0B9
:105C8000685F0ED0012350E8002F194640E8001C41
:105C90009CF0000FF7D1012AF5D0BFF35F8F0020F1
:105CA000704704487047044870476FF4E0407047FD
:105CB0002C5F5CA9E98FFFFFEA8FFFFF034680B1ED
:105CC000426809498A420AD012F0685F05D0BFF3E2
:105CD0005F8F002210461A607047044870470448DE
:105CE00070476FF4E04070472C5F5CA9E98FFFFFBD
:105CF000EA8FFFFF10B5044620B10023034A23605A
:105D0000626010BD0248FFF7D3FEF6E73A00003AA2
:105D1000D08D0000704729B101290CBF05206FF01C
:105D20001500704702207047002070472DE9F743A7
:105D30000E4617469946044628B94FF0FF384046AC
:105D400003B0BDE8F0830029F7D0002AF5D0CB6876
:105D50000D8938461D44042329460DEB030200F04B
:105D600042FB80460028E8D146F60812BDF8041030
:105D70007389914225D1BDF806109942DDD10423E3
:105D800038460DEB0302294400F02DFB0028D4D146
:105D900046F60713BDF804209A42CED1C4E9006745
:105DA0009DF82830A4F80890A3727389BDF80620E6
:105DB0002B44E360738913442B44043563612561EC
:105DC000BDE7002BE4D0B8E72DE9F3410E461746B6
:105DD0001D46044620B94FF0FF3002B0BDE8F08107
:105DE0000368002BF7D04368002BF4D04FF6FF7800
:105DF000D4E904239A4216D223685B8923B1E3686D
:105E0000934204BF043323610423216960680DEBCE
:105E1000030200F0E8FA0028DDD1A37A2BB1D4E91F
:105E200003329A4201D30120D7E72389BDF8061037
:105E3000434501F1040203D0BDF804C09C450BD1D9
:105E400015B1BDF804302B802369043333603980E9
:105E5000236913442361C0E7236913442361C7E71F
:105E600000F053BB4FF4C0735843303070470B7889
:105E7000022B06D0052B14BF4FF0FF304FF4C0703B
:105E800070474FF4C070704710B5044600F0E9FA4F
:105E90004FF4C072A368303B02FB103010BD816824
:105EA0000122183921F00701083900F003BE13B5AB
:105EB0000446019100F08FFD0423A0F108010DEBD1
:105EC0000302204600F0CAFD02B010BD70B51346B3
:105ED0000E461546002102460446FBF705F850B968
:105EE0002B460121204604F12C02FAF7FDFF10B1E8
:105EF000002E08BF002070BD73B5044600200D467B
:105F00001646FFF708FF6946C0B2FBF7FFFE30BB3D
:105F10002C2303FB0544E368258900981D440423D2
:105F200029460DEB030200F05EFAC0B946F60813ED
:105F3000BDF8042064899A42009815D1BDF8063056
:105F40009C420CD1042361190DEB030200F04BFAC3
:105F500028B946F60713BDF804209A4207D00098E6
:105F600000F040FA02B070BD002CF2D0F7E7BDF8A7
:105F70000610214429443160F1E737B580250446F5
:105F8000426A01A902200195FBF7E8FE58B9019B7E
:105F90000520226DA36201A90195FBF7DFFE0546EE
:105FA00028B1092500E00125284603B030BD019B3A
:105FB000206A636500F055FAE065F5E701230360A8
:105FC00003F1012343600023C0E9023370474379A2
:105FD000012B07D10368012B04D10079431E5842DD
:105FE00058417047002070477FB506460D46022095
:105FF00001A9FBF78BFE38BB0198FFF745FFF16D58
:106000000446284600F0E5F80444019800F029FA17
:106010000646019800F02CFA082201460DEB02001A
:1060200000F0A5FA2B7921468DF808300198334607
:1060300002AA00F0EDF9041E019818BF012400F037
:10604000D1F9204604B070BD0124FAE700F0F5B99B
:106050002DE9F8430E46002107460846FFF75BFE90
:10606000044601210020FFF756FE33789C4221D0E0
:10607000984221D101252C2303FB0575F86DAC6AEC
:10608000FFF7F0FE4FF000080746013C6B6A304610
:1060900003EBC40253F83410D2F804901B684A464C
:1060A000C91AC844FFF7D2FFB84504F1FF34EDD355
:1060B000BDE8F8830025DEE70120F9E737B515468E
:1060C0000C460520694600F00CFDE979012903D052
:1060D0000022204600F019FD9DF80330012B02D16B
:1060E000204600F0F1FCA9682046FFF7E0FE2046BC
:1060F000FDF7A0FE002003B030BD73B50D46064687
:10610000FAF7DAFF0446E86050B302282DD101A95E
:10611000FBF7FCFD58BB2A4631460198FAF732FFDF
:106120000446D0B9019800F056FC012301460DF158
:106130000302019800F057F90446A0B90122019822
:106140000DF1030100F05BFC10B101238DF8033069
:106150009DF8033003F00F03EB71019800F042F952
:10616000204602B070BD0124F7E70724F8E70124B8
:10617000F6E713B5022001A9FBF7C8FD48B901985D
:10618000FFF78DFE0446019800F02CF9204602B07E
:1061900010BD0124FAE71FB5022001A9FBF7B6FDE7
:1061A000A8B9019802A9FDF765FE044668B99DF8F3
:1061B0000B30032B03D1019800F086FC04460198B4
:1061C00000F010F9204604B010BD0124F7E70124C7
:1061D000F8E710B543790279012B06BF00230C467E
:1061E000CB0102F1FF3201FB0233026818BF4C0001
:1061F000013A04FB023010BD002070470FB407B510
:1062000004A951F8040B0191FBF782F903B05DF882
:1062100004EB04B07047038B13F0070305D1036848
:10622000002B0CBF002003207047022B05D1408BB0
:10623000B0FA80F0400980007047012B05D1036857
:10624000002B0CBF0020052070470020704710B5C0
:106250000C4600B111B96FF0150010BD081D00F01B
:1062600095F80028F9D1A368032BF6D9F3E72DE9B7
:10627000F0410D4607461946281D90461E4600F07F
:1062800096F8044638B13346424629463846A44675
:10629000BDE8F0416047BDE8F08110B44FF0200444
:1062A000EFF3118284F31288BFF36F8F416110BC4A
:1062B0000121FBF73BB938B50C46054658B151B141
:1062C0000B6843B14B6833B11C22002100F04FF939
:1062D00000202C6138BD6FF01500FBE770B5054656
:1062E0000E46FFF7B4FF041E15DB4FF02003EFF35B
:1062F000118283F31288BFF36F8F4FF6FF716B8BA0
:106300002C8B8B4204F0070407D182F31188BFF372
:106310006F8F6FF00A04204670BD022C0CD1013340
:106320006B8382F31188BFF36F8F002322463146BF
:106330002846FFF79CFFEEE7062C14D8DFE804F0B0
:1063400004131313041A0400002333606B683BB971
:10635000C5E90066ACB902212846FBF7E7F8DAE7A1
:106360001E606E60F6E782F31188BFF36F8F6FF0E7
:106370000404D0E782F31188BFF36F8F6FF08504B8
:10638000C9E782F31188BFF36F8FC4E7034658B1A2
:10639000426802F00302012A03D0032A04D10268F2
:1063A00012B10020986070476FF015007047426886
:1063B000034602F00302032A4FF00002816014BF7B
:1063C000104600685A60704770470FB407B504A9BB
:1063D00051F8040B0191FBF79BF803B05DF804EB57
:1063E00004B070477047002930B4044618460BDBF0
:1063F000A5680844A84207D8E06864682144846816
:106400002468A44630BC60476FF0150030BC70476C
:10641000002930B4044618460BDBA5680844A8429E
:1064200007D8E0686468214484686468A44630BC86
:1064300060476FF0150030BC70470029034610B468
:1064400010460ADB9C680844A04206D8D8685B68FE
:106450001944836810BC9B6818476FF0150010BC86
:10646000704708B5C0688368DB689847006808BD56
:1064700008B5C0688368DB689847007908BD70B5C7
:106480004C680368A34201D2012070BD8A6822448F
:10649000934201D30020F8E74E69D1E90325B542C4
:1064A00003D36FF00B038B61F4E71B1B42F835300D
:1064B0004368086902EBC00253600B6901330B614A
:1064C000E2E7002008B5FBF763FB70470146006870
:1064D000FBF7A6BC00210120FBF7A2BC08B5FBF727
:1064E00013FDBDE80840FBF771BD40E800F313F46D
:1064F000803FD8B208BF6FF01500704703460020F8
:106500001A5C02B970470130FAE710B55AB1013987
:10651000841810F8012B11F8013FA04201D09A42D3
:10652000F7D0D01A10BD1046FCE7431A934210B5BD
:1065300000EB020308D3024601399A420BD011F84E
:10654000014F02F8014BF8E70A4412F8014D8A4264
:1065500003F8014DF9D110BD10B5431E0A44914214
:1065600000D110BD11F8014B03F8014FF7E70346C6
:10657000C9B20244934200D1704703F8011BF9E706
:106580004FF0FF3070470C220369C9B201FB0233A0
:10659000986F00F0070070474FF02003EFF311826F
:1065A00083F31288BFF36F8F036803F0C00343F0D7
:1065B0000203036082F31188BFF36F8F704770B5D9
:1065C000C9B203694FF02004EFF3118584F31288F8
:1065D000BFF36F8F0C2606FB0134A46F14F0C004C8
:1065E00008D0A24206D085F31188BFF36F8F4FF019
:1065F000FF3070BD012271430B449A6785F3118807
:10660000BFF36F8F43680B445B6898470020F0E747
:106610008022FFF7D4BFF8B5069F0469C9B24FF0D6
:106620002005EFF3118685F31288BFF36F8F0C25D9
:1066300069430C44A56F05F0070CBCF1010F0BD1A9
:10664000A76786F31188BFF36F8FC4E91C234368E3
:106650005B5898470020F8BD05F0C005AF4286F3AF
:106660001188BFF36F8F0CBF6FF077004FF0FF30D2
:10667000F1E713B580240094FFF7CDFF02B010BD01
:106680006FF08500704710B41C240069CBB203FB87
:106690000400002110BC1047032001F0DBBE0220E3
:1066A00001F0D8BE002001F0D5BE032001F031BFBB
:1066B000022001F02EBF002001F02BBF4368002014
:1066C0005B681B690B607047436802EA01005B6806
:1066D00021EA020198600020D960704743680020D9
:1066E0005B6899607047436800205B68D9607047B9
:1066F00043685A68536821EA03000B409060002009
:10670000D360704710B503695868F8B1884219D151
:106710009C680868A142586000D198600020086019
:106720002AB15A680A609A68596002B999600020D3
:1067300010E0814206D10868206098688142EDD15E
:106740009C60EBE7044600680028F2D1002AE8D1FB
:106750006FF0150010BD08B901230B7070477FB5AD
:10676000FF238DF803300DF1030300210193012372
:10677000CDE90231052303A88DF80C3001AB04915B
:106780000593FCF7EDFA0028A8BF9DF8030007B0B9
:106790005DF804FB1FB5002188420CBF06230423CB
:1067A00001A8CDE9011103918DF80430FCF7D8FA66
:1067B000002818BF6FF0040005B05DF804FB38B581
:1067C00005460C4601F0FFFE002D07DBA84205D967
:1067D000401B84428CBF0020012038BD0020FCE714
:1067E000F7B51C460023164682682360A3600D4659
:1067F0001369694601AA9847019B5A1E01921BB969
:106800006FF0150003B0F0BD0098A26847682168DA
:10681000676085B9B31AD0F800C0634528BF6346E6
:1068200003FB07111A442160A26002689A4206D84D
:1068300008300090E0E76B1AB3FBF7F3EBE70020BA
:10684000E0E713460022FFF7CBBF2DE9F047002415
:10685000836886B0884691461B6902AA01A99847B9
:10686000A2462546029BAB4202D806B0BDE8F0879F
:106870000026019F07EBC5077B6804933A680AEB83
:106880000603B24202D89A460135EBE74946039423
:10689000059303A8C0470028E7D0049B01361C4499
:1068A000ECE70B460269D2E9010183E8030000200E
:1068B000704743681B68D3F88004C3F880047047AE
:1068C000436802691B68D3F8100150B10020526977
:1068D00012780A70C3F81001D3F8102101221A604F
:1068E00070474FF0FF30704702680346D2F85801F6
:1068F00040B95B689B0706D4D2F82001003818BF66
:10690000012070470120704742681368D3F80413D0
:10691000C90518D5D3F82011A9B14FF02000EFF325
:10692000118180F31288BFF36F8FD3F8200130B14B
:106930000020C3F82001D3F820010120D86081F3A2
:106940001188BFF36F8F5268D20615D54FF0200122
:10695000EFF3118281F31288BFF36F8FD3F85811D0
:1069600011B10021C3F800154FF48001C3F80813DA
:1069700082F31188BFF36F8F7047002200F150033C
:106980009B009BB203F1502303F580331A601B6810
:10699000704708B5FCF760FF08BD30B54368136069
:1069A000057A446804EBC504A34202D36FF00100EA
:1069B00030BD5C798C4201D00833F0E70020F7E766
:1069C000FFF748B808B5FBF7F9F9FFF77EFDBDE81A
:1069D0000840FFF73FB88068183820F007001038EB
:1069E0007047042809D0052803D1481E18BF01208C
:1069F0007047431A5842584170470120704738B5D4
:106A000015460C4661B15AB1FFF732FD21462544C7
:106A100011F8013B834203D1A942F9D1012038BDCD
:106A20000020FCE738B50C460123114622460546F6
:106A3000FFF7D9FC00280FDB012221462846FFF78B
:106A4000DEFF38B92378012B14BF02230123002075
:106A5000237038BD0323FAE70120FAE72DE9F74355
:106A60001D4606460F469046FFF7FBFC6C1E04448D
:106A700040420440082C1AD83046FFF7F9FC814602
:106A80002A4641466846FFF767FD4946621B0DEB03
:106A90000500FFF76CFD23466A4639463046FFF78E
:106AA000B7FC003818BF012003B0BDE8F0834FF0F9
:106AB000FF30F9E707B501238DF8042001AAFFF79D
:106AC000CDFF03B05DF804FB81680122183921F085
:106AD0000701FFF7EFBF8268183A22F00702FFF7BD
:106AE000A1BF13B50C46C0B201A9FBF70FF950B90D
:106AF00021460198FDF7BEF904460198FFF772FCA4
:106B0000204602B010BD0124FAE713B541EA021194
:106B100004468DF80710FFF75EFF012301460DF1D3
:106B200007022046FFF79AFF02B010BD0020704711
:106B300070B50368CD1A002D02DC6FF05F0070BDE8
:106B400093F900601C78002E0ADB5C1C04601B7843
:106B500013600368C91A13688B42EED80020EEE771
:106B600004F07F04013C032C2BD8DFE804F0020A78
:106B70001421012DE1D05B781360036802330360B8
:106B8000E7E7022DD9DDB3F801305BBA9BB21360A1
:106B900003680333F3E7032DCFDD9C785D7824028F
:106BA000DB7844EA05442343136003680433E6E7D3
:106BB000042DC2DDD3F801301BBA1360036805331E
:106BC000DDE76FF06300BAE770B404680E1B002EB7
:106BD00007DD26789E4208D10134046070BCFFF7BF
:106BE000A7BF6FF05F0070BC70476FF06100FAE7FD
:106BF00073B50223154601AA0446FFF7E5FF40B925
:106C0000019E28463246216800F018FB2368334471
:106C1000236002B070BDF0B5844617460E46144698
:106C20000025BCF10F0F06F1400604F1400477D8AF
:106C30006FF00F02040902FB040007284FEA841CCE
:106C400001EB841607EB84145DD951F80C10083859
:106C5000A3FB0112691857F80C5042F100024919C0
:106C600047F80C10716842F10002A3FB0151521960
:106C7000656841F1000152196260B26841F100019A
:106C8000A3FB02524919A56842F100024919A1600B
:106C9000F16842F10002A3FB01515219E56841F18C
:106CA00000015219E260326941F10001A3FB025276
:106CB0004919256942F1000249192161716942F1BE
:106CC0000002A3FB01515219656941F100015219FB
:106CD0006261B26941F10001A3FB02524919A56941
:106CE00042F100024919A161F16942F10002A3FBDE
:106CF00001155218E16945F100055218E26145F1AC
:106D000000052034203627464FEA800C06EB800031
:106D1000B04240F006816444002D40F01081F0BD87
:106D200056F8402CACF1100CA3FB02E215EB0E0E52
:106D300054F8405C42F1000215EB0E0544F8405C4B
:106D400056F83C5C42F10002A3FB05E512EB0E0E87
:106D500054F83C2C45F1000512EB0E0244F83C2C93
:106D600056F8382C45F10005A3FB02E215EB0E0E98
:106D700054F8385C42F1000215EB0E0544F8385C1B
:106D800056F8345C42F10002A3FB05E512EB0E0E4F
:106D900054F8342C45F1000512EB0E0244F8342C63
:106DA00056F8302C45F10005A3FB02E215EB0E0E60
:106DB00054F8305C42F1000215EB0E0544F8305CEB
:106DC00056F82C5C42F10002A3FB05E512EB0E0E17
:106DD00054F82C2C45F1000512EB0E0244F82C2C33
:106DE00056F8282C45F10005A3FB02E215EB0E0E28
:106DF00054F8285C42F1000215EB0E0544F8285CBB
:106E000056F8245C42F10002A3FB05E512EB0E0EDE
:106E100054F8242C45F1000512EB0E0244F8242C02
:106E200056F8202C45F10005A3FB02E215EB0E0EEF
:106E300054F8205C42F1000215EB0E0544F8205C8A
:106E400056F81C5C42F10002A3FB05E512EB0E0EA6
:106E500054F81C2C45F1000512EB0E0244F81C2CD2
:106E600056F8182C45F10005A3FB02E215EB0E0EB7
:106E700054F8185C42F1000215EB0E0544F8185C5A
:106E800056F8145C42F10002A3FB05E512EB0E0E6E
:106E900054F8142C45F1000512EB0E0244F8142CA2
:106EA00056F8102C45F10005A3FB02E215EB0E0E7F
:106EB00054F8105C42F1000215EB0E0544F8105C2A
:106EC00056F80C5C42F10002A3FB05E512EB0E0E36
:106ED00054F80C2C45F1000512EB0E0244F80C2C72
:106EE00056F8082C45F10005A3FB02E215EB0E0E47
:106EF00054F8085C42F1000215EB0E0544F8085CFA
:106F000056F8045C42F10002A3FB055E521954F8E6
:106F1000045C4EF1000EAA184EF1000544F8042C52
:106F20007FE656F8042BA3FB0221AA1841F10005C5
:106F30003968891845F1000547F8041BE8E623681D
:106F40005B192CBF0125002544F8043BE4E62DE93C
:106F5000F04F8A46174685B00E9C00906268A06884
:106F6000002192000393FFF702FB7E68DAF80430F9
:106F7000A568B34228BF3346A9464FF00008741CE9
:106F80000193A400009BB04598681CD1043C2544A3
:106F900022462946FFF7E0FA00222B59281F013329
:106FA0002B511346D7F808E09E422BD12B5930467F
:106FB0009B1A2A4600992B518968DBB205B0BDE8BF
:106FC000F04F00F0E5BFDAF8081050F828B0D9F813
:106FD00000300868039A00FB0B33534301984A467C
:106FE00002935B46FFF717FE4A46029B3046B9689C
:106FF000FFF711FE002349F804BB49F8043008F1FB
:107000000108BFE750F804CF5EF82370ACEB020133
:10701000B9422CBF4FF000084FF00108C91B94453E
:107020002CBF424608F1010201600133BCE773B591
:1070300001F18042013A00EB8202824201D202B0A9
:1070400070BD03680024019304230DEB030529465A
:1070500015F8016B013B13F0FF0346EA0424F7D156
:10706000156801951D46013311F8016BDBB2042B45
:1070700046EA0525F7D140F8045B42F80449DCE70D
:10708000002301228360C0E90023704710B5044645
:1070900068B1806830B161688900FEF733FDA0688F
:1070A000FDF748F900230122C4E90023A36010BDC5
:1070B00042F21073994270B504460D4602D96FF042
:1070C0000F0070BD43688B4201D30020F9E7042113
:1070D0002846FDF729F906460028F0D0A16859B1E5
:1070E00062689200FFF738FA6168A0688900FEF7CD
:1070F00009FDA068FDF71EF9C4E90156E5E738B5BA
:1071000004460D4619B9FFF7C1FF002038BD42689B
:107110008A4207D1002180689200FFF728FA0123F4
:107120002360F2E7FFF7B2FF29462046BDE838406A
:10713000FFF7BEBF884270B505460E4609D04968C4
:10714000426841B92AB10123920003608068FFF7C9
:107150000EFA002070BD4C1E84B93368013494428D
:107160002B6012D921462846FFF7A2FF0028F1D153
:10717000B168A868A200FFF7EFF9EAE7B36853F82F
:107180002430002BE9D1013CE6E7A868121B00215E
:10719000920000EB8400FFF7EAF9E9E770B50E46CC
:1071A00001210446FFF784FF054688B9626801465D
:1071B0009200A068FFF7DBF9A36886EAE672002E6A
:1071C000A2EBE6721A60ACBF01234FF0FF332360DD
:1071D000284670BD4368B1EB431F3FBF83684A092F
:1071E00053F8220001F01F013ABFC84000F001002F
:1071F000002070470246406898B19268431E8BB9E0
:1072000052F823100020002908DB4FF00042013023
:1072100020284FEA520201D01142F8D00133C0EBCE
:107220004310704752F823100029E9D1013BE6E7EB
:1072300008B5FFF7DFFF0730C00808BD2DE9F041B2
:1072400012F0030418BF012404EB9204884621467F
:1072500007461546FFF753FF064668B965B1BB6898
:10726000C5EB84002A4641461844FFF775F9B86813
:1072700014B12146FFF7DBFE3046BDE8F081F8B5DA
:10728000044663680846B2EB830F4FEA83051AD9B8
:10729000521B8E180021FFF76AF930462A4600215A
:1072A00083188A4211D10020F8BDA16823F003079A
:1072B000C95903F00306F600F140C9B289B9013398
:1072C000AB42F2D1EBE71346FAE7A66821F00300E0
:1072D000305801F00305ED00E84003F8010D0131DD
:1072E000DFE76FF00700DFE7F8B505460E464C090B
:1072F00001F01F07FFF77EFF6B683044B0EB431FC0
:1073000005D81F2E0FD8002F41D100200AE010F021
:107310001F0118BF012101EB50112846FFF7C8FEDD
:107320000028EED0F8BD6FF003006B68604319468B
:107330009A00A142A2F104020CD8E21A9C4288BF32
:107340000022134400229B00043B191DDBD0A968D6
:10735000CA50F9E7AE68013906EB020C5CF800C0D0
:1073600046F802C0E5E7AB6853F8241001FA07F0CD
:1073700043F82400A86850F82430134340F8243020
:1073800021FA06F201346B68A342ECD8BDE7002273
:10739000C7F12006F7E7F0B443684C09A34201F0B7
:1073A0001F0201D309D11AB1F0BC0021FFF7F6BECC
:1073B0001F2904D8F0BC002070471F2909D90023D9
:1073C000A5004168091B99421BD8002441689942D5
:1073D0001ED8002AEED000244368C2F12007013BEA
:1073E000E8D3816851F8235025FA02F641F823606A
:1073F000866856F82310214346F8231005FA07F44F
:10740000EDE781684E59043541F823600133D8E730
:10741000816841F823400133D8E710B542683AB992
:107420004B6873B9B2B9181E18BF0120404210BD95
:10743000836803EB820353F8043C002BF0D1013A3C
:10744000EDE78C6804EB830454F8044C002CE9D17C
:10745000013BE6E79A4210D811D3013A836853F80A
:1074600022408B6853F822309C4206D802F1FF324A
:1074700005D3531CF2D10020D9E70120D7E74FF004
:10748000FF30D4E7024630B5436823B9486858B99D
:10749000002B36D12FE0906800EB830050F8040CED
:1074A0000028F3D1013BF0E78C6804EB800555F828
:1074B000045C15BB0138EAE70D6802D20868404257
:1074C00020E01068002803DD002D07DA012019E014
:1074D000002D03DD10B14FF0FF3013E0013B916848
:1074E00051F8235054F823108D420BD803F1FF3389
:1074F000E5D3591CF3D1002004E0002BDED08342F9
:10750000DAD9106830BD1FB581EAE173A3EBE173EE
:1075100000290093ACBF01234FF0FF3301930123F7
:1075200001A90293CDF80CD0FFF7ACFF05B05DF8D0
:1075300004FB90422DE9F04106460F46154602D065
:10754000884229D12F46012333607D6865BB2946D7
:107550003046FFF7ADFD044618BBB368B9689C46DA
:107560000746854229D103EB8503D7B1726805F13F
:107570000108AA4207D841463046FFF799FD68BB8B
:10758000B36803EB85031A684546D2192CBF01275F
:10759000002743F8042BE8E7FFF7CCFD044600285A
:1075A000D0D02046BDE8F081BB6803EB850353F8DB
:1075B000043C002BCBD1013DC8E7DCF80020D219F8
:1075C0002CBF4FF0010E4FF0000E51F8207001302B
:1075D000D2194CF8042B4EF10007C2E70446E0E74D
:1075E0002DE9F84305460E46904654683CB971684B
:1075F000A1420ED26FF009073846BDE8F883D8F8EB
:10760000083003EB840353F8043C002BEFD1013C1A
:10761000ECE72846FFF74CFD07460028ECD17268DE
:10762000A24209D9B168A868121B920001EB84013B
:1076300000EB8400FEF790FF6A687068824207D909
:10764000AB68121A0021920003EB8000FEF78FFF57
:1076500000221346D5F808C0D6F808E0D8F808800C
:107660009C4212D172B14FF0FF316B68A34225D911
:10767000AB6853F82420EAB1AA6852F82430013BE1
:1076800042F8243001232B60B6E75EF8236058F8F7
:107690002300B11A81422CBF4FF000094FF00109BD
:1076A000091A4CF8231096422CBF4A4609F10102F0
:1076B0000133D5E743F824100134D6E7DCD199E74C
:1076C000F8B50F68136805467B430C46164616D579
:1076D00011462046FFF7A1FE002806DB3246214670
:1076E0002846FFF77DFF38B1F8BD22462846FFF750
:1076F00077FF0028F8D17F4200202F60F4E7FFF7E2
:1077000018FFF0E7F8B50F68136805467B43002BB8
:107710000C46164616DD11462046FFF77EFE002871
:1077200006DB324621462846FFF75AFF38B1F8BD3E
:1077300022462846FFF754FF0028F8D17F42002058
:107740002F60F4E7FFF7F5FEF0E72DE9F04105467D
:107750000F4690464E6846B1BB6803EB860353F86C
:10776000043C43B1B8F1000F07D12846BDE8F04111
:107770000021FFF713BD013EEDE72846711CFFF71E
:1077800097FC044660B939462846FFF7D3FC044607
:1077900030B93046AA68B96808F1FF33FFF73BFA01
:1077A0002046BDE8F0812DE9F04F83469DB00F469D
:1077B0001846002116460393FFF7A5FE002800F0A7
:1077C00087810323002401251793304619AB0399C1
:1077D000CDE90A54CDE90C45CDE90E44CDE910546C
:1077E000CDE91245CDE9144416951893FFF715FE1F
:1077F000A04228DABBF1000F05D1E7B900242046EA
:107800001DB0BDE8F08F21465846FFF7C7FC04467F
:107810000028F2D00AA8FFF739FC0DA8FFF736FCC4
:1078200010A8FFF733FC13A8FFF730FC0C2119A8B0
:10783000FEF768F9E3E731463846FFF77BFC04467C
:107840000028E7D1DAE731460AA8FFF773FC0446BF
:107850000028DFD103990DA8FFF76CFC044600282F
:10786000D8D1716810A802310D950A95FFF720FC58
:1078700004460028CED1014610A8FFF78FFC04462D
:107880000028C7D1716813A80231FFF711FC044624
:107890000028BFD10DA8FFF7ADFC00F01F001F2886
:1078A00070D0C0F11F0319460AA80193FFF71CFD11
:1078B00004460028AED101990DA8FFF715FD044636
:1078C0000028A7D10B9DDDF838800DA8A5EB080A8C
:1078D0004FEA4A194946FFF707FD0446002899D1A7
:1078E0004FEA8A0A0DA90AA8FFF7CCFD00284BDA57
:1078F00049460DA8FFF74FFD044600288AD108F13C
:10790000FF3305939B0005F1FF3A069305F180458F
:1079100008F18043023B013D9B00A5EB080508935D
:10792000AB000293059B9A453DD8BBF1000F0CD0EC
:10793000584610A9FFF7FEFB002840F0C580039AC7
:10794000336812685343CBF80030002F3FF462AF26
:1079500001990AA8FFF71FFD002840F0B5803368A1
:107960000AA938460A93FFF7E5FB0146002840F0D4
:10797000AD803846FFF7C7FD00287FF44BAF0123E9
:107980003B6047E701949DE7129A0AA952F80A3032
:107990000846013342F80A300DAAFFF7B3FE044649
:1079A00000289FD036E70F9B069A04931344DDF816
:1079B00030900793049B4FEA8A089A5859F82A1086
:1079C000A8F10403129D0993029B91421D4476D2B3
:1079D000A8F10400002359F80000F8F7BBFB0029C8
:1079E00014BF4FF0FF330346BAF1010F2B600EBFF7
:1079F000002309EB080353F8083C1993A8F104038A
:107A000059F803301A9359F80830DDF810801B93A9
:107A10002B6801332B60089B98442B680021013BA5
:107A20002B6013A8FFF7BAFB00284DD1059B002B54
:107A300048D0D8F80020159B13A91A60079A084669
:107A400012685A602A68FFF780FE00283CD116A908
:107A500013A8FFF717FD0028DFDC2A680DA913A87B
:107A6000FFF773FE80BB029B13A84FEAC308414691
:107A7000FFF73AFC40BB0AA9084613AAFFF742FEEB
:107A8000014618BB0AA8FFF73EFD002812DA0DA92F
:107A900013A8FFF74FFBB8B9414613A8FFF724FC22
:107AA00090B90AA9084613AAFFF70AFE60B92B6825
:107AB000013B2B60029B0AF1FF3A043B31E74FF098
:107AC000FF3391E7059AB6E70446A3E60C46A1E624
:107AD0006FF00B0493E670B504460D461046002186
:107AE0001646FFF710FD002824DB2A4633462146C0
:107AF0000020FFF758FE054638B1284670BD3246D3
:107B000021462046FFF7DCFD90B900212046FFF713
:107B1000FAFC0028F3DB31462046FFF7B3FC0028CF
:107B2000EBDB324621462046FFF7ECFD0028F2D081
:107B30000546E2E76FF00905DFE72DE9F04F06465D
:107B4000ADF55B7D8946184600211D460592FFF77D
:107B5000DAFC002840F31382AB681C6814F00103C0
:107B6000089300F00C8200210598FFF7CCFC002858
:107B7000C0F205820598FFF73DFBB0F5006F00F2FB
:107B8000FE812846FFF736FBB0F5006F00F2F78163
:107B9000032104F102084FEA480808F00808A0444D
:107BA00008FB04F30139C3F1020303FB08F8F7D122
:107BB00001234FF440721AA8CDE90B31CDE90D1322
:107BC000CDE90F11CDE91431CDE9113116911391A1
:107BD000FEF7CDFC0598FFF70DFBB0F5287F80F090
:107BE000F580EF2800F2F4804F2800F2F380089B24
:107BF000182834BF1F4603276B68304603F1010A7B
:107C00005146FFF755FA0446002840F0BD80514622
:107C10001DA8FFF74DFA0446002840F0B5804FEA52
:107C20004A010EA8FFF744FA0446002840F0AC8051
:107C3000D9F80030069301330BD1494614A8FFF759
:107C400079FA0446002840F09F8001230DF1500985
:107C50001493E49B1BB19B68002B40F0BD80012175
:107C60000BA8FFF79BFA0446002840F08D80696856
:107C70000BA88901FFF738FB0446002840F08480F8
:107C80000BA92A460846FFF726FF044600287BD1A9
:107C9000E49B23B10C2218460BA9FEF75DFC294694
:107CA0004846FFF7EFFB0028C0F29A802A46494673
:107CB0001DA8FFF710FF0446002865D169681DA8BC
:107CC0000131FFF7F5F9044600285DD10DF1380BBD
:107CD000C8F100032A460BA91DA8CDF800B00393F4
:107CE000FFF735F930460BA9FFF724FA04460028C0
:107CF0004AD101230AAACDE917330A9319923046D3
:107D00002A46039BCDF800B017A9FFF720F9012FF1
:107D10006BD14FF0000AD046D346D146059B5B6835
:107D20000493BBF1000F40F0AF80049B002B40F0A8
:107D3000A6804FF0010B0DF1380A0BFA07FB049BEC
:107D4000434540F0FA8001230AAACDE917330A938C
:107D50001992039B2A463046CDF800A017A9FFF7D9
:107D6000F6F8069B01330FD1059B5B6863B1059B59
:107D70009B681B68DB0707D5069B324629463046C1
:107D80003360FFF79DFC044601237D1E03FA07F6CE
:107D90000C2703FA05F5AE4200F2EA801DA8FFF7B2
:107DA00075F90EA8FFF772F914A8FFF76FF911A87B
:107DB000FFF76CF9E49B0BB19B6813B90BA8FFF7B5
:107DC00065F920460DF55B7DBDE8F08F062713E7CA
:107DD000052711E704270FE70C22E4990BA85CE7BD
:107DE00049461DA8FFF7A6F96DE70C2307F1FF39F7
:107DF000696803FA09F31AAA02EB03084046013145
:107E0000FFF756F90028BED140461DA9FFF792F9A9
:107E10000028B8D1A2462A4641464046039BCDF8E9
:107E200000B00AF1010AFFF792F8CA45F3D34FF008
:107E3000010A0AFA09F9D1440AFA07FACA457FF693
:107E400068AF696808F10C0B58460131FFF730F94B
:107E5000002898D141465846FFF76CF9002892D186
:107E60000EAB00932A465846039B1DA9FFF76FF8F7
:107E7000D84609F10109E1E74FF0020A51E74FF056
:107E8000200B049B013B0493059B049A9B680BF118
:107E9000FF3B53F8223023FA0BF313F001030FD109
:107EA000BAF1000F3FF43DAFBAF1010F08D10EABAC
:107EB00000932A4631463046039BFFF748F830E7E7
:107EC00008F10108A7EB08029340474549EA030976
:107ED000D2D14FF0000A0EAB00932A46314630460D
:107EE000039B0AF1010AFFF732F8D045F3D80123CA
:107EF0004FF0000A03FA08F30DF1680849465046AE
:107F0000099300F03FF84146C2B211A800F052F8C0
:107F1000079058BB099B0AF1010A534508F10C0868
:107F2000ECD10EAB00932A463046039B11A9FFF714
:107F30000EF8DDE9079AC846F3E62A463146304690
:107F4000039BCDF800A04FEA4909FFF700F81BEAB0
:107F5000090F07D02A463046039BCDF800A01DA983
:107F6000FEF7F5FF049B01330493E8E6079C0BE75B
:107F70001AAB07FB0530FFF789F801350BE76FF007
:107F800003041EE7414048420843C043C00F704706
:107F9000F0B500255F420439013B854200D1F0BDB8
:107FA00052F8256051F8044F3E401C4034430C60A9
:107FB0000135F2E72DE9F8430F4649680546914639
:107FC000FFF776F88046C8B9C9F1000646EA090607
:107FD000F617F6432B683C68013301345C4004EA31
:107FE00049045C40013C2C604B46BA68A96878683B
:107FF000FFF7CEFF7B686A689A4202D84046BDE828
:10800000F883A96851F82320324041F82320013336
:10801000F1E700207047704770472DE9F8430446A8
:10802000DDE90876914698460D4651B9B9F1000F41
:1080300010D1B8F1000F15D1E7B91EBB55BB002018
:1080400006E00830FFF776F80028EFD0A0F5814071
:10805000BDE8F883494604F12C00FFF76BF80028CF
:10806000E7D0F3E7414604F13800FFF763F8002852
:10807000E2D0EBE7394604F12000FFF75BF8002877
:10808000DBD0E3E7314604F11400FFF753F8002892
:10809000D4D0DBE704F10800FFF7CAF86060CEE750
:1080A00010B5AC2200210446FEF761FA0023C4E9B2
:1080B000293310BD10B50446A0B38C30FEF7E6FF9F
:1080C00004F19800FEF7E2FF04F16800FEF7DEFF1E
:1080D00004F12000FEF7DAFF04F13800FEF7D6FFC6
:1080E00004F12C00FEF7D2FF04F11400FEF7CEFFDE
:1080F00004F10800FEF7CAFF04F18000FEF7C6FF96
:1081000004F17400FEF7C2FF04F15C00FEF7BEFF4D
:1081100004F15000FEF7BAFF04F14400BDE810403E
:10812000FEF7B4BF10BD6C220021FEF720BA2DE986
:10813000F84305460E4614467AB3036803F03F073A
:108140009B18036022BF4368013343609FB1C7F1AE
:1081500040094A450FD300F128084A4608EB0700BA
:10816000FEF7FAF941462846FCF720FAB0B93C443C
:1081700007464E44403C264404E02846FCF716FAE5
:1081800060B9403C3F2CA6EB0401F6D82CB105F1B8
:10819000280022463844FEF7DFF90020BDE8F883C6
:1081A00070B50D468021036800F1280603F03F03F7
:1081B0005A1C382A0344044683F8281006EB0200B0
:1081C00061D80021C2F13802FEF7D1F9D4E90031BB
:1081D0005A0F42EAC102DB0012BA1BBA31462046EE
:1081E00022666366FCF7E2F900284BD1E37A2B7034
:1081F00063896B70A3681B0AAB70A368EB70E37BA9
:108200002B71E3896B71E3681B0AAB71E368EB7157
:10821000E37C2B72638A6B7223691B0AAB7223693E
:10822000EB72E37D2B73E38A6B7363691B0AAB7399
:108230006369EB73E37E2B74638B6B74A3691B0A16
:10824000AB74A369EB74E37F2B75E38B6B75E36908
:108250001B0AAB75E369EB7594F823302B76638CBE
:108260006B76236A1B0AAB76236AEB76A36E4BB957
:1082700094F827302B77E38C6B77636A1B0AAB7714
:10828000636AEB7770BD0021C2F14002FEF76FF91F
:1082900031462046FCF78AF90028F3D101463822FE
:1082A000304691E7004700F0BAB973B5032800F2F1
:1082B000A780DFE800F0021927354FF05023022293
:1082C000C3F808230022C3F80421D3F804210122B3
:1082D000DA60002401238DF80730032800F2908033
:1082E000DFE800F02C69789A4FF05023012200213A
:1082F000C3F80823C3F80011D3F800110DF10704E7
:108300005A60E7E74FF050234FF40072C3F8082398
:108310000022C3F82421D3F8242101225A62D8E78D
:108320004FF050234FF48072C3F808230022C3F8A3
:108330002021D3F820210122DA61CAE742F2107528
:108340004FF050266CB3D6F8183403F003032370B3
:10835000D6F81834D90353D59DF8070001284FD11A
:10836000FFF7A1FF013DEDD14AE09DF8070001288C
:1083700046D1FFF798FF013D52D141E09DF807003B
:1083800001283DD1FFF78FFF013D39D0C4B1D6F8A8
:108390000C3403F001032370D6F80C34DB032FD523
:1083A000ECE7D6F81834DA032AD50120FFF77BFF73
:1083B000013DF6D124E042F210754FF05026E5E77A
:1083C000D6F80C34D8031BD50120FFF76CFF013D14
:1083D000F6D115E042F210754FF0502694B1D6F860
:1083E0005C3403F001032370D6F85C34D90307D55D
:1083F0009DF80700012803D1FFF755FF013DEDD19E
:1084000002B070BDD6F85C34DA03F9D50120FFF76D
:108410004AFF013DF6D1F3E742F210754FF05026C6
:10842000D6F85434DB03EBD5002C9ED10120A0E715
:1084300008B50520F9F744FD10B90520F9F71EFD30
:108440004FF050230122C3F81825C3F81425C3F8B0
:10845000802508BD08B5032819D8DFE800F00232EE
:108460003E4C4FF05022D2F81834D2F81814C903F9
:108470000ED4D2F81434DB0713D5D2F81C3403F031
:108480000303013B012B09D80223C2F8043308BDC2
:1084900003F00303022B05D0012B02D00020FFF7CD
:1084A00004FF01234FF05022C2F818350023C2F810
:1084B0000431D2F804310223C2F80433012393605B
:1084C000E5E74FF050230022C3F80021D3F8002144
:1084D0000122C3F804231A60D9E74FF05023002289
:1084E000C3F82421D3F824214FF40072C3F80423E5
:1084F00001221A62CBE74FF050230022C3F820215B
:10850000D3F820214FF48072C3F8042301229A612A
:10851000BDE7FFF7CABEF7B51646DDE9084701908B
:1085200001A81D46FCF762FA019BB6F1000C18BFCA
:108530004FF0010C00EB83000B1E18BF0123002D30
:1085400043EA4C0314BF4FF00C0C4FF0000C002C0E
:1085500043EA0C0314BF4FF4706C4FF0000C002F73
:1085600043EA0C0314BF4FF4403C4FF0000CD0F82A
:10857000002243EA0C0322EA030301B109780EB199
:108580003678760019430DB12D78AD0031430CB12A
:108590002478240229430FB13F783F040C433C4325
:1085A000C0F8004203B0F0BD1FB50DF10F030193F9
:1085B00000238DF80F101A4619460093FFF7ABFF02
:1085C00005B05DF804FB4FF4801070474FF4805005
:1085D00070474FF4807070470021FCF75DBE0223A6
:1085E000FCF7B2BD0323FCF7AFBD00210220FDF76D
:1085F00049B8704740B1C368587810F001001EBFF9
:108600001878B0FA80F040097047FDF7B0BFFDF769
:10861000A3BFEFF30580003818BF0120704708B1F1
:10862000F9F760BB70470000607BFF7F010000002E
:10863000D51B0000000000001528000090860000F7
:10864000592B0000A8860000592B0000C0860000AE
:10865000C1690000000000008D360000D8860000CF
:10866000312A000000000000B139000000000000C5
:108670002D6B000000000000C56900000000000034
:1086800025330000F08600009131000008870000CB
:108690005B990000D48A0000048B00002821002090
:1086A000702E00206689000095990000208B000044
:1086B000408B00002A210020142F00206089000038
:1086C000A1990000308B0000408B00002C2100207D
:1086D000202F00205A890000339C0000F48B0000FA
:1086E000288C000032210020142000205489000032
:1086F000EE9B000000000000D88B0000302100201D
:10870000000000004E8900006F9B00006C8B000091
:10871000BC8B00002E210020B048002048890000BA
:1087200000000000D564000000000000D5640000D7
:1087300000000000D564000000000000D5640000C7
:1087400000000000D564000031490000A58200004F
:1087500000000000D564000000000000D5640000A7
:10876000D88600000969000000000000D564000000
:1087700000000000D564000000000000D564000087
:1087800000000000D5640000114F0000A582000029
:1087900000000000D564000000000000D564000067
:1087A00000000000D564000000000000D564000057
:1087B00000000000D564000000000000D564000047
:1087C00000000000D564000000000000313A000005
:1087D00000000000D564000000000000D564000027
:1087E00000000000D564000000000000D564000017
:1087F00000000000D564000000000000D564000007
:1088000000000000D564000000000000D5640000F6
:1088100000000000D564000000000000D5640000E6
:1088200000000000D564000000000000D5640000D6
:1088300000000000D564000000000000D5640000C6
:1088400000000000D564000000000000D5640000B6
:1088500000000000D564000000000000D5640000A6
:1088600000000000D564000000000000D564000096
:1088700000000000D5640000E9560000A582000059
:1088800000000000D564000000000000D564000076
:1088900000000000D564000000000000D564000066
:1088A00000000000D564000000000000D564000056
:1088B00000000000D564000000000000D564000046
:1088C00000000000D564000000000000D564000036
:1088D00000000000D564000000000000D564000026
:1088E00000000000D564000000000000D564000016
:1088F00000000000D564000000000000D564000006
:1089000000000000D564000000000000D5640000F5
:1089100000000000D564000000000000D5640000E5
:1089200000000000D564000000000000D5640000D5
:1089300000000000D564000000000000D5640000C5
:1089400000000000D564000000800080FF7F0080F0
:108950000080FF7F00800080FF7F00800080FF7F1D
:1089600000800080FF7F00800080FF7FA19D0000CD
:1089700000000000AC9D000000000000B69D00005B
:1089800000000000C29D000000000000A99300004C
:10899000030000008799000003000000639C0000B2
:1089A00003000000059C000003000000F88E00009A
:1089B00003000000CD980000030000009B9E000013
:1089C00003000000ED9C0000030000007C9B000001
:1089D0000300000021940000030000003D9C000003
:1089E00003000000FFFFFFFFFFFFFFFFFFFFFFFF90
:1089F0000338FDD870470000010000009B92000082
:108A0000048A00000E0100000800000000000000C1
:108A10000000000000C00000F0860000010000001F
:108A200000C0000000020000F0860000020000000C
:108A300000C0000000800700F08600000300000076
:108A400000C20000007E0700F08600000400000065
:108A500000C20000007E0700F08600000500000054
:108A60000040080000800700F086000006000000BB
:108A700000C00F0000200000F0860000070000008A
:108A800000E00F0000200000F08600000000000061
:108A9000C364000000200020000000000600010068
:108AA00002000000A88A0000000000004C990000AD
:108AB00002000000E0FF0F00002000205499000099
:108AC00021000000E0FF06209D2700006D27000028
:108AD00000000000DD280000E1270000669900008A
:108AE000A5660000B76600006C9900009F66000054
:108AF000B16600007299000099660000AB66000044
:108B00007C99000081660000116600007366000019
:108B10000000000087650000000000000000000069
:108B2000FFFF00000028845000000000010000004A
:108B3000FFFFFFFF00258450000000000000000040
:108B4000DD2B0000BD660000C9660000DD66000088
:108B5000E7660000F1660000812A0000056700005A
:108B60000000000004000000FF0000000000000002
:108B700000000000000004030000000000020001EB
:108B80000100000000008000C2281700908B000048
:108B900000B002509C8B000001000000A48B00007C
:108BA0000600000011001D000D001F000E00200037
:108BB0000F0021001000220012001E00352E0000C0
:108BC0007D2F00008D3000002D2D00001D2D000098
:108BD000000800000010000015340000A933000058
:108BE0003D3300001D3300000D3300000400000081
:108BF000FF000000008000500200000000000000A4
:108C0000048C000000800050108C00000100000067
:108C1000188C000004000000140000001300020083
:108C20009601010095010300C16800004D34000069
:108C3000B368000011350000A3680000982F8A4235
:108C400091443771CFFBC0B5A5DBB5E95BC256399E
:108C5000F111F159A4823F92D55E1CAB98AA07D8B6
:108C6000015B8312BE853124C37D0C55745DBE72D9
:108C7000FEB1DE80A706DC9B74F19BC1C1699BE459
:108C80008647BEEFC69DC10FCCA10C246F2CE92DE9
:108C9000AA84744ADCA9B05CDA88F97652513E980D
:108CA0006DC631A8C82703B0C77F59BFF30BE0C614
:108CB0004791A7D55163CA0667292914850AB727A2
:108CC00038211B2EFC6D2C4D130D385354730A653F
:108CD000BB0A6A762EC9C281852C7292A1E8BFA216
:108CE0004B661AA8708B4BC2A3516CC719E892D17E
:108CF000240699D685350EF470A06A1016C1A41901
:108D0000086C371E4C774827B5BCB034B30C1C39FF
:108D10004AAAD84E4FCA9C5BF36F2E68EE828F74BE
:108D20006F63A5781478C8840802C78CFAFFBE90D8
:108D3000EB6C50A4F7A3F9BEF27871C6519E000007
:108D40005F9E0000739E0000829E00008E9E0000C9
:108D500030860000308600006886000070860000C3
:108D60009086000090860000FF8FFFFFFF8FFFFFBF
:108D7000FE8FFFFFFE8FFFFFFD8FFFFFFC8FFFFFCA
:108D8000FC8FFFFFFB8FFFFF436F756C64206E6FDE
:108D900074206C6F636B20706F77657220736176DF
:108DA00065206D75746578006D757465785F6672A1
:108DB00065652063616C6C65642077697468204E1A
:108DC000554C4C20706172616D65746572000000D5
:108DD00043616E277420696E697469616C697A6594
:108DE000206D757465782C20776173204E554C4C3E
:108DF0000D0A00000000F0FFF0FFF0FFEAFF74FF33
:108E0000F0FFF0FFF0FFF0FFEAFF77C295F360D2CA
:108E1000EF7F3552500F2CB6798025633A2053747A
:108E2000617274696E6720626F6F746C6F616465E4
:108E3000720A0025633A20556E61626C6520746F7A
:108E40002066696E6420626F6F7461626C65206970
:108E50006D6167650A0025633A20426F6F746C6F1D
:108E60006164657220636861696E6C6F6164206122
:108E7000646472657373206F66667365743A20303C
:108E80007825780A0025633A204A756D70696E6707
:108E900020746F2074686520666972737420696D30
:108EA00061676520736C6F740A0025633A20507205
:108EB0006F74656374206D6375626F6F7420666C88
:108EC000617368206661696C65642C2063616E6300
:108ED000656C20737461727475702E0A0025633A94
:108EE000204E657665722073686F756C64206765C7
:108EF0007420686572650A006D6375626F6F740037
:108F000025633A20696E76616C696420666C6173D2
:108F1000682049442025643B20657870656374654A
:108F2000642025640A0000000000000000002563A2
:108F30003A20556E61626C6520746F2064657465BB
:108F4000726D696E6520666C617368207365637409
:108F50006F72206F662074686520696D6167652097
:108F6000747261696C65720A007072696D61727900
:108F7000007365636F6E646172790025633A2049FE
:108F80006D61676520696E207468652025732073A4
:108F90006C6F74206973206E6F742076616C6964E5
:108FA000210A0025633A2025642073746174757367
:108FB000207772697465206661696C7320706572D0
:108FC000666F726D696E6720746865207377617073
:108FD0000A0025633A204661696C65642072656108
:108FE00064696E6720736563746F72733B20424FD0
:108FF0004F545F4D41585F494D475F534543544F70
:1090000052533D2564202D20746F6F20736D616C69
:109010006C3F0A0025633A204661696C65642072E2
:10902000656164696E6720696D6167652068656167
:10903000646572733B20496D6167653D25750A0063
:1090400025633A204661696C6564207265616469D4
:109050006E6720626F6F74207374617475733B2048
:10906000496D6167653D25750A0025633A20706189
:109070006E6963210A0025633A2053746172746932
:109080006E67206E6574776F726B20636F726520F8
:109090007570646174650A0025633A20446F6E65DB
:1090A000207570646174696E67206E6574776F7285
:1090B0006B20636F72650A0025633A20446574650E
:1090C0006374656420696E636F6E73697374656E33
:1090D0007420737461747573210A0025633A204308
:1090E000616E6E6F7420757067726164653A206E90
:1090F0006F74206120636F6D70617469626C6520AC
:10910000616D6F756E74206F6620736563746F7226
:10911000730A0025633A2043616E6E6F7420757088
:1091200067726164653A206D6F7265207365637460
:109130006F7273207468616E20616C6C6F77656408
:109140000A0025633A2043616E6E6F742075706764
:10915000726164653A206E6F742073616D6520736F
:109160006563746F72206C61796F75740A00626157
:109170006400676F6F6400756E7365740050726988
:109180006D61727920696D6167650025633A2025FC
:10919000733A206D616769633D25732C2073776195
:1091A000705F747970653D307825782C20636F701E
:1091B000795F646F6E653D307825782C20696D612C
:1091C00067655F6F6B3D307825780A005365636F84
:1091D0006E6461727920696D6167650025633A206C
:1091E000426F6F7420736F757263653A2070726995
:1091F0006D61727920736C6F740A0025633A2042A6
:109200006F6F7420736F757263653A206E6F6E6551
:109210000A0025633A205374617274696E67207383
:10922000776170207573696E67206D6F7665206158
:109230006C676F726974686D2E0A0025633A204E60
:109240006F7420656E6F7567682066726565207340
:109250007061636520746F2072756E207377617022
:1092600020757067726164650A0025633A20726533
:109270007175697265642025642062797465732054
:10928000627574206F6E6C79202564206172652090
:10929000617661696C61626C650A003082010A0264
:1092A00082010100D106081A18442C18E8FBFDF7CA
:1092B0000DA34F1FBBEE5EF9AAD24B18D35AE96D2E
:1092C000188019F9F09C341BCBF3BC74DB42E78C9B
:1092D0007F10537E435E0D572C44D167080F0DBBA2
:1092E0005CEEECB399DFE04D840BAA774160ED159D
:1092F0002849A701B43C10E6698C2F5FAC414D9E14
:109300005C14DFF2F8CF3D1E6FE75BBAB4A9C888E2
:109310007E473C94C37767544BAA8D3835CA626147
:109320007EB7E115DB7773D4BE7B7221896924FB9C
:10933000F8656E643EC80ED785D55C4AE4530D2FA0
:10934000FFB7FDF31339833FA3AED20FA76A9DF990
:10935000FEB8CEFA2ABEAFB8E0FA823754F43EE146
:109360002BD0D3085818F65E4CC8888131AD5FB059
:109370008217F28A692723F3AB873E931A1DFEE812
:10938000F81A246659F81CABDCCE681B666435EC11
:10939000FA0D119DAF5C3AA7D167C647EFB14B2CD0
:1093A00062E1D1C9020301000163627072696E74E7
:1093B000665F7061636B616765002D002B0030781C
:1093C00000305800286E696C29004661696C65643C
:1093D00020746F207265626F6F743A207370696ECB
:1093E0006E696E6720656E646C6573736C792E2E82
:1093F0002E0A0025633A20416E6F6D616C79203131
:109400003630207472696767657220636F6E6469B5
:1094100074696F6E732064657465637465642E0A85
:1094200000736F630025633A2072302F61313A2058
:1094300020307825303878202072312F61323A2060
:1094400020307825303878202072322F61333A204E
:10945000203078253038780A0025633A2072332F7F
:1094600061343A2020307825303878207231322F1C
:1094700069703A2020307825303878207231342FC6
:109480006C723A20203078253038780A0025633A0B
:109490002020787073723A20203078253038780A8E
:1094A0000025633A204661756C74696E6720696EA9
:1094B000737472756374696F6E206164647265732E
:1094C0007320287231352F7063293A203078253087
:1094D00038780A0025633A202A2A2A2A2A20555356
:1094E000414745204641554C54202A2A2A2A2A0A17
:1094F0000025633A2020204469766973696F6E20E5
:109500006279207A65726F0A0025633A202020551F
:109510006E616C69676E6564206D656D6F72792030
:109520006163636573730A0025633A2020205374D6
:1095300061636B206F766572666C6F772028636F4E
:109540006E746578742061726561206E6F74207628
:10955000616C6964290A0025633A2020204E6F203F
:10956000636F70726F636573736F7220696E73746B
:1095700072756374696F6E730A0025633A20202048
:10958000496C6C6567616C206C6F6164206F66204C
:109590004558435F52455455524E20696E746F20B2
:1095A00050430A0025633A202020496C6C656761AE
:1095B0006C20757365206F66207468652045505374
:1095C000520A0025633A202020417474656D70743E
:1095D00020746F206578656375746520756E6465A9
:1095E00066696E656420696E737472756374696F01
:1095F0006E0A0025633A202A2A2A2A2A2042555335
:10960000204641554C54202A2A2A2A2A0A0025633A
:109610003A202020537461636B696E672065727213
:109620006F720A0025633A202020556E73746163BF
:109630006B696E67206572726F720A0025633A204B
:1096400020205072656369736520646174612062D3
:109650007573206572726F720A0025633A202020AC
:109660004246415220416464726573733A203078F7
:1096700025780A0025633A202020496D70726563C1
:10968000697365206461746120627573206572720C
:109690006F720A0025633A202020496E7374727538
:1096A0006374696F6E20627573206572726F720ADF
:1096B0000025633A202020466C6F6174696E672D27
:1096C000706F696E74206C617A792073746174654F
:1096D00020707265736572766174696F6E20657251
:1096E000726F720A0025633A202A2A2A2A2A204DFC
:1096F0005055204641554C54202A2A2A2A2A0A002D
:1097000025633A202020537461636B696E6720657E
:1097100072726F722028636F6E7465787420617244
:109720006561206D69676874206265206E6F7420C2
:1097300076616C6964290A0025633A20202044611F
:109740007461204163636573732056696F6C617443
:10975000696F6E0A0025633A2020204D4D46415224
:1097600020416464726573733A20307825780A006A
:1097700025633A202020496E737472756374696F93
:109780006E204163636573732056696F6C61746901
:109790006F6E0A0052657365727665642045786362
:1097A000657074696F6E20280053707572696F75EB
:1097B0007320696E746572727570742028495251F5
:1097C000200025633A20535053454C20696E207485
:1097D0006872656164206D6F646520646F657320D5
:1097E0006E6F7420696E64696361746520505350B4
:1097F0000A0025633A202A2A2A2A2A20484152446C
:10980000204641554C54202A2A2A2A2A0A00256338
:109810003A202020427573206661756C74206F6E4B
:1098200020766563746F72207461626C6520726566
:1098300061640A0025633A20202044656275672030
:109840006576656E740A0025633A202020466175AE
:109850006C7420657363616C6174696F6E2028732A
:1098600065652062656C6F77290A0025633A20419F
:109870005243485F455843455054207769746820E7
:10988000726561736F6E2025780A0A0025633A209D
:109890002A2A2A2A2A204465627567206D6F6E691C
:1098A000746F7220657863657074696F6E202A2A00
:1098B0002A2A2A0A0025633A202A2A2A2A2A202527
:1098C0007320256429202A2A2A2A2A0A006D707505
:1098D0000025633A204661696C656420746F2061DD
:1098E0006C6C6F63617465206E6577204D505520F8
:1098F000726567696F6E2025750A0A0025633A2034
:10990000506172746974696F6E2025753A207361B5
:109910006E69747920636865636B206661696C6544
:10992000642E0A0025633A20496E76616C696420D2
:10993000756E6465726C79696E6720726567696FB0
:109940006E20696E6465782025750A00464C415387
:10995000485F30005352414D5F3000636C6F636B62
:109960004035303030006866636C6B006C66636C49
:109970006B006866636C6B3139326D006866636CCE
:109980006B617564696F00636C6F636B5F636F6EAF
:1099900074726F6C006770696F40383432383030E1
:1099A000006770696F403834323530300025633AD3
:1099B0002063696E7374722025303278207472616E
:1099C0006E7366657220746F6F206C6F6E673A20DD
:1099D000257A750A0025633A2072656164206572F4
:1099E000726F723A2061646472657373206F7220C3
:1099F00073697A652065786365656473206578703E
:109A000065637465642076616C7565732E4164646A
:109A1000723A203078256C782073697A6520257A2F
:109A2000750A0025633A2077726974652065727241
:109A30006F723A2061646472657373206F72207371
:109A4000697A6520657863656564732065787065FB
:109A5000637465642076616C7565732E416464720D
:109A60003A203078256C782073697A6520257A75DC
:109A70000A0025633A206572617365206572726F12
:109A8000723A2061646472657373206F7220736927
:109A90007A652065786365656473206578706563B1
:109AA0007465642076616C7565732E416464723AE6
:109AB000203078256C782073697A6520257A750ABC
:109AC0000025633A20756E737570706F72746564EB
:109AD000206174203078256C782073697A652025A0
:109AE0007A750A0025633A20657261736520657294
:109AF000726F72206174203078256C782073697AD7
:109B00006520257A750A00636C6561720025633AE9
:109B10002052445352206661696C65643A20256482
:109B20000A0025633A205145202573206661696C3F
:109B300065643A2025640A0025633A204A45444575
:109B400043206964205B253032782025303278202C
:109B5000253032785D20657870656374205B253030
:109B60003278202530327820253032785D0A006D39
:109B7000783235723634333566403000717370692F
:109B80005F6E6F720025633A20756E616C69676E57
:109B9000656420616464726573733A20307825309F
:109BA000386C783A257A750A0025633A20696E7612
:109BB000616C696420616464726573733A20307803
:109BC0002530386C783A257A750A0025633A206E7C
:109BD0006F7420776F72642D616C69676E65643A8B
:109BE0002030782530386C783A257A750A00666C12
:109BF0006173682D636F6E74726F6C6C6572403345
:109C00003930303000666C6173685F6E72660025B3
:109C1000633A204661696C656420746F20616C6CE6
:109C20006F6361746520505049204368616E6E65B2
:109C30006C0A0075617274403830303000756172A2
:109C4000745F6E7266785F75617274650025633A41
:109C500020526573657474696E67207379737465D7
:109C60006D0A00666174616C5F6572726F720025C7
:109C7000633A205475726E6564206F6E206E657451
:109C8000776F726B20636F72650A0025633A204517
:109C900072726F72207768696C6520777269746977
:109CA0006E672050434420636D643A2025640A00A7
:109CB00025633A204E6574776F726B20636F72650F
:109CC00020757064617465206661696C65640A0062
:109CD00025633A205475726E6564206F6666206E47
:109CE0006574776F726B20636F72650A00706364CE
:109CF000007065726D0074657374004255473B20B7
:109D000063616E27742068617070656E007265769D
:109D10006572740025633A205365636F6E646172E7
:109D20007920696D616765206F6620696D6167657F
:109D30002070616972202825642E2920697320759E
:109D40006E726561636861626C652E205472656134
:109D50007420697420617320656D7074790A002520
:109D6000633A205377617020747970653A202573C7
:109D70000A0025633A205377617020747970653A40
:109D8000206E6F6E650A00040104030402040104DE
:109D900001040301030304010401010000010000A8
:109DA000004E5246585F434C4F434B004E5246586C
:109DB0005F44505049004E5246585F4750494F54F7
:109DC00045004E5246585F57445400556E6B6E6FB7
:109DD000776E206572726F720025633A203E3E3EB8
:109DE000205A455048595220464154414C20455232
:109DF000524F522025643A202573206F6E20435025
:109E0000552025640A0025633A204661756C74204C
:109E1000647572696E6720696E74657272757074AC
:109E20002068616E646C696E670A0A00756E6B6EFD
:109E30006F776E0025633A2043757272656E7420E9
:109E40007468726561643A20257020282573290A98
:109E50000043505520657863657074696F6E0055D6
:109E60006E68616E646C656420696E74657272758B
:109E7000707400537461636B206F766572666C6FEB
:109E800077004B65726E656C206F6F7073004B6569
:109E9000726E656C2070616E6963006F73002A2AB0
:109EA0002A20426F6F74696E67205A6570687972F4
:109EB000204F53206275696C642076332E322E3920
:109EC000392D6E637332202A2A2A0A00FFFFFFFF12
:109ED000FFFFFFFFF96100000C8A000081650000B0
:109EE0000000000000C201000001030000000000AB
:109EF000B4480020B3480020000000001780000094
:109F000019800000138000000090D003FFFFFFFFC6
:109F10000000000000000000000000000000000041
:109F20000000000000000000000000000000000031
:109F30000000000000000000000000000000000021
:109F40000000000000000000000000000000000011
:109F50000000000000000000000000000000000001
:109F600000000000000000000000000000000000F1
:109F700000000000000000000000000000000000E1
:109F8000FF0000000000000000000000C0200020D2
:109F9000C0200020000000008D5A00000021002099
:109FA0000C21002004210020FC200020D8200020CB
:109FB0009C2F00203A00003AF55C0000415C000054
:109FC000755C0000BD5C000020210020E420002022
:109FD000182100200000000010210020A02F0020E8
:109FE0003A00003AA42F00203A00003AA82F00209F
:109FF0003A00003A000000000000000000000000ED
:04A0000015E015E072
:10C000003DB8F3960000000000020000F8060200B0
:10C010000000000000000000000000000000000020
:10C02000FFFFFFFFFFFFFFFFFFFFFFFFFFFFFFFF20
:10C03000FFFFFFFFFFFFFFFFFFFFFFFFFFFFFFFF10
:10C04000FFFFFFFFFFFFFFFFFFFFFFFFFFFFFFFF00
:10C05000FFFFFFFFFFFFFFFFFFFFFFFFFFFFFFFFF0
:10C06000FFFFFFFFFFFFFFFFFFFFFFFFFFFFFFFFE0
:10C07000FFFFFFFFFFFFFFFFFFFFFFFFFFFFFFFFD0
:10C08000FFFFFFFFFFFFFFFFFFFFFFFFFFFFFFFFC0
:10C09000FFFFFFFFFFFFFFFFFFFFFFFFFFFFFFFFB0
:10C0A000FFFFFFFFFFFFFFFFFFFFFFFFFFFFFFFFA0
:10C0B000FFFFFFFFFFFFFFFFFFFFFFFFFFFFFFFF90
:10C0C000FFFFFFFFFFFFFFFFFFFFFFFFFFFFFFFF80
:10C0D000FFFFFFFFFFFFFFFFFFFFFFFFFFFFFFFF70
:10C0E000FFFFFFFFFFFFFFFFFFFFFFFFFFFFFFFF60
:10C0F000FFFFFFFFFFFFFFFFFFFFFFFFFFFFFFFF50
:10C10000FFFFFFFFFFFFFFFFFFFFFFFFFFFFFFFF3F
:10C11000FFFFFFFFFFFFFFFFFFFFFFFFFFFFFFFF2F
:10C12000FFFFFFFFFFFFFFFFFFFFFFFFFFFFFFFF1F
:10C13000FFFFFFFFFFFFFFFFFFFFFFFFFFFFFFFF0F
:10C14000FFFFFFFFFFFFFFFFFFFFFFFFFFFFFFFFFF
:10C15000FFFFFFFFFFFFFFFFFFFFFFFFFFFFFFFFEF
:10C16000FFFFFFFFFFFFFFFFFFFFFFFFFFFFFFFFDF
:10C17000FFFFFFFFFFFFFFFFFFFFFFFFFFFFFFFFCF
:10C18000FFFFFFFFFFFFFFFFFFFFFFFFFFFFFFFFBF
:10C19000FFFFFFFFFFFFFFFFFFFFFFFFFFFFFFFFAF
:10C1A000FFFFFFFFFFFFFFFFFFFFFFFFFFFFFFFF9F
:10C1B000FFFFFFFFFFFFFFFFFFFFFFFFFFFFFFFF8F
:10C1C000FFFFFFFFFFFFFFFFFFFFFFFFFFFFFFFF7F
:10C1D000FFFFFFFFFFFFFFFFFFFFFFFFFFFFFFFF6F
:10C1E000FFFFFFFFFFFFFFFFFFFFFFFFFFFFFFFF5F
:10C1F000FFFFFFFFFFFFFFFFFFFFFFFFFFFFFFFF4F
:10C2000090800020DD02010003350200B102010030
:10C21000B1020100B1020100B1020100B10201004E
:10C220000000000000000000000000009DFD000074
:10C23000B10201000000000045FD0000B102010054
:10C240001DFE00001DFE00001DFE00001DFE000082
:10C250001DFE00001DFE00001DFE00001DFE000072
:10C260001DFE00001DFE00001DFE00001DFE000062
:10C270001DFE00001DFE00001DFE00001DFE000052
:10C280001DFE00001DFE00001DFE00001DFE000042
:10C290001DFE00001DFE00001DFE00001DFE000032
:10C2A0001DFE00001DFE00001DFE00001DFE000022
:10C2B0001DFE00001DFE00001DFE00001DFE000012
:10C2C0001DFE00001DFE00001DFE00001DFE000002
:10C2D0001DFE00001DFE00001DFE00001DFE0000F2
:10C2E0001DFE00001DFE00001DFE00001DFE0000E2
:10C2F0001DFE00001DFE00001DFE00001DFE0000D2
:10C300001DFE00001DFE00001DFE00001DFE0000C1
:10C310001DFE00001DFE00001DFE00001DFE0000B1
:10C320001DFE00001DFE00001DFE00001DFE0000A1
:10C330001DFE00001DFE00001DFE00001DFE000091
:10C340001DFE00001DFE00001DFE00001DFE000081
:10C350001DFE0000FFFFFFFF53B94AB9002908BFC7
:10C3600000281CBF4FF0FF314FF0FF3000F00CB839
:10C37000ADF1080C6DE904CE00F008F8DDF804E03A
:10C38000DDE9022304B07047704700BF2DE9F04794
:10C3900086468C460846089E154674461946002B6C
:10C3A00040F0C1808542B2FA82F245D94AB1C2F169
:10C3B000200300FA02FC954094402EFA03F343EA6E
:10C3C0000C0C4FEA154EA8B2230CBCFBFEF80EFB7A
:10C3D00018CC08FB00F943EA0C43994528D9EB181F
:10C3E00008F1FF3704D2994502D9A8F102072B447E
:10C3F000A3EB0903A4B2B3FBFEFC0EFB1C330CFB46
:10C4000000F044EA0344A04214D92C190CF1FF3384
:10C4100004D2A04202D9ACF102032C44241A43EA0C
:10C4200007401EB1D440002334607360BDE8F0873C
:10C430004746DDE76346F1E792BB431B01214FEA24
:10C44000154EAFB2200CB3FBFEFC0EFB1C330CFBF5
:10C4500007F840EA0343984561D9EB180CF1FF3027
:10C4600004D2984502D9ACF102002B44A3EB080397
:10C47000A4B2B3FBFEFC0EFB1C330CFB07F744EA33
:10C480000344A7424DD92C190CF1FF3304D2A74223
:10C4900002D9ACF102032C44E41B43EA0040C0E79C
:10C4A000C2F120039540944020FA03F12EFA03F3E1
:10C4B0004FEA154E9040AFB20343B1FBFEFC0EFBBA
:10C4C0001C10190C0CFB07F841EA0041884522D9E1
:10C4D00069180CF1FF3004D2884502D9ACF1020092
:10C4E0002944A1EB08019BB2B1FBFEFC0EFB1C1121
:10C4F0000CFB07F743EA01439F420ED9EB180CF1FE
:10C50000FF3104D29F4202D9ACF102012B44DB1B64
:10C5100041EA004193E76046E3E76146F7E760469A
:10C52000A4E76346B8E7834206D916B90021084656
:10C530007CE7C6E900E0F9E7B3FA83F78FB98342F5
:10C5400001D3724508D8BEEB020460EB030301205F
:10C550009C461EB9002169E73846FAE7C6E9004C57
:10C56000F8E7C7F1200CBB400EFA07F522FA0CF4ED
:10C570002EFA0CF1BA401C4320FA0CF3B8404FEAF3
:10C58000144901431FFA84FEB3FBF9F809FB183084
:10C590000B0C08FB0EFA43EA00439A4540D9E31816
:10C5A00008F1FF3004D29A4502D9A8F102002344D1
:10C5B000A3EB0A0389B2B3FBF9F809FB183308FBB4
:10C5C0000EFE41EA03418E452CD9611808F1FF3374
:10C5D00004D28E4502D9A8F10203214443EA004067
:10C5E000A1EB0E01A0FB02984145CE46434602D383
:10C5F00006D14D4504D20138B9EB020E68EB0403B5
:10C60000002EA7D0B5EB0E0261EB030101FA0CFC82
:10C6100022FA07F3F9404CEA0303C6E9003199E72F
:10C620004046C5E74346D9E72DE9F3415B4DD5F8D0
:10C630006031996811F001011AD140F6034001AA56
:10C6400004F02EFE0446002840F0A3800198C36841
:10C650001B785BB905F1CC03D3E8AF2F02F00902D8
:10C66000D3E8EF1FC3E8E42F002CF9D10DF03AF81E
:10C67000002141F2030001AA04F012FE0446002842
:10C6800040F08780019E0822F1684548013117F08B
:10C6900037F830460DF026F8214641F2010001AA94
:10C6A00004F0FEFD0446002873D10198C3685A784F
:10C6B00085F868205A88A5F86A201A7985F86920D3
:10C6C000B3F80720A5F86C20B3F80530A5F86E3054
:10C6D0000DF008F8214641F2020001AA04F0E0FD45
:10C6E0000446002855D1019C4022E1682D480131C3
:10C6F00017F006F820460CF0F5FF06F007FA04469E
:10C70000002846D195F882309A0638D5072140F6A0
:10C71000334004F07BFD0746002800F04D810721DF
:10C720000C300DF0E5F821460722064616F0F3FF1F
:10C730006FF009034FF0010833700623224634716D
:10C74000394640F6334086F80180F37004F0A8FDC6
:10C750000446F0B9414640F6314004F057FD064624
:10C76000002800F0298141460C3019F08FFB224649
:10C77000314640F6314004F093FD044648B995F83F
:10C7800074305B0612D44521074815F072FC6FF037
:10C790001204204602B0BDE8F08100BF0020002056
:10C7A00070200020782000200F9E0200002142F21D
:10C7B000030001AA04F074FD04460028E9D1019E9B
:10C7C0000822F168B848013116F09AFF30460CF0A3
:10C7D00089FF214642F2020001AA04F061FD0446ED
:10C7E0000028D6D1019CE368B3F8012091B2A5F8E6
:10C7F000FC2021B1DA78AD4811461AF061FF2046DD
:10C800000CF070FF95F8746016F0200618D1022124
:10C8100040F66D4004F0FAFC0446002800F0CC809D
:10C8200002210C300DF064F801232146037046709C
:10C83000324640F66D4004F033FD04460028A8D18E
:10C8400095F894301F0712D5002142F21C0001AA6E
:10C8500004F026FD044600289BD10198C368D3F854
:10C860000120D3F80530C5E936230CF03BFF95F8DD
:10C87000D0309E0624D568460DF1020104F068FD13
:10C880000446002885D1042142F2240004F0BEFCB5
:10C890000646002800F0908004210C300DF028F8A6
:10C8A000BDF8003022460380BDF802303146438097
:10C8B00042F2240004F0F4FC044600287FF469AF3F
:10C8C00095F8D0305C0610D5002142F22A0001AA6A
:10C8D00004F0E6FC044600287FF45BAF0198C368CF
:10C8E0005B7885F818310CF0FDFE082142F201005A
:10C8F00004F08CFC044600285ED008210C300CF0BB
:10C90000F7FF95F8D01040F2022311F0400F08BF56
:10C910000323024688074CBF43F02C0043F00C0071
:10C9200095F8D1308F0648BF40F0400013F0090F52
:10C9300095F89A3018BF40F4006003F00603CE0764
:10C9400048BF40F01000062B08BF40F4C070002123
:10C9500016F0DDFF2146002242F2010004F0A0FCA7
:10C96000044600287FF415AF95F87430B5F8FC1034
:10C97000980624D4C9B941F2050001AA04F090FC3C
:10C98000044600287FF405AFB5F8FC30019C4BB994
:10C99000E368B3F80120A5F8FC209A8843481146C3
:10C9A0001AF08EFE20460CF09DFE082140F6014054
:10C9B00004F02CFC044658B96FF06804E9E600293D
:10C9C000F3D145213A4815F054FB6FF00404E0E63A
:10C9D00008210C300CF08CFF95F8D0300246D907B6
:10C9E00057D44FF00051334816F091FF21460022F2
:10C9F00040F6014004F054FC044600287FF4C9AE20
:10CA0000014601AA4FF6014004F04AFC044648BB27
:10CA100001980CF067FE21464FF6024001AA04F08F
:10CA20003FFC0446F0B9019E0222F1682248013120
:10CA300016F066FE30460CF055FE95F8B9305B07EF
:10CA400010D521464FF6034001AA04F029FC48B94D
:10CA50000122019C1948E168114416F051FE20465C
:10CA60000CF040FE17F0BDF8044600287FF491AEAC
:10CA700007F09EF8044600287FF48BAEEB79002B7C
:10CA80003FF487AE08210E4816F02DFF05F002F99D
:10CA90007FE603A1D1E90001A6E700BFAFF3008064
:10CAA0009088000200800020D0200020002100207B
:10CAB000389E020010880002B9200020B820002013
:10CAC000CC200020014B1878704700BF384600206A
:10CAD00008B5044814F0F7FFBDE80840012019F03C
:10CAE0006ABC00BF568A020008B521B1BDE8084003
:10CAF000054814F0E8BF054814F0E5FFBDE808401C
:10CB0000012019F055BC00BF708A02008C8A020017
:10CB1000CB0710B506D500F00104204602F092FDC7
:10CB2000014B1C7010BD00BF3846002070B5037863
:10CB30008AB004460E4607AD032B20D8DFE803F089
:10CB400002191B1D1149284616F066FD05956378EC
:10CB50001E210493A37830460393E3780C4A029392
:10CB60002379019363790093A37914F0B9FF0AB094
:10CB700070BD0849E7E70849E5E70849E3E70A2106
:10CB80002846074A14F0ACFFE0E700BF978A02008E
:10CB9000C08A02009E8A0200A58A0200AF8A0200B3
:10CBA000B98A020030B5154689B00C4617F000FA74
:10CBB0006946FFF7BBFF35B922466946054814F0C0
:10CBC00082FF09B030BD2B4622466946024814F068
:10CBD0007AFFF6E7E38A0200028B020010B50C46EA
:10CBE00088B017F0E5F96946FFF7A0FF22466946CD
:10CBF000024814F068FF08B010BD00BF278B020088
:10CC000010B50C4688B017F0D3F96946FFF78EFFD0
:10CC100022466946024814F056FF08B010BD00BF16
:10CC20004B8B020000B589B017F0C2F96946FFF7D7
:10CC30007DFF6946024814F046FF09B05DF804FB29
:10CC40006E8B020010B50C4688B017F0B1F969463A
:10CC5000FFF76CFF22466946024814F034FF08B023
:10CC600010BD00BF858B020030B5304889B014F08C
:10CC70002AFF0EF085FE014628B12D4809B0BDE817
:10CC8000304014F020BF2B480EF0AAFE044648B9ED
:10CC9000294806F057FF60B1284809B0BDE8304088
:10CCA00014F011BF0146264814F00DFF2146254817
:10CCB000E4E7254806F060FF08B12448EDE704F0FA
:10CCC000FBFF014608B12248D8E7224814F0FBFEDA
:10CCD00015F0C6FE204802F0ABFC014608B11F4823
:10CCE000CCE71F4D03AC0FCD0FC42B68022223608D
:10CCF00001231C49009303A81B4B05F003FE0446C7
:10CD000028B10146194814F0DEFE09B030BD1848BC
:10CD100014F0D9FE013404F0010100200EF0F0FE01
:10CD200000214FF4803013F015FDF3E79B8B0200D8
:10CD3000C68B020011CB0000802100201D8C020058
:10CD4000E18B0200008C0200702100204A8C02005E
:10CD50007C8C02009C8C020068210020B38C0200B5
:10CD6000D07F02009080020088800200D08C0200F8
:10CD7000F68C0200014B1B68184700BF9821002069
:10CD8000014B1860704700BF9821002007B50B4683
:10CD9000002102460091034800F0E2FB03B05DF879
:10CDA00004FB00BF75CD000030B5002587B0CDE98C
:10CDB00003010446009503A90548059500F0D0FB42
:10CDC000DDE904309842B8BF255407B030BD00BF3C
:10CDD000A11A020070B589B306680122304614F02A
:10CDE000CEFE01460446304614F091FEC30708D437
:10CDF0001349AF22134815F028F9AF21104815F058
:10CE00001DF92146304614F098FE251829460022C7
:10CE1000304614F07CFE2D1AAC4206D00849B722E9
:10CE2000084815F012F9B721E8E72146304614F01A
:10CE30008AFE2146BDE8704014F0C6BF70BD00BF39
:10CE4000348D0200558D02002DE9F8430F46066827
:10CE50001446B2684B1EB2F5004F34BF04210821BE
:10CE60003B4010D0C7F1000909EA0709494503F121
:10CE7000FF3028BF494618420CD11F46BCB90025D7
:10CE80002846BDE8F8838F420FD82146BDE8F84315
:10CE900014F0DCBF2C492D484FF4A27215F0D5F8E0
:10CEA0004FF4A271284815F0C9F89946E6E7B2EBAD
:10CEB000D40FE4D9E319591A104614F06AFE01465A
:10CEC000304614F0C0FE80460028D8D0B36809EB85
:10CED000C005B3F5004F34BF042308231D44354477
:10CEE0007B1E1D447F423D40A5EB09052946304687
:10CEF00014F045FE2C44073424F00704A41B80459D
:10CF000007464FEAE40408D202464146304614F090
:10CF1000D4FE4146304614F015FF3946304614F031
:10CF20000CFE3844844208D239463046224614F07A
:10CF3000C4FE2146304614F005FF01223946304632
:10CF400014F001FE9CE700BF348D0200558D0200F5
:10CF5000B2F5802FF8B50CD2042A20D83B494FF403
:10CF6000F9723B4815F071F84FF4F971374815F034
:10CF700065F80823D21ACC1D114424F0070421F0CF
:10CF80000701091B17294FEAD1060AD82F4940F299
:10CF9000FB122F4815F059F840F2FB11E6E7042385
:10CFA000E8E70027046031463046A660E76014F0E9
:10CFB000F9FD012185000246304614F0EAFD1B35DB
:10CFC000ED082844B04234D83B46384604F10C0101
:10CFD0009A4237DA2A462046002114F0CCFD00237D
:10CFE00020461A46194614F09DFD771B1946204627
:10CFF000012214F0A8FD3A46294614F0BCFD2B4648
:10D0000000222946204614F08DFD3146204614F0BA
:10D01000B2FD3B4631462046002214F083FD3146E6
:10D020002046012214F08FFD2946BDE8F84014F097
:10D0300089BE06494FF40372054815F006F84FF40F
:10D04000037193E741F8040F0133C1E7348D020007
:10D05000558D02002DE9F84F0446A38B08461907A9
:10D06000164612D4022803F0070162D1204614F0BC
:10D070001FFF88B10138042800F22181DFE810F099
:10D0800059001F017E00C400F10001280CBF43F0CD
:10D09000100143F02001A18304F1140011F056FCAB
:10D0A000002800F0A98086F31188BFF36F8FBDE8D8
:10D0B000F88F03F00702501F01281ED80020062A0F
:10D0C0002768C4E9000014D13A4603E0E08B013040
:10D0D000E0831268002AF9D123F0070343F002022B
:10D0E0002046A28314F0E4FE90B342F02002A28313
:10D0F0002EE023F007039AB2F2E7042A33D123F09B
:10D1000007039AB22046A28314F0D2FE10B142F077
:10D110002002A283A38B03F00709894540F0D88041
:10D12000A18BCA0640F11E8121F01003A38301F0F8
:10D130000701D4F81880A38BB8F1000FB9DA0022E8
:10D14000276823F00703C4E9002243F00103A38307
:10D15000A38B03F00709894540F0BB80002FDFD087
:10D160000025AA463EE0844940F21B12834814F091
:10D170006CFF40F21B11804814F060FF41B17E4902
:10D180004FF4AB727D4814F060FF4FF4AB71F2E7DF
:10D19000236843B9784940F25712784814F055FF94
:10D1A00040F25711E7E723691D6845B972494FF40A
:10D1B000AD72724814F049FF4FF4AD71DBE70F46D2
:10D1C00088464FF00609A38B23F0070343F00603BC
:10D1D0009BB2A383A268002A7DD1002F7ED1002DAF
:10D1E0009ED0BA4643F0080304F1140B5846A383BB
:10D1F00011F0ACFB002873D16149C2225F4814F0E2
:10D2000024FFC2215E48B7E7022908D05A4940F2FC
:10D210005D125A4814F019FF40F25D11ABE7E78B3D
:10D2200047B155494FF4AF72544814F00EFF4FF414
:10D23000AF71A0E723695D6845B94F4940F26112BB
:10D240004E4814F002FF40F2611194E7A38BB846F8
:10D2500023F0070343F004039BB24FF00409A383B8
:10D26000B8E7012908D044494FF4B272434814F09A
:10D27000ECFE4FF4B2717EE7236843B93E4940F2B9
:10D2800065123E4814F0E1FE40F2651173E7236930
:10D290009D6845B938494FF4B472384814F0D5FE4A
:10D2A0004FF4B47167E70027A38BB84623F0070358
:10D2B00043F005039BB24FF00509A3838AE72E498B
:10D2C00040F26B122D4814F0C0FE40F26B1152E791
:10D2D000002700257EE74FF0010A83E7924681E7A9
:10D2E00086F31188BFF36F8FBAF1000F17D14FBBD0
:10D2F00015B120462349A8474FF02003EFF31186CC
:10D3000083F31288BFF36F8F584611F011FB08BBEF
:10D310001B499422194814F098FE942172E7A168E1
:10D320000029E4D00E680029E1D043464A46204651
:10D33000D1F804A0D0471EB1336831461E46F2E74B
:10D340003346FAE7394643464A4620463F6814F0DA
:10D35000DBFDCCE7584611F007FBA38B23F0080355
:10D36000A383DDE68B067FF597AE21F02003A38330
:10D3700001F007017AE600BF6D8D0200558D0200B5
:10D380008F8D020089D30000F8B504460D4600F1E8
:10D3900014064FF02003EFF3118783F31288BFF3D5
:10D3A0006F8F304611F0C4FA40B90A490A489422F6
:10D3B00014F04BFE9421074814F040FE304611F063
:10D3C000D3FAA5613A462046BDE8F8400121FFF7AF
:10D3D00041BE00BF8F8D0200558D02002DE9F04740
:10D3E00004460F4614F080FD051E5CDB04F11409B1
:10D3F0004FF02003EFF3118A83F31288BFF36F8F8E
:10D40000484611F095FA804638B93249942232489C
:10D4100014F01BFE94212F483AE0484611F0A4FA7C
:10D420004FF6FF72E38BA68B934206F007063DD0C2
:10D43000022E0ED135460133E383484611F086FAB9
:10D44000002839D12349C222234814F0FEFDC2210D
:10D45000E1E7062E13D8DFE806F0092C12120904C2
:10D4600009006FF085054FF00008E6E700233B60F8
:10D4700063687BB9C4E900777EB13546F3E71749A5
:10D4800015484FF4E47214F0E0FD4FF4E4711348D2
:10D4900014F0D4FD1F606760EEE75246022120467B
:10D4A000FFF7D8FD35462846BDE8F0876FF00A053E
:10D4B000D9E76FF00405D6E78AF31188BFF36F8FC1
:10D4C000B8F1000FEFD0002332463946204614F061
:10D4D0001BFDE8E78F8D0200558D02006D8D020067
:10D4E00008B54268034602F00302022A81600AD0AE
:10D4F000032A4FF0000103D0012A0AD1596006E047
:10D500001868596008BD186800225A6050B9002098
:10D51000F8E706490648452214F097FD45210348DF
:10D5200014F08CFD13F0F4FFF1E700BFBC8D020096
:10D53000558D020010B5094C0A44914200D110BD2E
:10D5400011F8013B58400309E35C0001C0B24340BD
:10D550001809205C1B01DBB25840EEE7DF8D0200AA
:10D560002DE9F04F81468B4617461C46002595B0A5
:10D57000387808B9284657E37B1C2528039306D042
:10D580005946C8470028C0F24F830135FBE11822F5
:10D5900000210EA816F0BFF87B78252B7DD0002344
:10D5A00098469E469C461E46781C014610F8012B64
:10D5B0002B2A00F0A18000F29880202A00F09F80A2
:10D5C000232A00F09F802BB19DF8403043F04003A8
:10D5D0008DF84030B8F1000F05D09DF8403043F091
:10D5E00020038DF84030BEF1000F05D09DF840308B
:10D5F00043F010038DF84030BCF1000F05D09DF8CA
:10D60000403043F008038DF840302EB19DF8403093
:10D6100043F004038DF840309DF8403003F044009F
:10D62000442803D16FF386138DF840309DF84030C5
:10D630002A2A43F080038DF840307FD19DF84120A5
:10D640004B1C42F001028DF841201A782E2A0CBFA3
:10D65000012100219DF8412061F341028DF8412014
:10D6600078D15A782A2A6ED000224FF00A0C013362
:10D67000194611F8010BA0F13006092E40F29580F1
:10D680009DF840101292C1F3400040EAD2700A4661
:10D6900060F341028DF840205CE0BA1C03928DF8E3
:10D6A00043309DF84130DA0740F12E8154F8048B65
:10D6B000B8F1000F07DA9DF84020C8F1000842F0E9
:10D6C00004028DF840205E0740F1278154F804AB36
:10D6D000BAF1000F80F226819DF841306FF34103CB
:10D6E0008DF841304FF0FF3A1CE12D2A0DD0302A41
:10D6F0007FF469AF012358E74FF0010C55E74FF075
:10D70000010E52E74FF001084FE701264DE70346AF
:10D710000EFB0262303A184610F8016BA6F1300C8D
:10D72000BCF1090FF3D999428FD09DF840101192A6
:10D73000D20F62F341018DF8401086E70B460022BC
:10D740004FF00A0EE7E79DF84120023342F0040251
:10D750008DF841201A786C2A47D02BD8682A31D00E
:10D760006A2A4BD04C2A51D01A4612F8013B782B2A
:10D7700003928DF843309DF8412000F2BE806D2B5E
:10D7800051D8692B00F2B980572B67D8412B03D0B1
:10D79000453B022B00F2B18004229DF8423062F337
:10D7A00002038DF84230012373E00CFB02020B46AA
:10D7B000303A5DE7742A25D07A2AD5D106219DF822
:10D7C00041200CE05A78682A9DF8412006D10121B9
:10D7D00061F3C6028DF841200233C5E7022161F3EF
:10D7E000C6028DF841200133BEE75A786C2A9DF8B5
:10D7F000412001D10421EBE70321F0E705219DF849
:10D800004120ECE707219DF84120E8E7BDF84020E2
:10D8100022F4F04222F0020242F4804242F002027C
:10D82000ADF84020DFE76E3BD9B201238B4040F2D8
:10D8300082410B4237D113F0240F51D1D8075CD568
:10D8400003219DF8423061F302038DF8423002F06B
:10D850007803A3F140014B424B411AE00120A3F1B0
:10D860005801C9B200FA01F111F4624F94D140F6A7
:10D87000010631421DD111F4043F3ED09DF84230E3
:10D8800060F3020302F07802402A8DF8423034D06F
:10D8900000239DF84020C2F340010B4363F3410293
:10D8A0008DF84020FDE602219DF8423061F302032D
:10D8B000E8E702209DF8421002F0780260F30201CE
:10D8C000402A8DF8421002BF9DF8401041F001013E
:10D8D0008DF84010632BDBD1131E18BF0123D8E74E
:10D8E00003219DF8423012F0780F61F302038DF8A6
:10D8F000423014BF01230023CBE79DF8403043F0B2
:10D9000001038DF84030C3E79DF94020002AACBFE9
:10D910004FF0FF38DDF84480D5E698077FF5E2AE9A
:10D92000DDF848A00023CDE911339DF842309DF881
:10D93000411003F00703012BC1F3C30133D1CB1E08
:10D94000042B04D8DFE803F0214646212100236898
:10D9500001294FEAE372CDE90E321CD19DF938302E
:10D96000DA17CDE90E3204349DF8403013F0030687
:10D9700050D03A4659464846039B14F048FB0028CD
:10D98000C0F252810544039FF2E554F8043BDA17D4
:10D99000CDE90E32E8E70229E5D11AB243F3C033EC
:10D9A000CDE90E23DFE7022B24D1CB1E042B04D8B4
:10D9B000DFE803F018101018180001294FF00002DA
:10D9C00054F8043B14D00229CDE90E32CCD19BB2DD
:10D9D0000E93C9E7073424F00704F4E80223CDE9E5
:10D9E0000E23C1E754F8043B0E9300230F93BBE7CB
:10D9F000DBB2CDE7042B08D1073424F00704D4E9C7
:10DA000000230834CDE90E23AEE7032BACD154F844
:10DA1000043BDDE79DF843007828B4D862281CD881
:10DA200025283FF4ADAD5828ADD1DDE90E010DF14B
:10DA30003603009310AA08AB14F0A3FABAF1000F52
:10DA4000074680F29980002F9DD00DF13603D81B38
:10DA5000002E00F0C0800130BDE06338152892D858
:10DA600001A252F820F000BF3DDB00004FDB0000B8
:10DA700087D9000087D9000087D9000087D9000026
:10DA80004FDB000087D9000087D9000087D900004C
:10DA900087D90000DBDB000073DB000099DB0000AE
:10DAA00087D9000087D90000C1DA000087D90000BB
:10DAB00073DB000087D9000087D9000073DB00000A
:10DAC000BAF1000F0E9F35DB5146384615F0C9FDFF
:10DAD00007EB000A002F3FF456AF00269DF84230B6
:10DAE00013F01002059200F0928002305B06119A4A
:10DAF00048BF129B104448BFC018B8F1000F0492F1
:10DB000040F39F809DF84020A8EB0008C2F38003FB
:10DB10005007069300F19580510640F188803EB190
:10DB200059463046C84700287EDB069B01351E4615
:10DB300030227DE0384615F08DFDC9E70E9B0026AA
:10DB400001208DF8203008AF0DF1210AC6E7190732
:10DB50005ABFC3F300135E012B26DDE90E23002B11
:10DB6000BFF663AF524263EB43032D26CDE90E238C
:10DB70005BE7002659E700269DF840200DF13603AB
:10DB8000DB1B6FF386129A458DF840207FF65BAF62
:10DB9000AAEB0303119356E70E9890B30DF13603E9
:10DBA0000093002108AB10AA14F0EBF9BDF8423045
:10DBB000BAF1000F03F0EF0343F4F04343F0100316
:10DBC0000746ADF84230D6DA00283FF4DCAE002636
:10DBD0000DF13603181A9A4680E70E9B07293FF687
:10DBE000D2AEDFE801F00C04060C08080C0C1D7026
:10DBF000C9E61D80C7E6EA17C3E90052C3E61D6007
:10DC0000C1E62F4F064607F1050A052066E71A0709
:10DC100048BF01306AE71046079306925946C84745
:10DC2000DDE90623002804DA15B0BDE8F08F2022D4
:10DC300043461946002903F1FF33ECDC454498467E
:10DC40006D1A2EB159463046C8470028ECDB013525
:10DC50009DF84230DA0601D41B0705D5594630201D
:10DC6000C8470028E0DB0135059B33B159469DF8D4
:10DC70004300C8470028D7DB0135049E2E4405E049
:10DC800059463020C8470028CEDB0135731B002BD6
:10DC9000F6DC53463A465946484614F0B8F900288F
:10DCA000C2DB0544A844A8EB0503002B7FF76BAE4D
:10DCB00059462020C8470028B6DB0135F3E700BFEE
:10DCC000EF8D020008B54FF02002EFF3118382F3CD
:10DCD0001288BFF36F8F02F031FB034813F0F3FE9D
:10DCE00001F04CFFFCE700BFF58D020008B54309C9
:10DCF0000CD0012B1BD01249124840F2472214F0DD
:10DD0000A4F940F247210E4814F098F94FF0FF3380
:10DD1000C340DA07EFD50C4B03EB8003D3F80022A6
:10DD200022F0E04242EA0171C3F8001208BD4FF64A
:10DD3000FF7300F01F00C340DB07DCD5034BEBE7AC
:10DD40001E8E0200558D020000258450002884504C
:10DD5000F8B54FF02003EFF3118783F31288BFF378
:10DD60006F8F0124234B244EC3F800450223032167
:10DD7000C6F8D0360020FFF7B9FF20460321FFF791
:10DD8000B5FF7E237F220025C6F80C37C6F83C3944
:10DD90001A4B2146C3F81821194A2120C2F8045E03
:10DDA000C2F8085E02F54822C2F81051C3F82451A7
:10DDB000C3F82C5103F5FF1303F58053C3F8A052A9
:10DDC000C6F80447C6F80449C6F8004BFFF78EFFB3
:10DDD00021462020FFF78AFF21460B20FFF786FF10
:10DDE00021460A20FFF782FF87F31188BFF36F8F68
:10DDF0002846F8BD001000500040005000200050A0
:10DE000000900350F8B50523194D1A4F2C781A4E7F
:10DE10000134B4FBF3F303EB8303E41A18F0EDF9D8
:10DE2000164A137873B157F82430C01A072809D856
:10DE300033782BB95721124814F01BF901233370A2
:10DE40000020F8BD00214FF050233170D3F81401A9
:10DE500038B1C3F81411D3F814312C700CB9012364
:10DE600013702C7818F0C9F947F824000120E8E76E
:10DE70003B460020C8360020394600203A460020A4
:10DE8000518E020048B1054B054A1B68B3FBF2F303
:10DE90005843044B43F001031847704764240020A3
:10DEA00040420F0080800200062807D10122044B67
:10DEB000C3F80025BFF34F8F20BFFDE7704700BFB9
:10DEC000004000500DF0CABF2DE9F7430F4606464B
:10DED0000821C06A14F067F980463C68DFF8489072
:10DEE000241A3C6004EA0905AC4203D8002003B0C0
:10DEF000BDE8F08308236A462146304614F0C6F890
:10DF00000028F4D16946304614F057F940B1BDF805
:10DF10000230BDF8042005EA090513441D443C60A5
:10DF2000A4EB0804E0E700BF0000FFFF2DE9F04785
:10DF3000044688B000F11407384619F08CFBA06A3B
:10DF40008368DB689847E06248B94521AB4814F024
:10DF500090F86FF01505284608B0BDE8F087A06A74
:10DF60008368DB6898470368013B1F2B02D9452172
:10DF7000A348ECE7A06A216805AA18F0A1F810B13F
:10DF80004521A048E3E7A5892DB1069BB5FBF3F237
:10DF900003FB125515B145219B48D8E7E389012BB6
:10DFA00002D845219948D2E7E36A009593F8049096
:10DFB0004FF0FF334FF0FF32384610F00BFD0821D1
:10DFC000E06A14F0F0F8A8460646E3891FFA85FADD
:10DFD000534508D8E389434523D1384610F0B0FDB6
:10DFE0006FF02C05B7E7A1892B04891B13FA81F187
:10DFF0004A4608232046009114F08DF878B169460E
:10E00000204614F051F808F1010808234A4620463A
:10E0100000991FFA88F814F07EF80028DAD001354C
:10E02000D3E753450BD1009908234A462046891B64
:10E0300014F071F818B96946204614F035F86946AD
:10E040002046FFF741FF054618B1384610F078FD2D
:10E0500081E7009B4FEA13484FEA08486360C4F821
:10E060000880D4E9011399420FD30823204601AA5E
:10E0700014F00CF805460028E7D101AB13F8012B8A
:10E0800091453CD10135082DF8D1636869461B0CD8
:10E090001B042046009314F007F84A462046A38943
:10E0A000009914F038F8051ECFDB636869D04FF68D
:10E0B000FF7906EB0308A3891FFA88F29B1B9A429B
:10E0C000CDF8008037D34921514813F0D2FF2046C4
:10E0D000616814F045F805460028B6D163684D4ADA
:10E0E000A18913400B44A3EB460363601340204611
:10E0F000A36014F044F90546002D5ED0A5E7204644
:10E1000001A914F05AF8626810B9921B6260A8E77E
:10E11000BDF80850BDF80610E06AC4F8088029442C
:10E1200014F041F840449042A060EED1002DECD0B4
:10E130006FF01C057AE008234146204603AA13F03D
:10E14000A5FF0546002880D1204603A914F035F824
:10E1500038B1BDF80C304B4503D1BDF81030002B61
:10E160006AD0B044A7E74A4620465B1A13F0D3FFB3
:10E17000051EFFF66AAF08D0E26AA368126813446E
:10E18000A360D4E901318B42EDD86168A38901EB2A
:10E1900046029A42B0D1DFF87C80A26801EA080307
:10E1A0009A42A9D0204613F0DBFF054600287FF4F1
:10E1B0004CAF636803EA0803A360A389A288A3EBBA
:10E1C00046039A422ED0384610F0BAFC012349216A
:10E1D000E28911482374A38913F04BFF6268492137
:10E1E00093B20E48120C13F044FFA268492193B277
:10E1F0000B48120C13F03DFF0025ACE69C8E02008C
:10E20000C38E0200E58E0200028F02001B8F020007
:10E210008C8F02000000FFFF438F02005F8F02001F
:10E22000768F0200204614F095F80546384610F027
:10E2300087FC002DCAD08EE64921084813F019FF4B
:10E24000636869461B0C20461B04009313F02CFFE7
:10E250002046009913F084FF4DE700BFB88F0200FD
:10E260002DE9F04F1D46037C04468946904689B04F
:10E270004BB94521624813F0FCFE6FF00C063046A6
:10E2800009B0BDE8F08FC26A0821104613F08BFF79
:10E2900082462946104613F086FFA3890746A3EB62
:10E2A0008A039D4200F2A9801DB1B8F1000F00F071
:10E2B000A48063680393204604AA03A9DDF80CB088
:10E2C00013F0B3FF06460028D9D1BDF810304B45F6
:10E2D00005D06268039B9A42EDD1E5B9CFE72046AD
:10E2E00004A913F06AFF0028F3D0BDF81200BDF8AE
:10E2F000143075B19D420ED14FEA1B41090401440F
:10E300002B464246204613F0DCFE002803DC06467E
:10E31000B5E7002BB3D0002F3ED104F114030193D5
:10E320004FF0FF324FF0FF3304F1140010F052FBB6
:10E33000DFF8D0B0E3899E425CD0D4E90123F9181C
:10E340008A422CD3ADF81A30FF2306A88DF81E3070
:10E35000ADF81890ADF81C5013F01CFF2B46424648
:10E36000A168204613F0ABFF29468246E06A13F00D
:10E370001AFFA2680244A260BAF1000F07D120463A
:10E3800006A913F0D6FF002814BF8246AA460198BA
:10E3900010F0D6FB564672E75744BFB2BDE70821DE
:10E3A000E06A13F000FF4FF6FF73ADF8183000235A
:10E3B000ADF81C301318ADF81A30A38902EA0B022D
:10E3C0001A44101A606006A813F0E4FE06A920465D
:10E3D00013F0AFFF2046211D13F066FE6368204650
:10E3E00003EA0B03A36013F0CAFF82460028CED1D4
:10E3F00001369FE76FF01B0AC9E76FF015063EE78D
:10E40000838E02000000FFFF2DE9FF471E46037CBC
:10E4100004460F469046BDF8309043B92C4845213C
:10E4200013F027FE6FF00C0004B0BDE8F087082160
:10E43000C06A13F0B8FEA389A3EB40039E4243D801
:10E440000025D4F804A0CDF804A0A9455146DDF874
:10E4500004A009D2636853451ED1BDF80830BB4201
:10E460001AD06FF00100DFE7204602AA01A913F0DD
:10E47000DCFE0028D8D1BDF80830BB4206D12046CA
:10E4800002A913F09AFE08B10135ADB26268019B92
:10E490009A42DAD15146E0E7BDF80C30002BE0D0CB
:10E4A000A945DED8BDF80A00090CB3424FEA014184
:10E4B00028BF334601444246204613F0E7FD0028BA
:10E4C000B2D1BDF80C00AFE76FF01500ACE700BFAC
:10E4D000838E020010B530B90B48452113F0C9FDF9
:10E4E0006FF0150010BD836833B90848452113F05B
:10E4F000C0FD6FF00400F5E71B6813B1BDE81040E4
:10E5000018471846EEE700BFD98F0200EF8F0200D0
:10E5100070B508B101B132B90B48452113F0A9FD1E
:10E520006FF0150070BD84680CB1E56835B9074817
:10E53000452113F09EFD6FF00400F3E741F8040B52
:10E54000E368BDE87040184712900200EF8F0200A8
:10E5500070B51346044630B91048452113F089FDC3
:10E560006FF0150070BD006830B90D48452113F0FB
:10E5700080FD6FF00100F5E782680AB1956835B952
:10E580000848452113F075FD6FF00400EAE70A46DC
:10E59000AC466168BDE87040604700BF4390020030
:10E5A00059900200EF8F020008B5042200210248B2
:10E5B00015F0B1F8002008BD0000072030B50C466A
:10E5C0000E4985B00291D0F8AC110546CDE9003175
:10E5D00000F1E0014FF0FF3320460FF0C9F950B9C8
:10E5E000012384F86430D5F8A83123B1204605B062
:10E5F000BDE83040184705B030BD00BF1F260200FF
:10E6000038B50C461146054614F00BF8034638B9E8
:10E610002846044914F005F803460020236038BD5D
:10E620000120FBE7C0B302002DE9F04F0123814632
:10E630000569466885B005F55977D7E8EF2F002AB8
:10E6400003D1C7E8E13F0029F7D140F0B880B368B3
:10E65000B26A043B2632B3EB420F4FEA420126BFB7
:10E66000B3FBF1F3B3FA83F300234FF0010428BFA7
:10E67000C3F12003013B9C4005F5E47800F099804C
:10E680001022082170689A4002EB4402043099403D
:10E690000932C5F86002063122F003020A44B16A69
:10E6A00001FA03FC510001EB4C01C5F86412B16A98
:10E6B000994000EB4103C5F858320333134423F06B
:10E6C0000303C5F854327368C5F85C42C5F850328C
:10E6D0003C4B4046C5E9A963316800F01DFA044689
:10E6E00030BBD9F804A0D9F81090DAE9073409F55D
:10E6F000307B012B584608BF103C10F0EFFE002382
:10E70000DAF8240030494FF4806201EB8021009355
:10E710005846234610F0F8FE09F52C702B4910F0EE
:10E72000EFFDDAF8140083685C681CB96FF05704D9
:10E73000002137E04B46264ADAF81810A047044675
:10E740000028F5D1DAF8140083681B69002BEDD09E
:10E750000122DAF81810984704460028E8D11D4B2A
:10E760002846C5F8A8311C4BC5F8AC311B4B0393A8
:10E77000D5F810320293D5F80832CDE90083D5F8E8
:10E780006832B26AD5F8601300F08EF904460028AA
:10E79000CED105F1E0000FF085FA0028C5F8680336
:10E7A0000ADB0221384613F071FF204605B0BDE8B0
:10E7B000F08F6FF00B04BBE76FF01504B8E76FF054
:10E7C0007704F2E775260200A84600205B260200C7
:10E7D0004F260200A5E800002D270200BD260200FA
:10E7E0002DE9F84306464FF001090569D0F8048089
:10E7F00005F55977D7E8EF3F022B03D1C7E8E29F31
:10E80000002AF7D149D1264805F1400114F032FF22
:10E8100020B16FF00F042046BDE8F883204805F1D1
:10E82000B00114F027FF0028F3D12846D5F8601373
:10E8300013F0AFFF044670BB71683669486983689E
:10E840001B6933B3224689699847044618BB06F50D
:10E8500030764946304610F0B7FE304605F5E4768E
:10E8600001F0B6FD3046D8F8001013F0CFFF044693
:10E8700088B90146E822304614F04DFF21464FF496
:10E88000E272284614F047FF2146384613F0FEFE98
:10E89000C1E76FF057040221F7E76FF07704BAE79A
:10E8A000C0B3020013B5044640B100230122CDE9F4
:10E8B0000032074BD0E909120FF00EF8A36E1B6867
:10E8C00023B1E06E02B0BDE81040184702B010BDA1
:10E8D000C0B3020013B504460846216901F5597119
:10E8E000D1E8AF1F022910D193B1A0B10121CDE928
:10E8F00000311346D0E909120EF0EEFF074B9842A3
:10E9000008BF6FF00B0002B010BD6FF00F00FAE708
:10E910006FF04C00F7E76FF00100F4E72EF8FFFF0F
:10E920002DE9F74388461546066906F55973D3E87D
:10E93000AF3F022B5FD1136823B96FF0150003B00E
:10E94000BDE8F0831B78002BF7D0D6F86093B9F1BF
:10E95000000F33D106F5D8774FF0FF324FF0FF3379
:10E96000384610F037F830462A6801A9FFF748FE0C
:10E97000019C1CB9384613F087FEDEE705F1080359
:10E98000A3666B6984F86490E366E46360B138461B
:10E9900013F07AFE21463046236E2A68FFF70EFEFA
:10E9A0000020C8F80040CAE72022296804F140008E
:10E9B00014F03CFE384613F067FEF1E730460F498D
:10E9C00013F02FFE04460028B7D005F10803836634
:10E9D0006B69C063C366002380F864302022296815
:10E9E000403014F023FE22460121304600F03EF86C
:10E9F0000028D5D0A1E76FF00F00A0E7C0B3020058
:10EA00002DE9F04F05460E4690460027D0F8B0A0FD
:10EA100085B0AAF5AE742146304614F02BFEE0B95D
:10EA2000114BA4F1400B0293DAF810303246CDE9D5
:10EA3000008329464FF0FF335846AAF5CE790EF0F1
:10EA400097FF60B97023012203FB079383F86420CA
:10EA5000DAF80C300BB158469847703417B105B04E
:10EA6000BDE8F08F0127D6E78F2702001FB51446B7
:10EA700090B18AB1012912D10A4B00F1E001029351
:10EA8000D0F8AC31403201934FF0FF332046009371
:10EA90000EF06EFF04B010BD6FF01500FAE7002015
:10EAA000F8E700BF8F2702002DE9F04387B00E463C
:10EAB000DDE90E811446DDE910251F4630B329B388
:10EAC000DFF850C000F1E009002D08BF65469EB98F
:10EAD000CDE9034400F5CE742046059618F08CFA73
:10EAE00003ABCDE900432A463B46414648460FF07A
:10EAF000FFF807B0BDE8F083002241460E92484679
:10EB00002A4607B0BDE8F0430FF01CBA6FF01500BD
:10EB1000EFE700BF01EA0000F0B50E46044689B0F9
:10EB200000286FD001230246C3630023D0F8981059
:10EB3000364F403040F80C7C42F8301FCDE90133AD
:10EB40004FF0FF330093C36D17F0BFFD304A06ABA3
:10EB500092E8030083E8030018460EF0DDFD054649
:10EB6000D8B904F134000EF0B7FD0546A8B939460E
:10EB7000284805AA17F081FD054670B9059B9A68DB
:10EB800072B10C33D4F89400C4F8A03013F030FE06
:10EB9000C4F8D40030B96FF00B05284609B0F0BDB9
:10EBA0000346EFE7D4F8940013F022FEC4F8D8002F
:10EBB0000028F0D0D4F88C30D4F8A010C4F8A830D5
:10EBC0000423C4F8AC30C4F8C4300223A362124B4F
:10EBD000B4F89420D4F8D470C4F8B810C4F8D010A5
:10EBE000D4F89010236204F1A403A4F8B020C4F870
:10EBF000A470C4F8C010A4F8C820C4F8BC00A66172
:10EC0000E362CAE76FF01505C7E700BF889002000E
:10EC1000E47F020092900200CC80020070B5114B9C
:10EC20000D461C68DCB1104B196800238B4202DBD7
:10EC30006FF0010070BD224612F8106B864202D0C0
:10EC400014460133F2E7E06810B96FF01200F1E703
:10EC500018F0A9FC0028F8D000202C60EAE76FF03B
:10EC60000C00E7E7082200206881020070B588B038
:10EC700005460C46C0B269461646FFF7CFFF00288E
:10EC80001BDB0098C8B14368226802938368019532
:10EC9000CDE903360023CDE906230593C56813F0BB
:10ECA00024FE6DB12846084901AA17F00DFA07980D
:10ECB00008B9059B236008B070BD6FF01500FAE736
:10ECC0006FF01200F7E700BF89290200F8B58368EA
:10ECD0000446002B31D0D0E90476C06813F076FEEC
:10ECE000A568B5FBF0F300FB13555DB1451BE0686B
:10ECF0008368DB689847A368017920682A4618442E
:10ED000014F009FDA368E06822683E442B44816842
:10ED10004D683146A847054638B10246334645217D
:10ED2000174813F0A6F92846F8BDE3695BB92369D3
:10ED3000A268134423610023A3600025F3E7535D19
:10ED4000DB4353550135A3682268AB42F7D8E0682E
:10ED500081680D683146A847054628B1452102461D
:10ED6000084813F086F9DEE73246E369A1682068B7
:10ED7000984705460028DAD0024645210248F0E7C8
:10ED80009A900200C3900200DE90020010B5436822
:10ED90000A680C469A4207D90548452113F069F9DB
:10EDA00000231846636010BD4A6801201344F9E748
:10EDB000F79002002DE9F7430D46DDE90A869146FA
:10EDC0001F46044680B179B172B100930023084612
:10EDD000019313F0FBFDB7FBF0F303FB107040B1A0
:10EDE0004521184813F045F96FF00D0003B0BDE858
:10EDF000F0836A462846144917F066F9019B002BF8
:10EE0000F2D008EB0602934202D245210F48E9E70F
:10EE1000284613F0DBFDB8FBF0F303FB108000285D
:10EE2000F3D1C4E90097E5602061A060C4F81480C4
:10EE300016B9019EA6EB08060C9B0020A661E361B3
:10EE4000D4E700BF1C9102008DED00005891020034
:10EE50002DE9F0410F4B05461C680E461746ACB134
:10EE60004FF0FF324FF0FF330B480FF0B3FD6368F4
:10EE70003246D3F8088029463B462046C047044620
:10EE800005480FF05DFE2046BDE8F0816FF00104FB
:10EE9000F9E700BFDC360020842700200023036050
:10EEA000044B5A6812B9C3E90000704710605860FB
:10EEB000704700BFE0360020014B1860704700BF6C
:10EEC000DC360020002330B585B00546CDE902339D
:10EED00001904FF0FF334FF0FF320B480FF07AFDF7
:10EEE0000A4B1C684CB9284600F0DCF8044606487A
:10EEF0000FF026FE204605B030BD636820461B6833
:10EF000001A998472468EDE784270020E036002017
:10EF10001FB5CDE9010103924FF0FF334FF0FF32EF
:10EF200009480FF057FD094B1C682CB906480FF033
:10EF300007FE204604B010BD636820461B6801A987
:10EF400098472468F1E700BF84270020E0360020BE
:10EF50000022024BC3E90022704700BFE0360020C8
:10EF60000022024BC3E90022FFF7F2BFE83600207F
:10EF70002DE9F74307460C4609B100230B60002634
:10EF8000234DDFF890904D4520D923492348942202
:10EF900013F05BF89421204813F050F8D5F8008066
:10EFA0003846414601AA13F062FD50B116B954B972
:10EFB0002E4606E000224046316813F058FD002836
:10EFC000F5D11435DFE7019B2360F1E7E6D3144B5D
:10EFD0001D68C5B155F8148C3846414601AA143D48
:10EFE00013F045FD50B116B954B92E4606E0002283
:10EFF0004046316813F03BFD0028F5D16D69E8E724
:10F00000019B2360F1E7304603B0BDE8F08300BF09
:10F01000447F0200BC7F02007E910200558D0200F9
:10F02000E83600202DE9F341DDF8208004460D4646
:10F0300016461F460190B8F1000F07D0D8F800100F
:10F04000C1B9D8F804E0BEF1000F1CD1204601A9D7
:10F05000FFF78EFF98B13B46D0F80880324629462C
:10F060000198C047034650B1224645210C4813F091
:10F0700000F804E001AA13F0FAFC0028E1D1002016
:10F0800002B0BDE8F081D8F808303246089329462E
:10F090003B46F446019802B0BDE8F041604700BF2E
:10F0A000B0910200F8B5064600251C4C1C4FBC422E
:10F0B0001BD91C491C48F42212F0C7FFF42119483F
:10F0C00012F0BCFF2EB9E3685BB92846054614343C
:10F0D000EDE700223146206813F0C9FC0028F2D188
:10F0E000F3E79847002DF0D1F0E7EBD30F4B1C6806
:10F0F00094B1143C1EB9E3684BB96469F8E7002287
:10F100003146206813F0B3FC0028F4D1F5E79847A6
:10F11000002D08BF0546F0E72846F8BD447F0200F1
:10F12000BC7F02007E910200558D0200E83600206F
:10F1300038B50C4D4FF0FF334FF0FF320A480FF057
:10F1400049FC2B783BB9FFF70BFF00F06DF8044644
:10F1500010B901232B70002403480FF0F1FC204666
:10F1600038BD00BF3C460020842700202DE9F04731
:10F1700080468946048FDFF8ACA0013498B0A4B271
:10F1800000F10806651EADB2B5F5004F47D04A2321
:10F19000294605AA304613F0C3F904F57F543F34DD
:10F1A000A4B207462146012330460DF10B0213F0AD
:10F1B000B7F9002F014603DC002803DC2C46E1E709
:10F1C000002816DCB8F83830AB4209D142466B1E35
:10F1D00022F8383F4FF4004102233046FFF740F851
:10F1E0002946304613F098F92146304613F094F939
:10F1F000E4E707F160030DEB03070023524607F82D
:10F200004C3C05A8CDF8009003AB0396ADF8104038
:10F21000FFF708FF0028D1D018B0BDE8F087002024
:10F22000FAE700BFDF2A02007FB501236946062006
:10F230000193FFF7F3FC0446002834D1062002AA0C
:10F2400001A9FFF713FD10F1130F04462BD038B1BD
:10F250000C3405D0404080F311884FF0040002DFE9
:10F260000399B1F5803F23D200231846009A946891
:10F27000084484421AD30133082BF9D10E4DA982D8
:10F28000EB8253682846AB60D368EB6313F0C1FC94
:10F29000044640B9094E28466E60FFF7FFFD284638
:10F2A0006E60FFF709FE204604B070BD9BB2E5E733
:10F2B0006FF02004F7E700BFF0360020C8210020DF
:10F2C0002DE9F84305464FF02003EFF3118683F351
:10F2D0001288BFF36F8F1B480FF02AFB40B91A4901
:10F2E00094221A4812F0B1FE9421174812F0A6FE9B
:10F2F0004FF00C0913480FF037FB154B154F1C68E6
:10F30000DFF8548054B90F480FF020FBA0B90E4924
:10F31000C2220E4812F099FEC221E6E7D4E9012389
:10F32000002D18BF13462BB198F8142009FB02F2E8
:10F33000B85C98472468E5E786F31188BFF36F8FC0
:10F34000BDE8F883303700208F8D0200558D020014
:10F350005037002044370020E8430020012270B5D8
:10F36000164B1C7D04F01F039A40D043144B6109D7
:10F3700003EB8103D3E8EF1F01EA0005C3E8E65F72
:10F38000002EF7D10A4213D00E4B0F4D8BB10C2338
:10F390006343EA185178E85C12F065FE0020FFF73D
:10F3A0008FFF0C235C4300232A192B51C2E9013340
:10F3B00070BD83F31188BFF36F8FEFE7E843002040
:10F3C0005837002067200200443700202DE9F04123
:10F3D000404B07461D7D4FF02003EFF3118883F368
:10F3E0001288BFF36F8F3C480FF0A2FA40B93B4937
:10F3F00094223B4812F029FE9421384812F01EFE58
:10F400000C246C4334480FF0AFFA364B364E195D7E
:10F410001A1991B107CA06EB040C8CE80700002208
:10F420001A552D480FF092FA044688B92B49C2228A
:10F430002B4812F00AFEC221DFE73946284600F0C9
:10F440005DF80028EDD007C8344484E80700E8E7F9
:10F4500088F31188BFF36F8F0C236B43F218F35CB2
:10F46000ABB37B1C0FD04FF4004C0021D2F808E066
:10F470001E480023EEFB0C011D4AFCF76DFF012125
:10F48000381A11F01BFC10F075FC0120FFF718FF73
:10F49000184B6A0903EB8203012205F01F018A4021
:10F4A000D3E8EF0F1043C3E8E10F0029F8D1124B66
:10F4B00033B10C236B43F2185178F05CFEF7F4FC87
:10F4C000FFF74CFF10F0A2FC2046BDE8F0811C467F
:10F4D000FAE700BFE8430020343700208F8D020098
:10F4E000558D020038370020443700203F420F007E
:10F4F00040420F0058370020A9DE00002DE9F04FF0
:10F5000085B00E4603A900F043F84FF400470446C7
:10F510004FF0000B1B4B039DD3F800A0431E1BB202
:10F5200003EB4303DFF8608005EB830524B9A146B4
:10F53000484605B0BDE8F08FC446594668680023C8
:10F54000E0FB07C1114A6046FCF706FFC446594676
:10F550000190A8680023E0FB07C10C4A6046FCF755
:10F56000FBFEBAF1FF3FA94601D0824505D9731CC5
:10F57000DED0019B1844B042DAD9013CA4B20C3D64
:10F58000D4E700BFDC2100203F420F0040420F00C3
:10F5900008B9024B0B600020704700BFF0800200EA
:10F5A0004B1E59425941014B197070473E4600208D
:10F5B00008B5012BBDF808100CD171B90A4B1B68B6
:10F5C0000BB9012008BD1078012809D800F001000E
:10F5D0009847F6E76FF00C00F4E76FF00600F1E7EC
:10F5E0006FF01200EEE700BF5C3700202DE9FF410D
:10F5F0001F460D4B054658680C46164680B1D1F89B
:10F600000C808047094B324618700123CDE90183F5
:10F61000BDF828302146009328463B4615F0ADFC46
:10F6200004B0BDE8F08100BF5C3700203D460020FB
:10F6300020B1034B02681A6042685A60002070478C
:10F640005C37002000B50E4B89B01B788DF80700A1
:10F650009BB10021182202A814F05DF8094B00208C
:10F6600003930DF107030493012302A9ADF81430AD
:10F6700006F06AFD09B05DF804FB6FF00C00F9E7D5
:10F680003E460020188102000449431E0F3013F843
:10F69000012F8A5C83421A70F9D17047E49102000D
:10F6A000F0B50746264E8DB001AD0C460FCE0FC506
:10F6B0000FCE0FC596E8070085E807003846002FF3
:10F6C00039D0002C39D0381F0246214610344B78EF
:10F6D0000D781B0443EA0563CD7804312B4311F800
:10F6E000025C8C4243EA052342F8043FEFD1042137
:10F6F000144C8A07036916D1C3F30742A55C1A0E9E
:10F70000A25C42EA0562C3F30725655DDBB2E35CF8
:10F7100042EA054242EA032221F0030330336B44FC
:10F7200053F82C3C534050F8042F013153402C29FE
:10F730000361DED101200DB0F0BD2046FBE700BF24
:10F74000EC7F0200E49102002DE9F04F00270368EE
:10F750009DB002934368DFF8BCA103938368DDE9A1
:10F7600002460493C36805930369DDE904BE06936A
:10F77000436907938369DDE9062C0893C3699846BA
:10F780000993089B0093CD590CAB2DBA5AF8049BF2
:10F79000DD514FEAF223A94483EAB213009D83EAC4
:10F7A00072634B4425EA020502EA0C0985EA090561
:10F7B0002B44434486EA0B054FEA743888EAB408C0
:10F7C000254006EA0B0985EA090588EAB45804379A
:10F7D000A844402F03EB0E054344DE46DDF80080CD
:10F7E00040F088804FF0100A4B490A9151460AF1C7
:10F7F000010A0DF1700E0AF00F070EEB870757F89C
:10F80000407C01F00F094FEAB748019788EAF718E2
:10F8100001F10E0707F00F070EEB870757F8407C42
:10F8200009314FEAF74E8EEA774ECDF82CE001F021
:10F830000F010DF1700E0EEB81010EEB890959F8E5
:10F8400040EC51F8401CBAF1400F7144DDF804E07F
:10F8500088EADE08DDF82CE041448EEA972E7144F8
:10F8600005EA02084FEAF52E2CEA050787EA0807A1
:10F870008EEAB51EDDF828808EEA756E774458F85A
:10F8800004EF49F8401C77440F4400994FEA733E57
:10F89000394484EA0607CDF828808EEAB30E07EAD9
:10F8A000030704EA06088EEAB35E87EA080777448E
:10F8B0000F4401EB0B0ECDF800C0B34622D10299E4
:10F8C0003944016003991944049B416023448360D7
:10F8D000059B3344C360069B73440361079B2B4421
:10F8E0004361089B13448361099B6344C3611DB05A
:10F8F000BDE8F08FB346CDF800C0264694461C46BE
:10F900002A4640E7944626462A461C4675463B460C
:10F910006CE700BFEC8102002882020010B50446AB
:10F92000C8B17022002113F0A2F90B4B0B4A0C490D
:10F93000C4E900230B4B0C48C4E902130B4BC4E988
:10F94000040301200A4BA36103F17453A3F52303BD
:10F95000A3F69243E36110BD85AE67BB67E6096A13
:10F9600072F36E3C3AF54FA57F520E518C68059BA1
:10F97000ABD9831F014811F0D1BE00BFEC82020059
:10F9800038B5044618B90F4B0F485B689847616853
:10F99000B1F5683F0FD0B1F5680F0CD00B4DA942FF
:10F9A00009D011F4686107D0214609480EF072FEB3
:10F9B00000232360656038BD1422206813F0ABFE7D
:10F9C000F8E700BF24250020E49202002C5F5CA928
:10F9D000643C002008B560B34368B3F5683F0ED0BF
:10F9E000B3F5680F18D0144A934220D000684FF046
:10F9F000FF324FF0FF330EF0EDFF58B115E001225A
:10FA00000368D3E8EF1F002903D1C3E8E02F0028E3
:10FA1000F7D10AD1002008BD0368084A1B7803F516
:10FA2000807352F82330002BF4D00548F3E70548E3
:10FA3000F1E76FF4E040EEE72C5F5CA900000350B3
:10FA4000E98FFFFFEA8FFFFF08B520B34368B3F5E6
:10FA5000683F09D0B3F5680F13D0114A93421DD007
:10FA600000680FF06DF814E000220368D3E8EF1F80
:10FA7000012903D1C3E8E02F0028F7D109D00948B4
:10FA800008BD00210368084A1B7803F5807342F81B
:10FA900023100020F4E76FF4E040F1E70348EFE7BC
:10FAA0002C5F5CA9E98FFFFF00000350EA8FFFFF86
:10FAB00010B5044618B91D4B1D485B68984763682C
:10FAC000B3F5683F2FD0B3F5680F2CD0194A934295
:10FAD00019D1236803BB4FF0FF324FF0FF332146AB
:10FAE00015480EF07FFD08B923681BB90F4B13486A
:10FAF0005B68984714220021206813F00CFE4FF435
:10FB00006863636008E0B3F5683F0DD83A2B03D013
:10FB100040F6BA629342DED1206817F09CFD63681C
:10FB200043F03A03636010BD054AF3E72425002043
:10FB3000E49202002C5F5CA9643C00200A9302005E
:10FB40003A00003A08B5064940231422054817F048
:10FB500057FDBDE808400449044811F051BE00BFFC
:10FB600064370020643C0020F48202000883020015
:10FB7000014910220A60704710ED00E072B6404063
:10FB800080F31188BFF36F8F01B5FEF73BF90028B2
:10FB900002D0BFF34F8F30BFBDE8014062B6BFF364
:10FBA0006F8F704772B6494081F3118801B5FEF737
:10FBB00029F9002802D0BFF34F8F20BFBDE80140D4
:10FBC00080F3118862B6704737B505460C46C9B157
:10FBD0008B6810480093D1E90023452112F049FABF
:10FBE000636945210093D4E903230B4812F041FADD
:10FBF0004521E269094812F03CFA4521A26908480A
:10FC000012F037FA2146284603B0BDE830400EF026
:10FC10009BBA00BF379302006B9302009F930200D0
:10FC2000B393020040B2002807DB01234109034AD5
:10FC300000F01F00834042F82130704700E100E0EF
:10FC400040B200280CDB01220649430900F01F00E6
:10FC50008240203341F82320BFF34F8FBFF36F8FD3
:10FC6000704700BF00E100E0054B420953F8222035
:10FC7000012300F01F0003FA00F01040704700BF9E
:10FC800000E100E00131072908B508D90D490E4807
:10FC90005B2212F0DAF95B210A4812F0CFF940B288
:10FCA0000028ACBF00F16040084B4FEA4111C9B2D7
:10FCB000ABBF00F5614000F00F0080F8001319544D
:10FCC00008BD00BFE6930200558D020014ED00E070
:10FCD00030BFFFF7FDBF00BF0B4A08B50B4B22F04A
:10FCE0007F029A60BFF34F8FBFF36F8FD3F88820E6
:10FCF00022F47002C3F888200EF0BEFA10F05CFE09
:10FD000000F0E0FA0EF0F8FA00C2000000ED00E0AA
:10FD1000094A0A49936809689867D96708494B688E
:10FD200043F080534B60002383F31188BFF36F8F40
:10FD30009368D86F704700BFE843002074890200C1
:10FD400000ED00E013498A684FF030001044EFF3F3
:10FD5000098C80E8F01F202080F31288BFF36F8F9A
:10FD60000D4F4FF00066CA698A603E60906F0023B5
:10FD7000936780F3118802F1300090E8F01F8CF354
:10FD8000098802F1000004B513F0C2FBBDE804408D
:10FD900070470000E843002004ED00E01EF0040F6F
:10FDA0000CBFEFF30880EFF30980816911F8021CA2
:10FDB0000229FFD001B513F09CFB01BD42F8203CA5
:10FDC000009B0B4942F81C3C019B21F0010142F8C9
:10FDD000183C029B42F8081C42F8143C4FF0807318
:10FDE00042F8043C0023203A02658367704700BF55
:10FDF000FB1A0200084B9860836E83F30B88104651
:10FE000081F30988002163B681F31188BFF36F8FF6
:10FE10000022002311F071FEE843002001B572B604
:10FE20000B4A906900281EBF0021916117F004FC65
:10FE300062B6EFF30580A0F110004FEAC00005495B
:10FE4000014409C99847BDE801400349084700003B
:10FE5000E84300202C7B02005DFE0000044B996803
:10FE6000D869884203D003494FF080520A60704736
:10FE7000E843002004ED00E038B5214C452121483D
:10FE800012F0F7F8A36A9D0103D545211E4812F030
:10FE9000F0F8A36ADC0103D545211C4812F0E9F80B
:10FEA000174DAC6A14F4801404D04521184812F0A0
:10FEB000E0F80224AB6A180303D54521154812F077
:10FEC000D8F80F4DAB6A590303D54521124812F0FB
:10FED000D0F8AB6A9A0303D54521104812F0C9F84F
:10FEE000074DAB6ADB0303D545210D4812F0C1F87D
:10FEF000AB6A20466FEA03436FEA1343AB6238BD37
:10FF000000ED00E01C9402003994020051940200BC
:10FF1000709402009F940200C2940200EC940200CC
:10FF20000B95020070B5234C06460D46224845212C
:10FF300012F09FF8A36AD90403D545211F4812F097
:10FF400098F8A36A1A0503D545211D4812F091F8C7
:10FF5000184CA36A9B0510D51A48452112F089F860
:10FF6000A26BA36A180408D54521174812F081F83E
:10FF70001EB1A36A23F40043A3620E4CA36A590581
:10FF800003D54521114812F074F8A36ADA050BD5A0
:10FF900045210F4812F06DF80020064A936A43F499
:10FFA0007F439362287070BDA36A9B04F4D54521FA
:10FFB0000848EFE700ED00E03B950200569502008F
:10FFC0006C95020084950200A2950200BC95020087
:10FFD000DC950200F995020070B52E4C06460D46E0
:10FFE0002D48452112F045F8A36ADB0603D54521CB
:10FFF0002A4812F03EF8A36A1C0703D54521284879
:020000040001F9
:1000000012F037F8234CA36A980710D545212548EC
:1000100012F02FF8626BA36A190608D54521224811
:1000200012F027F81EB1A36A23F08003A362194CD3
:10003000A36ADB0703D545211C4812F01AF8A36A0E
:100040009E0603D545211A4812F013F8114B9A6AFF
:10005000D40602D49A6A90070DD59B6AD9060AD5B0
:10006000144915484FF4AE7211F0EFFF4FF4AE7122
:10007000104811F0E3FF0020064B9A6A920642BF37
:100080005A6A22F400525A629A6A42F0FF029A6255
:10009000287070BD00ED00E02D9602004896020029
:1000A0006C950200809602009D960200B8960200B0
:1000B000F9950200DC960200558D020070B5694B7F
:1000C0000546586800268AB0C0F3080386F31188F5
:1000D000BFF36F8F02F07F44B4F17F4F07D102F07E
:1000E0000C04082C0ED145215F4811F0C2FF5F4976
:1000F0004FF484625E4811F0A8FF4FF484615B48BE
:1001000011F09CFF14074CBF0D460126002DEED0C8
:100110000024DA1E8DF80740092A00F29280DFE8F9
:1001200002F00585897090909090908D45215148FE
:1001300011F09FFF8DF807404A4CE36A9A0705D5F6
:1001400045214D4811F095FF002429E0E36A002B7A
:1001500002DA45214948F5E7E36A5B005DD54521B0
:10016000474811F086FF6369AA6943F480736361AD
:10017000BFF34F8FBFF36F8F636932F8022C23F404
:1001800080736361BFF34F8FBFF36F8F4DF60273C0
:100190009A421ED145212A683A4811F06AFF2C681C
:1001A0009DF807309BB92022294602A813F0A8FA2F
:1001B000099B002E51D0C3F3080222B96FEA5323E2
:1001C0006FEA43230993204602A9FFF7FDFC0AB01A
:1001D00070BDA36ADBB233B101200DF10701FFF757
:1001E000FBFE0446DCE7A36A13F47F4F05D0012031
:1001F0000DF10701FFF796FEF3E7A36AB3F5803F21
:1002000002D3FFF739FEECE7184940F2F222184812
:1002100011F01BFF40F2F22171E7144940F2F6227F
:10022000134811F012FF40F2F62168E700200DF1AB
:100230000701D4E700200DF10701DBE74521124853
:1002400080E7124910F4F87F114A124808BF0A46A5
:10025000103B452111F00DFF76E723F4FF7323F0E7
:100260000103AFE700ED00E044970200DC960200D6
:10027000558D02007497020090970200B697020015
:10028000C9970200ED9702000E980200169702002F
:100290002B97020037980200044B5A6942F0100273
:1002A0005A615A6942F480625A61704700ED00E079
:1002B000EFF30880EFF3098101B57246FFF7FEFE08
:1002C00001BD00BF002320210348C2180133452B84
:1002D00082F80013F9D1704700E100E0002080F3BC
:1002E0001488BFF36F8F002080F30A8880F30B8897
:1002F000FDF7E8FD00200E490860BFF34F8F0D4861
:1003000080F3088800F03EF8202080F311880A4826
:100310004FF40061401880F30988EFF31480022144
:10032000084380F31488BFF36F8FFFF7D5FC0000FC
:1003300094ED00E090800020506F0020BFF34F8FBD
:100340000549064BCA6802F4E0621343CB60BFF371
:100350004F8F00BFFDE700BF00ED00E00400FA058D
:10036000002318460649D1F89020C2F30722934291
:1003700000DB7047C1F89830C1F8A0000133F6E700
:1003800000ED00E010B572B6002484F31388FFF787
:10039000E7FF23464FF0FF300C4A03F12001013301
:1003A000102B42F82100F8D100234FF0FF30074A0C
:1003B00003F160010133102B42F82100F8D162B63D
:1003C000BFF34F8FBFF36F8F10BD00BF00E100E0A0
:1003D000084B9B6883420BD1EFF3058343B1064B77
:1003E0005A6842F080525A605A6A22F400425A62B5
:1003F00010F0E2B9E843002000ED00E01FB5094C21
:10040000094A23460121094800F024F900230393F7
:10041000074B0121E41A01A80193029400F034F97A
:1004200004B010BD00000720002000201883020047
:10043000B829002010B50C7A0B6804F01F0223F0D5
:100440001F031A43CB68640923F01F03054943EADD
:10045000440343F00103C1F89800C1F89C20C1F89F
:10046000A03010BD00ED00E030B50C684B6885B0E1
:100470000A894D890094013B24F01F04234402F0B3
:100480001F0242EA451223F01F03072804468DF895
:100490000820039309D902464521064811F0E9FDD9
:1004A0006FF01504204605B030BD6946FFF7C2FF66
:1004B000F8E700BF539802002DE9F04F8946144633
:1004C00006464FF00008544D85B0C84527DAD6F8E7
:1004D00004A0BAF1000F44D0BAF11F0F18D91AF0D6
:1004E0001F0F15D1D6F800B01BF01F0F10D15846C2
:1004F00013F012F807460AEB0B00013813F00CF862
:10050000874210D06FF015073A464521434802E074
:1005100042464521424811F0ACFD6FF015042046DB
:1005200005B0BDE8F08F17F1160FEDD0BC42EBDD42
:10053000C5F89870D5F89C10C5F89870D5F8A0301B
:1005400021F01F0143F01F0BD6E900321A449942F3
:1005500002F1FF3A1DD1D34507D13146F8B2FFF77A
:1005600083FF08F101080C36AFE73146C5F89870F3
:10057000D5F89C3022F01F0203F01F031343C5F887
:100580009C30E0B2FFF770FF10F1160FC5D0441C8D
:10059000E7E7C5F89870D5F8A020013B23F01F03CA
:1005A00002F01F021343D3453146E0B2C5F8A03034
:1005B000E8D0FFF759FF10F1160FAED0C5F89870CC
:1005C000D5F89C209DF808300BF1FF3B62F3040343
:1005D0008DF80830D5F8A0309DF808205B0863F34B
:1005E0004712D6E900310B44009323F01F0301307A
:1005F0005B44A3EB0A03C0B223F01F0307288DF866
:100600000820039303D902464521064883E769463B
:10061000FFF710FFBBE700BF00ED00E0A698020067
:100620007E980200539802000522044BC3F89420E0
:10063000BFF34F8FBFF36F8F704700BF00ED00E037
:10064000BFF35F8F0022024BC3F89420704700BFB6
:1006500000ED00E010B5094C2278FFF72DFF207067
:1006600016300AD1064907484FF48D7211F0EDFC9F
:100670004FF48D71024811F0E1FC10BD3F4600209F
:10068000CE980200558D02002DE9F74F2E4D8A4677
:1006900006464FF00008AB462C4FD04502DB03B0B6
:1006A000BDE8F08FD6F80490B9F1000F47D031685B
:1006B0000846019112F030FF0199044609EB010050
:1006C000013812F029FF84424FF01402204B10D061
:1006D00002FB08F36FF015024BF803201D491E487A
:1006E0004FF4957211F0B1FC4FF49571194811F067
:1006F000A5FC14F1160F2C60F0D01978A142EDDDA5
:1007000002FB08B0C7F89840C7F89840D7F89C405B
:1007100000F10801007B64F304000871D7F8A00021
:100720000C79400860F347140C71D7F89C1021F045
:100730001F016960D7F8A01021F01F01296108F19D
:10074000010814350C36A8E7843C002000ED00E0D9
:100750003F460020CE980200558D020038B51A4D54
:100760002C68082C0AD9194940F25112184811F086
:100770006CFC40F25111154811F060FC0020FFF7AD
:100780005FFF144B144AC3F8C020844213D1134BAB
:100790001C70FFF749FF0F4BD3F89030C3F30723CA
:1007A000082B0FD0094940F2BB12094811F04DFC4B
:1007B00040F2BB11DFE7696801EB0011FFF73AFE79
:1007C0000130E2E7002038BD24830200CE98020009
:1007D000558D020000ED00E0AAFF44003F460020D6
:1007E000014B1860704700BF2C2200200CB410B5DC
:1007F00086B009B90DF10B000024CDE9040109AB65
:10080000089A009404A905480393FCF7A9FE049BE9
:100810001C7006B0BDE8104002B070472F370200D0
:100820001022044B0020C3F840244FF05023C3F89B
:10083000140670470030005030B503788BB0044682
:1008400007AD032B21D8DFE803F0021A1C1E124962
:10085000284612F0E1FE059563781E210493A378E3
:100860000E4A0393E3780E48029323790193637948
:100870000093A37911F034F909480BB030BD094950
:10088000E6E70949E4E70949E2E70A212846084A78
:1008900011F026F9DFE700BF978A0200C08A020044
:1008A000404600209E8A0200A58A0200AF8A02000C
:1008B000B98A020008B508490848CA79C2EBC202E1
:1008C000FEF7C6FA024628B1BDE8084045210448B3
:1008D00011F0CFBB08BD00BF002000204E990200E0
:1008E00054990200F7B5054616461F461A4CD4E83F
:1008F000AF3FDA0729D538B94521184811F0B9FBBF
:100900006FF0010003B0F0BD01A912F0D4F8144952
:100910000246284612F0BAFE0028F1D1D4E8AF3FD3
:10092000C3F3C0051B0710D4CC3C07222146384630
:10093000B04706280BD845210A4811F09AFB072238
:100940002946204612F0E7FEE5710020DAE707238A
:10095000B0FBF3F0E071F8E7CC20002074990200BE
:10096000AC8A02009A9902002DE9F04188B0DDF8C6
:1009700038809C795D791E79DF7893F802C093F80E
:1009800001E01B78B8F1000F0ED0CDE90638CDE9B3
:1009900004CE1346CDE90267CDE90045084A11F0BF
:1009A0009FF808B0BDE8F081CDE905E3CDE9037C0F
:1009B0001346CDE90156034A009411F091F8F0E78F
:1009C000C4990200E899020001480EF033BD00BF4F
:1009D00030220020F8B5184DD5E8AF3F13F0010FD5
:1009E0002E4627D015F8C53CA5F1CC0783B901F0F8
:1009F000A3FC044628B14521104811F03AFB2046DB
:100A0000F8BDFB7923B901F0D9FC04460028F2D1E6
:100A1000D5E8AF3F5A0701D401F03CF9D6E8EF3FE3
:100A200023F48032C6E8E12F0029F7D1DB0301D59A
:100A3000FFF7CAFF0024E2E7CC200020099A020059
:100A400010B5FEF775FB044620B102464521024869
:100A500011F00FFB204610BD329A020030B5002481
:100A6000094D0A4B85B02846029303940EF036FDDB
:100A700002AB284600934FF4A3620A2304490EF008
:100A800043FD204605B030BD282D00206B9A0200A2
:100A9000A84A0020014601480EF032BE282D002051
:100AA000014601480EF092BE282D0020034630B4C6
:100AB0001A780846012A13D0022A26D072B9154A9C
:100AC00002F1100452F8045BA24241F8045BF9D130
:100AD00012780A705B8843731B0A837330BC7047BB
:100AE0000C4A02F1100452F8045BA24241F8045B84
:100AF000F9D112780A705B68C3F3072243731B0CA9
:100B0000C3731B0A82730374E8E7112230BC1946D1
:100B100012F0F6BD749A020038B50546012D104654
:100B200019460CD0032D16D0052D14D00C490D48B4
:100B30003D2211F08AFA3D21094811F07FFA0A4856
:100B400015F076F9044620B101210C3008F0F2FCD2
:100B50002576204638BD02460B460448F0E700BF24
:100B6000859A0200558D0200B0280020142800202C
:100B700010B50B460A490246D1F8380120B9BDE844
:100B800010400120FFF7C8BF08F0EEFD012100234F
:100B90000446017603820C3008F0CCFC204610BDE0
:100BA0000020002070B504460F2C0D461046194653
:100BB00005D80D2C0DD9BDE87040FFF7D9BF132C17
:100BC00007D10C4815F034F9044638B90024204602
:100BD00070BD02460B4645B10748F3E701210C30D2
:100BE00008F0A8FC01232376F1E70120BDE870405E
:100BF000FFF792BF4C2900207C28002038B5C3683D
:100C0000B3F801401B7863B9204602F085FB054626
:100C100040B9084B1A8822B96FEA04506FEA1050A5
:100C2000188038BD012102F07FFB2846BDE838401E
:100C300002F04ABB1C460020F8B5C5682E78BEB944
:100C4000B5F80170384602F067FB044630B93A4601
:100C5000BDE8F8404521074811F00BBAEB78314662
:100C6000037302F061FB2046BDE8F84002F02CBBA4
:100C7000F8BD00BFB49A020010B5C368B3F80140D4
:100C8000204602F049FB30B92246BDE8104045211C
:100C9000034811F0EEB9BDE8104002F015BB00BFEB
:100CA000DF9A020010B5C3681C88204602F034FBAE
:100CB00030B92246BDE810404521034811F0D9B9AA
:100CC000BDE8104002F000BBDF9A0200012108B528
:100CD0000C3008F0F3FDBDE80840027845210148DA
:100CE00011F0C7B9089B0200014608B5074808F093
:100CF00041FC0749074816F046FD021E05DABDE82B
:100D000008404521044811F0B4B908BD3C21002039
:100D10007C220020482E00202F9B020010B5084C9A
:100D20000146052294F8670002F03CFD38B994F8BA
:100D300067000422BDE81040024902F033BD10BD37
:100D4000002000202D99020070B5C568B5F801603B
:100D5000304602F0E1FA044630B93246BDE8704050
:100D600045210A4811F085B92B7823B90822E91CDE
:100D7000B53012F0C5FC201D4FF4805112F0B3FDC8
:100D80002046BDE8704002F09FBA00BFDF9A020023
:100D900030B405461446084602EBC3039C4201D119
:100DA00030BC7047224612F8081BA9420CD1028AB7
:100DB0006378934205D92B4630BC4521034811F096
:100DC00058B9636830BC18471446E7E7519B0200E6
:100DD00010B5012104460C3008F070FD2146BDE835
:100DE00010400A23014A0078FFF7D2BFE4830200D3
:100DF00070B5444808F010FC0446002800F08180DB
:100E0000027E012A4DD0032A78D1038A032B0BD806
:100E100040F2ED123C493D4811F017F9404080F393
:100E200011884FF0030002DF042104F10C0008F0E8
:100E300045FDFF22438806886276228AC6F30B00AE
:100E40009342608307D04521314811F012F92046C2
:100E500008F048FC14E002F05FFA054628B9452185
:100E6000628B2C4811F005F9F1E702F00FFB2146E7
:100E70006076320B284602F015F9284602F024FA73
:100E8000254BD3F83C31002B3BD02449244816F0A5
:100E90007AFC021E35DABDE870404521214811F088
:100EA000E8B8038A012B0BD840F66D121649174893
:100EB00011F0CBF8404080F311884FF0030002DFBF
:100EC000022104F10C0008F0F9FC0546007812F04C
:100ED000DCFC83070BD440F671120B490B4811F070
:100EE000B4F8404080F311884FF0030002DF06237E
:100EF00021460D4A2878FFF74BFFA8E745210B480C
:100F0000B0E770BD3C210020789B0200558D0200A7
:100F1000AC9B0200D59B0200002000207C22002018
:100F2000482E00202F9B0200B4830200FC9B02008D
:100F3000F8B50746907A0E46144608F0D3F9284BC8
:100F400083424BD1204608F0D5F90C23254D03FBF5
:100F500000504388BB4241D1234FD7F8380120B11C
:100F600008F0C0FB0023C7F83831204608F0C2F96A
:100F70000C2707FB005043689BB196B9204608F048
:100F8000B9F9012107FB00504268D2E90003127A47
:100F900003F01F07B9405B09D2B100EB830012F0E8
:100FA000A2FC204608F0A6F90C2707FB0050836836
:100FB000A3B1204608F09EF978432E54204608F04D
:100FC00099F907FB0055A868BDE8F8400DF008BF87
:100FD000C94300EB830012F091FCE2E7F8BD00BFCB
:100FE00018290020983C00200020002038B504215A
:100FF00004460C3008F062FC4578017822464088AF
:10100000FFF796FF25B1BDE8384002480DF0E8BE75
:1010100038BD00BF2021002038B5032104460C3024
:1010200008F04CFCE368057822461978B0F8010016
:10103000FFF77EFF25B1BDE8384002480DF0D0BE75
:1010400038BD00BF202100202DE9F0470025A8462B
:10105000C768DFF8D0903B789D4201DBBDE8F087A0
:1010600007EB8503B3F801A0B3F80360504602F024
:1010700053F90446D0B100F1280A46B34FF02003DB
:10108000EFF3118283F31288BFF36F8FE369A3B18B
:10109000013BE36182F31188BFF36F8F204601F0BB
:1010A0008FFF013E0DF09CFEB6B2E6E752464521A9
:1010B0001D4810F0DEFF0135CDE763695BB982F3AF
:1010C0001188BFF36F8F4521484610F0D2FF2046AC
:1010D00002F0FAF8EFE7A16918688B42606108BF77
:1010E000A06182F31188BFF36F8F4FF02002EFF3FE
:1010F000118182F31288BFF36F8FDA68E261C3F85F
:101100000C80C3F80080626A4AB9C4E9083381F3ED
:101110001188BFF36F8F50460EF08CF9BEE7136055
:101120006362F4E7369C0200159C020073B5C56843
:10113000B5F80160304602F0EFF8044638B932469F
:101140004521284802B0BDE8704010F092BF2B78CE
:10115000061D1A2B19D1C378012B2AD14FF48061B7
:10116000304612F0C0FB42050FD4D4F8A8306946CF
:101170000093D4F8B0302046019302F045FE20469B
:1011800002B0BDE8704002F09FB82B788BB9B5F87B
:101190000330A4F8A630B5F80530A4F8AC30B5F8A3
:1011A0000730A4F8AE306FF48071304612F0A6FB21
:1011B00014E0D6E8AF3FDB05F5D52B78202BF2D134
:1011C00094F8B430002BEED0013B84F8B4304FF4E7
:1011D0002032002304F160000EF0F2FA204602F003
:1011E0009DF9CCE7DF9A020010B5C1E900239DF814
:1011F00008300C460B7208F07DF80C22024B02FB03
:1012000000335C6010BD00BF983C00202DE9F04722
:101210004FF0FF3206464FF0FF331D480F4614F0E3
:1012200007FE044650B91B491B4840F2011210F05A
:101230000CFF40F20111174810F000FF4FF00008BA
:1012400000F10C0A0121504608F074F9204684F898
:10125000188008F04FF84FF00C09104D09FB0050B2
:101260004680204608F046F809FB0050C0F8088088
:10127000204608F03FF809FB005503215046C5F809
:10128000048008F035FB068087702046BDE8F087B3
:1012900018290020789B0200558D0200983C002000
:1012A00070B515460C4686B021B9FFF7AFFF04466E
:1012B000002841D001220021684616F001FA20469C
:1012C00008F018F80C231E4E03FB0060C0F808D08D
:1012D000204608F049FA01461A4808F0E3F94FF4AD
:1012E000A022002368460DF0B5FD58B140F2491226
:1012F0001549164810F0A9FE404080F311884FF0C0
:10130000030002DF204607F0F5FF0C235843365C4C
:1013100056B1204608F0E6F9092E14BF6FF004001C
:101320006FF06E0006B070BD15B12C600020F9E7BB
:10133000204608F0D7F9F9E76FF06800F2E700BF40
:10134000983C002044210020789B0200558D02002B
:1013500073B506460D4642F22F00002101AAFFF7A1
:101360009FFF044630B14521084810F082FE204618
:1013700002B070BD0198C368B3F801203280B3F8A1
:1013800003302B8008F0AEF9F1E700BF529C020059
:10139000F7B5144B054693F993300C46002B1DDA34
:1013A00014B9204603B0F0BD082C4FF0000142F202
:1013B000180001AA264628BF0826FFF771FF00285B
:1013C000F0D1019F3246F9682846013112F098F9B0
:1013D000384608F087F93544A41BE1E76FF0850033
:1013E000E0E700BF002000202DE9F047B0F80170D1
:1013F00000266FEA07536FEA135305468B4A9BB2E8
:10140000118888B0994204BF1680012600F0B4FD0F
:101410002C781FFA87F8F4B13C2C44D101F03AF94A
:101420006FF08001103012F069FA0020FFF776FCAF
:10143000054630B945217E4808B0BDE8F04710F0B8
:1014400018BE0473002101F06FFF284608B0BDE804
:10145000F04701F039BF2B7905F10409023B012B5C
:1014600024D8494606A812F03BFA9DF81830062207
:10147000023B05F111010DF111008DF8183012F049
:101480003FF901238DF81030EB78012B21D048462D
:10149000FFF7D2F945210246664810F0EAFD1F2108
:1014A000404612F044FA08B0BDE8F087EB784946B0
:1014B000012B04BF604B93F86740204612F052FBAB
:1014C000014606A812F00CFA494604A812F008FAE0
:1014D000DAE706A8FFF722FCEB780446012B0AD1D5
:1014E00001F0D8F882466FF08001103012F006FA51
:1014F000504612F051FC002CC9D0204606A920F815
:10150000907B12F0EDF90022B5F81730A4F8A63060
:10151000B5F81930A4F8AC30B5F81B30A4F8AE30EB
:10152000EB782273012BE37015D104A904F1970025
:1015300012F0D6F901F0AEF8217A3F4DC1EBC101AE
:10154000294404F19E0012F0CBF9D5F8DC305D0699
:1015500001D501F04BFA0721204601F0E5FE1EB14E
:101560000121204601F0E0FE204612F09AFC637B48
:10157000072B53D1231DD3E8AF3F13F4805F2E4ECA
:101580001FD1E3781BB196F8D030180719D5022186
:1015900042F21600FFF73AFE0546002842D002212B
:1015A0000C3008F0A5F9238800220380294642F276
:1015B0001600FFF775FE024618B145211F4810F0CE
:1015C00058FD96F8D130D9070CD5002102232046CA
:1015D0001A46009112F0E4F9024618B14521184864
:1015E00010F047FD96F8D0309A0617D5D6F860313E
:1015F0009B689B0712D50DF10E0103A8FFF7A8FE0B
:1016000060B9BDF80E202046BDF80C1012F0AAF902
:10161000024618B145210B4810F02BFD204601F081
:1016200053FE40E76FF06802C7E700BF1C4600208A
:10163000779C02009D9C020000200020BE9C0200BE
:10164000E49C0200009D020010B5C16888B00B78D0
:10165000164C8DF80030B1F8013001A8ADF801301A
:10166000CB7804318DF80330B1F80730ADF817307E
:10167000B1F80930ADF81930B1F80B30ADF81B30C6
:101680004B7B8DF81D3012F02BF9214606220DF10F
:101690000B0012F035F8062221460DF1110012F070
:1016A0002FF86846FFF7A0FE08B010BD4199020070
:1016B00029289ABF014B185C09207047AB9E020095
:1016C00070B5C368B3F801601D78304601F024FEA0
:1016D000044630B93246BDE870404521154810F047
:1016E000C8BC65B12846FFF7E3FF294602462046FD
:1016F00001F0ECFF2046BDE8704001F0E5BD8378C5
:10170000012BEFD106F05EF9204612F0D1F8002847
:10171000E8D10520FFF7CCFF05210246204601F065
:10172000D5FF4521044810F0A4FC0521204612F005
:10173000C1FBDFE7B49A0200219D0200F8B5C6683C
:10174000B6F801703578384601F0E6FD044630B948
:101750003A46BDE8F84045211A4810F08ABC65B108
:101760002846FFF7A5FF29460246204601F0AEFFB6
:101770002046BDE8F84001F0A7BD8278F378012A41
:10178000C37205D00020FFF793FF00210246ECE76B
:101790000BB106F017F9204612F08AF80028F1D1B3
:1017A0000520FFF785FF05210246204601F08EFF48
:1017B0004521054810F05DFC0521204612F07AFB1A
:1017C000D6E700BFB49A0200219D0200024BD3F875
:1017D00060315B69184700BF0020002038B505461E
:1017E0000C4619B9FFF712FD0446C0B140F6354367
:1017F0009D420ED12046FFF7E9FF054668B102463B
:101800004521084810F035FC204607F06BFF2846BC
:1018100038BD2146044807F045FF0025F7E76FF083
:101820006805F4E74C9D020044210020F8B5044609
:10183000458B467E807A07F055FD214615F036FF30
:101840001B4B93F882309B0631D5304602F0A8F945
:1018500068B3437B073B012B03D9BDE8F84001F097
:1018600033BD01F031FD052140F63540FFF7CEFCD8
:10187000044628B9BDE8F84045210E4810F0F9BBF0
:1018800000F10C070121384608F032F80126042146
:101890000670384608F02CF8002305808670C37067
:1018A0002146BDE8F84040F63540FFF797BFF8BD48
:1018B00000200020739D0200F0B5C46887B0268820
:1018C000B7B2384601F028FD054638B93A464521F9
:1018D000204807B0BDE8F04010F0CBBB02AFD4F811
:1018E0000220D4F8063001976189009113F01CFEA4
:1018F000F8B1122142F21A00FFF788FC044640B901
:101900004521154810F0B5FB284601F0DDFC07B075
:10191000F0BD12210C3007F0EBFF3946102220F801
:10192000026B11F0EDFE214642F21A00FFF756FF5E
:10193000EAE7022142F21B00FFF768FC0446002898
:10194000DED002210C3007F0D3FF2146068042F2A0
:101950001B00EBE7DF9A02009B9D020070B5064674
:101960000D4642F221000321FFF750FC044628B93E
:10197000BDE870404521084810F07BBB03210C30C6
:1019800007F0B6FF068085702146BDE8704042F240
:101990002100FFF723BF00BFB79D0200F7B5C36862
:1019A000D9789A781F8842EA0122ADF80020597947
:1019B0001A79BCB242EA0122ADF802209A79D979AB
:1019C000204642EA0122ADF804201A7A5B7A42EA04
:1019D0000323ADF8063001F09FFC064650B94521BF
:1019E0001C48224610F045FB02212046FFF7B6FFB7
:1019F00003B0F0BD694601F0E1FD38B91E21204673
:101A0000FFF7ACFF304601F05FFCF1E70E2142F238
:101A10002000FFF7FBFB05460028F3D00E210C3019
:101A200007F066FF04460E22002111F074FE2780A5
:101A3000BDF8003029466380BDF8023042F2200034
:101A4000A380BDF80430E380BDF806302381FFF7A2
:101A5000C5FED7E7DF9A02002DE9F047414FDFF8D6
:101A6000088107F11409FB6848466FF39433FB6063
:101A700001F0CEFB451C4FF0FF324FF0FF332946FB
:101A800038480FF093FC58B140F6E612414637480B
:101A900010F0DBFA404080F311884FF0030002DFC2
:101AA000304E15B90EF058FDDDE7F368C3F3863309
:101AB000042B4CD1337B002B4CD1002200232C482B
:101AC00014F0BBF9044658B94FF418624146274850
:101AD00010F0BBFA404080F311884FF0030002DFA2
:101AE000DFF890A04FF0FF334FF0FF3222480DF0A7
:101AF000B1F9DAF8383153B14521204810F0B9FA7C
:101B0000DAF8380107F0EEFD0023CAF83831204634
:101B100007F02AFECAF838012046FFF757FE0246B2
:101B2000A8B14521164810F0A4FA13480DF058F951
:101B3000204607F0DFFB0C22124B1F2102FB003076
:101B400022464088FFF7F4F9204607F0CBFD143613
:101B5000013DA6E7012BFAD13069383801F08CFF3E
:101B6000F5E700BF40220020789B0200558D02005F
:101B7000442100200020002020210020D69D0200CA
:101B80004C9D0200983C00202DE9F041044600F1F4
:101B90000C06304614F062F9B4F810800546B8F12E
:101BA000010F0BD840F67B521A491B4810F04DFA32
:101BB000404080F311884FF0030002DF30460221DD
:101BC00007F07CFE0746007811F05FFEC20706466C
:101BD0000BD440F67F520F490F4810F036FA4040C0
:101BE00080F311884FF0030002DF052321460B4AE2
:101BF0003878FFF7CDF8B30707D56369A4F81080EC
:101C000013FA85F5E560BDE8F0812046BDE8F041B6
:101C100007F068BD789B0200558D02008C8302009E
:101C200038B5027E0446012A05D0032A11D1FFF7F8
:101C30005BF8002038BDC368187811F026FEC20793
:101C4000054602D52046FFF79FFFAB07F1D520469A
:101C5000EDE74521044810F00CFA204607F042FD5C
:101C60006FF01500E6E700BFF69D0200084A034644
:101C7000D2F8600130B9D96839B1596929B1C2F8CF
:101C8000603170476FF0770070476FF01500704754
:101C9000002000200421014811F025BECC200020A6
:101CA00010B5FAF7C1FC034B1B6813B1BDE8104037
:101CB000184710BD103D002070B5354D0646D5F8CB
:101CC000603188B043B94521324810F0D2F96FF045
:101CD0001204204608B070BD6FF0020105F1CC007F
:101CE00011F00CFE012111F0FEFDC3074DD4FEF7EB
:101CF000A7FE04460028ECD1274B1E60012205F503
:101D00009070114615F0DCFC05F5A27015F0B6FCDC
:101D100000220023CDE906236FF008034FF4806210
:101D2000CDE90243CDE900441C4B1D4904941D48F4
:101D30000CF048FD1C491B4815F077FC1B480DF0C2
:101D4000CDFB6FF0070340F698021949174800943D
:101D50000DF0DAFB1749154815F067FCD5F860312E
:101D6000DB689847044628B102464521124810F026
:101D700080F9AEE726B908B0BDE87040FAF754BC68
:101D800005F1BC000DF056FBA3E76FF07704A0E768
:101D900000200020609E0200103D0020591A010022
:101DA000C04F0020C82D00207E9E0200482E00203B
:101DB000C0530020849E02008A9E020000487047A3
:101DC000188D0200F8B506460025094FFB79ECB2E4
:101DD000A34202D86FF0010009E0C4EBC401304611
:101DE000394411F034FE01350028EFD02046F8BD0B
:101DF0000020002037B504460D46A9B128461649F3
:101E000011F025FE80B929461448C4EBC4042044CF
:101E100011F025FE124811F025FE430701D5FEF70B
:101E2000D3FD002003B030BD684611F020FD00282E
:101E3000F8D16846FFF7C6FF0028F5DA074BC4EB78
:101E4000C4041C446946204611F009FE002DE1D06F
:101E500021462846DCE700BF34990200002000201C
:101E6000CC20002038B506221249054611F021FC8D
:101E7000D8B1062142F20500FFF7C8F90446B0B117
:101E8000062229460C3013F0F5FF0022214642F2CB
:101E90000500FFF705FA48B906222946054811F062
:101EA0002FFC0122044B83F86020002038BD6FF026
:101EB0006800FBE761200020002000202DE9F041B0
:101EC00005460C4686B051B929494FF45772294846
:101ED00010F0BBF84FF45771254810F0AFF80868C0
:101EE00040B9234940F25D32224810F0AEF840F28A
:101EF0005D31F1E745B91E4940F25E321D4810F0F0
:101F0000A4F840F25E31E7E7037A5A0708D518498A
:101F10004FF45872174810F098F84FF45871DBE7F7
:101F20004F68F7B92B7A5B071BD5691C013011F09C
:101F30008EFDD4F80080162239460646684611F018
:101F4000EAFB1022694608F12A0011F0B2FB58B1F1
:101F50002068102205F12A012A3011F0AAFB18B9D5
:101F6000656006B0BDE8F081002EF9D1F9E700BF49
:101F7000E19E0200558D0200084BD3E8EF2F22F4BA
:101F80000041C3E8E01F0028F7D1130404D5002264
:101F90000220034905F00CBE704700BFCC20002092
:101FA000C33B0200002307B50549CDE900036A469B
:101FB000022005F0FDFD019803B05DF804FB00BFB1
:101FC000BD1E0100F7B5054670B1494C94F81821C3
:101FD00094F819310AB19A4208D2013384F81931C0
:101FE0002B7A43F004032B7203B0F0BD00210622CC
:101FF000084601F0D7FB064688B1CC34D4E8EF3F61
:1020000043F40043C4E8E23F002AF7D12B7A43F0BF
:1020100001032B7203B0BDE8F04001F055B9014651
:10202000344800F031FB94F819318BB994F8192138
:1020300094F818319A4224D1002242F22900114624
:10204000FFF72EF998B145212B4810F012F804E063
:10205000304611F044FD0028E8D0012011F03FFD8A
:102060000021264803B0BDE8F04000F00DBB94F815
:102070001931013384F819312B7A43F004032B72A0
:10208000EBE72A466F1C394612F82A0B11F0EDFCDB
:10209000064610B145211A48D7E794F819310133A3
:1020A00084F819312B7A43F004032B7294F89F3093
:1020B0005B07D2D53946684611F0D1FC01230821CF
:1020C00042F24E008DF80730FFF7A0F8044660B1E9
:1020D000082269460C3013F0CDFE3246214642F20A
:1020E0004E00FFF7DDF80028B7D045210548ACE7E2
:1020F00000200020353B02000F9F02000F3B020032
:10210000349F0200599F02002DE9F041054698B323
:10211000444C94F8182194F81931D2B10132934209
:1021200023DC00210622084601F03CFB064628B3CA
:10213000CC34D4E8EF3F43F40043C4E8E23F002A44
:10214000F7D12B7A43F002032B72BDE8F04101F086
:10215000BBB853B93449354840F223420FF075FFFC
:1021600040F2234130480FF069FF013B84F81931F8
:102170002B7A23F004032B72BDE8F08101462C4832
:1021800000F082FA304611F0AAFC064680B1024601
:10219000452128480FF06DFF94F8193113B1012043
:1021A00011F09DFCBDE8F0410021234800F06CBA1D
:1021B00094F8193194F818219A420CD2013B84F812
:1021C00019312B7A024623F0040302201B492B729B
:1021D00005F0EEFCE0E7072142F22800FFF716F8D1
:1021E00005F10108074620B9452115480FF041FFC8
:1021F000D2E707210C3007F07BFB414611F02FFCA2
:102200003246394642F22800FFF74AF80028EBD15F
:1022100094F81931013B84F819312B7A23F0040327
:102220002B72B9E700200020E19E0200558D0200CC
:10223000353B0200799F02000F3B0200C93A0200C1
:10224000AB9F020070B50D46044618B9E5B16FF0BA
:10225000150070BD1D4911F0FAFB0028F6D1237856
:10226000012B04D1A37903F0C003C02B04D0452176
:1022700017480FF0FEFEEAE72046FFF7A3FD00280F
:10228000E4DB6FF07700E4E7124DEB79012B1AD015
:1022900005F1CC0011F0E6FBC3070BD5EE79214622
:1022A0003046FFF7A7FD0028D3D1EB793046013344
:1022B000EB71CEE7002CCAD02046044911F0C7FBD1
:1022C0000028EBD0C3E76FF00B00C2E7349902009F
:1022D000D59F02000020002073B5044698B100216C
:1022E00041F2090001AAFEF7DBFF064658B9019B3F
:1022F0000622DD680E490135284611F0DAF928B9C1
:10230000019807F0EFF9002002B070BD06222846C0
:10231000084911F0CEF90028F2D006222946601CA7
:1023200011F0EEF90198267007F0DCF90120EBE7D7
:10233000419902003B99020007B56846FFF7CCFFC0
:10234000044BD87118B169460020FFF753FD03B064
:102350005DF804FB002000202DE9F341164B0746F1
:1023600093F8BA308846DB0704D40026304602B022
:10237000BDE8F08100214FF6094001AAFEF790FF69
:1023800004460028F1D1019BDD686E780235464590
:1023900028BF46464FF01608A64203DC019807F016
:1023A000A1F9E3E7294608FB0470162211F0A8F909
:1023B00001341635F0E700BF00200020F0B5154EBF
:1023C00089B0F4792CB9012102A8FFF7C5FFF0719B
:1023D000C8B90021084609B0BDE8F040FFF732BF98
:1023E00002AB07FB053106220DF1010011F088F95F
:1023F0000123694628468DF80030FFF7FBFC0134C5
:1024000010B109B0F0BD1627F379E5B2AB42E7D8B9
:102410000020F6E7002000202DE9F04190460E460E
:102420001D46024600284BD0002B49D0CF07047828
:1024300031D5254FB8F1000F13D088060AD4C4EB6C
:10244000C403FB5C012B15D02B70B2060FD543F0F3
:1024500002030BE097F8D0305906F0D46FF08500F6
:1024600006E0C4EBC403FB5C012B03D02B700020FF
:10247000BDE8F081072101FB04711046013111F024
:102480007DFB0028F4D1C4EBC4043B5D2B70B8F194
:10249000000FECD0D9E74B070ED50B4EC4EBC407A9
:1024A000F35D012BE2D1072111FB0431314411F01E
:1024B00065FBF35D2B70DBE711F068FB0123F9E7A7
:1024C0006FF01500D4E700BF002000202DE9F74F82
:1024D0000C46202192460090FEF798FE0546002803
:1024E00054D020210C3007F003FA2022814600212D
:1024F00011F011F9002609F1010B04EBCA0A0023BF
:10250000D4F80080626893420CD30834A245F6D117
:1025100000222946009889F8006003B0BDE8F04F1A
:10252000FEF7BEBE98F80120B01C11181F2998F8BC
:1025300000C014D9BCF1090FC0F11F0201D1002A5B
:102540000BDC452113480FF094FD284607F0CAF82C
:102550006FF0150003B0BDE8F08F4FF0080CD7B254
:10256000791C0BF80610711CC9B20BF801C0D8F821
:1025700004105BFA80F00193023711F0C1F8019B5F
:102580003744FEB2013308F10808BBE76FF068007A
:10259000E0E700BF0EA0020070B50546164B15F827
:1025A000092B044683F867200E4607222846134964
:1025B00011F07FF8034620786BB9114901F0BCF89F
:1025C000044610B96FF00B0070BD042100F0ACFEA2
:1025D00000203460F8E7294611F0E2FC40B9207889
:1025E000294601F0A9F804460028EBD00521EDE7C3
:1025F0006FF01500E8E700BF0020002034990200CA
:102600002D99020038B543680446580501D50020CD
:1026100038BD22690AB1D907F9D5194D2078EB796F
:102620008342F4D9C0EBC00007221649284411F0B8
:1026300040F80028EBD06068C20706D495F86830EF
:10264000082B02D8A3689F2BE1D910F0300F02D0DD
:102650002369002BDBD0C30601D4236943B9D4E935
:1026600002239A42D3D81F2AD1D9B3F5804FCED8AE
:1026700000F46030B0F5603018BF0120C8E700BF3B
:10268000002000203499020003460148184700BF8B
:102690001820002000487047182000202DE9F04F36
:1026A0009A460023D1F810908DB0B9EB0306054689
:1026B000904818BF01260592079311F0A3FA42072C
:1026C0000C4640F10B810846FFF79CFF28B96FF0DC
:1026D000150B58460DB0BDE8F08F204611F06DFA8D
:1026E00080460028F3D005F11007384611F08AFA29
:1026F0000306C0F3C01B00F1F4800F22594608A85E
:1027000011F009F8A3686068ADF82030E368ADF80F
:10271000223011F068FA2A7823788DF82D009A4239
:102720008DF82EB004D06FF40051724811F06DFA9C
:102730002378714A2B7082F86730284632466168E8
:102740000DF12503FFF768FE83460028C1D107225B
:1027500005F10900B9F1000F13D0216910F0D0FF85
:10276000204611F0E2FA62680646D00716D49205B8
:1027700003D4169B0BB9022E52D102238DF82430BC
:102780001AE05E4910F0BCFF204611F0CEFA6268F4
:102790000646D107EBD58DF824900DE012F0100F0E
:1027A0000CBF0122042221698DF824200DF126009E
:1027B000072210F0A5FFD8460F2142F20600FEF7CF
:1027C00025FD8346002800F08F800F2208A90C30D9
:1027D00013F050FB0022594642F20600FEF760FD5E
:1027E000002840F08480B9F1000F1FD06368DB0738
:1027F0002AD42846012111F0A8FA079D8346002813
:1028000064D045213E480FF034FC002D3FF461AF09
:102810002846002100F088FD284600F055FD58E7C5
:102820000323DDF858808DF82430C5E7179B524606
:1028300000932846CDE90186169B059911F003FA0D
:1028400083460028D2D044E7284607A9FFF7A4FE14
:1028500083460028CDD010F10C0F7FF43AAFB9F1C8
:10286000000F7FF436AF626890073FF532AF6368C0
:1028700083F00203C3F3400B0BF001020E21384634
:1028800011F0CEF9731E5A425A410821384611F010
:10289000C7F9B11E4A424A413846092111F0C0F930
:1028A00062680A21384602F0010211F0B9F9424685
:1028B0000B21384611F0B4F962680D213846C2F395
:1028C000800211F0ADF94FF0000B02E715B1284678
:1028D00000F0FAFCB9F1000FCED1C8E76FF00A0B97
:1028E000F7E66FF0770BF4E66FF0680BF1E68346DE
:1028F000EFE600BFCC200020002000203499020029
:102900002CA0020073B51546069A0C46CDE900329C
:102910002B460A4601461148FFF7C0FE21460646EF
:10292000002340F201109D4202D1304602B070BD3A
:102930000A88824204D14A6812B11278D20702D4BE
:1029400001330831EFE7064906480CF0B3FE4FF4B7
:102950007022002303480CF097FFE6E718200020C0
:102960009F3D02003020002010B51A4811F014FAE3
:102970006FF48041184811F048F9174811F042F9F6
:1029800003461A06C0F3C01023D5134811F03AF9D4
:10299000430514D507221149114810F08AFE114B46
:1029A00098B904221049187E00F0FCFE044630B1AC
:1029B0000021017300F0B8FC204600F085FCBDE862
:1029C00010400021034811F0C0B9052203F1210194
:1029D000E9E710BD182000202820002034990200CB
:1029E00021200020002000202D99020073B51E4CEC
:1029F000204611F007F9400434D5204611F002F9C1
:102A000001062FD4204611F0FDF842052AD501A970
:102A1000A4F11000FFF7C0FD054618BB0121A4F189
:102A2000100011F092F9019E28B9304602B0BDE8BD
:102A3000704000F049BC2946304600F075FC6FF448
:102A40008041204611F0E1F80546304600F03CFC9C
:102A50006B0407D5D4E8EF3F43F48043C4E8E23F7A
:102A6000002AF7D102B070BD2820002030B58DB00B
:102A7000202104A8FEF78CFC0446E0B914F0C9FE3E
:102A80004FF47A75A0FB053205FB0121DB0B43EA0D
:102A90004143C90BCDE902310823202200930748A6
:102AA0006B4404A910F0C1FC28B9452104480FF07B
:102AB000E0FA6FF0040420460DB030BDE82E00208F
:102AC00053A00200884208B501F110030CD99842C6
:102AD0000FD20C490C4840F215220FF0B6FA40F222
:102AE000152108480FF0AAFAF3D000F11002914224
:102AF000EEE7013813F8012D8B4200F8012FF9D1D0
:102B000008BD00BF6FA00200558D020007B5082167
:102B10006846FEF73DFC58B908226946074810F0A0
:102B200064FC40B9064845210FF0A3FA6FF0040099
:102B300003B05DF804FBFFF799FFF9E7E82E0020EA
:102B4000A1A0020038B50D46044698B191B10B4AD8
:102B500010F084FC431C07D1FFF788FF48B92946D1
:102B60002046064A10F07AFC01280CBF00206FF0C6
:102B7000040038BD6FF01500FBE700BFE82E002011
:102B8000402208B5034910F094FDB0FA80F04009E6
:102B900008BD00BFFEA0020070B52D4B93F89A301F
:102BA00003F00603062B4AD100284BD0294E326889
:102BB00032B1131F834248D05B680BB1043BF9E785
:102BC00042607268031D336002B97360224CD4E81E
:102BD000EF2F42F02003C4E8E13F0029F7D112F0C3
:102BE000200202D00025284670BDD4E8EF3F23F034
:102BF0001003C4E8E13F0029F7D1114642F2250055
:102C0000FEF74EFB05460028ECD0452113480FF097
:102C100030FAD4E8EF3F23F02003C4E8E23F002A73
:102C2000F7D134683CB154F8043C043C0BB10020AB
:102C300098476468F6E70023C6E90033D3E76FF0EE
:102C40008505D0E76FF01505CDE76FF07705CAE78A
:102C500000200020183D0020CC200020CFA0020042
:102C6000044BD3E8AF3F13F0100F034808BF002018
:102C7000704700BFCC2000205E460020F8B51C4DF8
:102C800006462B688B422CD013B16FF00F00F8BDB5
:102C9000184BD3E8AF2FC2F340179206F5D4D3E810
:102CA000AF3FDB0620D5296042F226004021FEF727
:102CB000ADFA044690B140210C3006F019FE4022D6
:102CC000314610F01DFD3A46214642F22600FEF73D
:102CD000E7FA0028DBD000232B60D8E76FF068000C
:102CE000F9E76FF07700D2E76FF07C00CFE700BF25
:102CF000143D0020CC200020F8B5174CC668D4E85D
:102D0000EF3F23F02003C4E8E23F002AF7D13378F5
:102D100063B940221148711C10F0F2FCD4E8EF3F77
:102D200043F01003C4E8E23F002AF7D10C4D2C68B1
:102D30006CB10A4F043C23682BB13278002A0CBFD7
:102D400038460020984764680CB1043CF3E7002340
:102D5000C5E90033F8BD00BFCC2000205E4600204E
:102D6000183D002005490B6833B1C2680020086097
:102D7000117801B9501C1847704700BF143D00205E
:102D800070B50446104B1D6875B9104D104EB54214
:102D900018D91049104840F25B520FF056F940F232
:102DA0005B510C480FF04AF92B6813B12046217B88
:102DB0009847AD69E8E72B6813B12046217B984717
:102DC0001C35E4E7F7D370BD503D0020AC7D020018
:102DD000E47D020045A10200558D02002DE9F0417D
:102DE00004464FF00008144F4FF02002EFF3118318
:102DF00082F31288BFF36F8F216A29B983F3118898
:102E0000BFF36F8FBDE8F081606A0A68814208BF36
:102E10006262226283F31188BFF36F8FD1E901569A
:102E20003846C1E90188C1F80C8014F034FC002256
:102E300031462046A847D7E7F827002070B504465A
:102E400041B90D490D4839220FF0FFF839210A48E0
:102E50000FF0F4F80022D1E90156CA60C1E901225D
:102E6000074814F018FC314620462B46BDE8704058
:102E70006FF06D02184700BF45A10200558D02009A
:102E8000F82700202DE9F84304460E4617469946D8
:102E90008D694FF0FF334FF0FF3245480BF0DAFFFA
:102EA000637B072B78D14FF02003EFF3118283F37C
:102EB0001288BFF36F8F002D43D000232B60A369CE
:102EC000002B3BD1C4E9055582F31188BFF36F8F06
:102ED000042106F10C0006F0BBFC238807F0FD0777
:102EE00043EA07370780338A043B43800223304696
:102EF0003376FEF76BFC0246002857D045212D485B
:102F00000FF0B7F84FF02003EFF3118783F3128827
:102F1000BFF36F8F15B3294604F1140010F06DFF55
:102F200087F31188BFF36F8F21480BF059FF0023FF
:102F300029462046B361FFF781FF27E01D60A561A8
:102F4000C2E7A36933B103F10C08DB680133C8F8A9
:102F50000030B9E7E36904F11C08F7E7D8F800206E
:102F600052B91549154840F227220FF06EF840F289
:102F7000272111480FF062F8013AC8F8002087F3C2
:102F80001188BFF36F8F0A480BF02AFFB9F1000FC9
:102F900008D10020BDE8F88305480BF021FF002D83
:102FA000C5D1F3E7304606F09DFBF2E70120F1E7DB
:102FB000002100204C9D020045A10200558D020019
:102FC000004870470021002038B5002204468A429C
:102FD00002D10024204638BD012004F1C403D3E807
:102FE000EF5F002D04D1C3E8EC0FBCF1000FF6D168
:102FF00002D0C8340244EAE7002CEAD0C4220021FF
:10300000204610F088FB04F1600004490CF052FBEC
:10301000034904F128000CF073F9DBE711390100D2
:10302000473E02002DE9F0410446002704F138062E
:1030300000230022304612F000FF034660B96369A6
:10304000ABB116494FF42D7215480EF0FEFF4FF448
:103050002D7112480EF0F2FF9D699F6106F042FB50
:10306000002DE5D029462046FFF7E8FEDEE7E369BC
:1030700043B10A4940F2B52209480EF0E6FF40F29A
:10308000B521E6E7204610F0E1FE04F160000022E1
:10309000BDE8F04100230CF0F7BB00BF45A10200E2
:1030A000558D020070B5164604460D46FFF796FE94
:1030B000012E1FD0022E49D1236933B12B4845215F
:1030C0000EF0D7FF204610F0C1FE256121690A8A63
:1030D000012A49D9CB681B8804339BB29A4243D357
:1030E0003AD9234845210EF0C4FF2046BDE8704080
:1030F00010F0ACBE206938B945211E480EF0B9FF6A
:10310000204610F0A3FE01E02E8A26B92846BDE82D
:10311000704006F0E7BA0C3012F0A4FE86420BD9DC
:10312000452115480EF0A5FF00222046216900F038
:1031300043FE00232361E9E720692A8AE9680C300D
:1031400012F098FE284606F0CDFABFE73246452138
:103150000A480EF08EFFD3E7002323612046BDE826
:103160007040012200F028BE70BD00BF75A10200B2
:1031700009A2020097A10200BAA10200E6A1020082
:10318000F8B51F46437B0446072B0E46154606D06E
:1031900045211B480EF06DFF6FF07F0016E062B313
:1031A0000DF004FB174B8342174807BF0022002392
:1031B0004FF0FF324FF0FF330BF0BAFD014630B94C
:1031C000124845210EF055FF6FF06800F8BD637B93
:1031D0000022072B06D0C0E90122C2600A4814F081
:1031E0005AFAD9E7C0E90157C260B16104F1380069
:1031F000314606F057FA0020E8E71146F5E700BF30
:1032000029A2020020360020F82700203DA202005B
:1032100070B50446174814F0BDFB0022012120467A
:10322000144B0EF099F804F11406134BD3E8AF2FAA
:103230000AB9012070BDA3F1C40513F8B73C53B916
:103240006FF04001281D10F0F3FD430603D528461A
:10325000FFF7E8FEEDE76B7B072BEAD13046074B23
:10326000002204210EF078F80123022084F8203097
:10327000E0E700BF8C220020E4300020583000201E
:1032800010B580B100F1C402D2E8AF3FB3B1591C10
:10329000D2E8EF4F9C4204D1C2E8EC1FBCF1000F12
:1032A000F6D1F1D110BD0649064840F27C420EF03D
:1032B000CCFE40F27C4102480EF0C0FE1846F1E719
:1032C00045A10200558D020010B500F1C403D3E8FA
:1032D000EF2F511EC3E8E41F002CF8D1002A0ADCAE
:1032E0000B490C484FF493620EF0AFFE4FF493611C
:1032F00007480EF0A3FE40F201124188914206D128
:10330000D3E8AF3F1BB9BDE81040FFF76FBB10BD5E
:1033100045A10200558D020002460121014810F02E
:103320009EBD00BF2030002070B5457B04468D4215
:1033300000F08980417325B98378082B01D0FFF70D
:103340009FFF637B012B16D100264E4D4FF02002CC
:10335000EFF3118382F31288BFF36F8FE269002AC3
:103360006BD0013AE26183F31188BFF36F8F284677
:103370000BF036FDEAE7072B09D0002B63D1A378C9
:10338000042B21D12046BDE87040FFF79DBFA378F4
:10339000042B58D004F1380014F070F900213A4899
:1033A0000EF0B6F80023C4E91533E378012B4AD1B7
:1033B000032384F8B43004F160004FF42032BDE8F8
:1033C000704000230CF0FCB9013D052D3BD801A352
:1033D00053F825F0ED3301002D3401008533010051
:1033E000853301002D3401002D3401002046FFF704
:1033F000F5FCA378012B0AD104F16005284614F0EE
:10340000D3F910F00C0F02D028460CF043FA043424
:10341000D4E8EF3F43F04003C4E8E23F002AF7D18D
:10342000BDE87040002118480EF072B8237B002BD5
:10343000A8D02046FFF7A4FCA4E7616921B983F373
:103440001188BFF36F8F70BDA0690A68814208BF01
:10345000A261626183F31188BFF36F8F4FF0200286
:10346000EFF3118382F31288BFF36F8FCA68E261B2
:10347000CE6083F31188BFF36F8F2046FFF7DEFC29
:1034800075E700BF002100208C2200200A4A08B501
:103490000A49831ADB10904201FB03F30AD0084962
:1034A000084840F2B6420EF0D0FD40F2B641044862
:1034B0000EF0C4FDD8B208BD20300020295C8FC2B8
:1034C00045A10200558D0200F8B504460D46174689
:1034D0001E4614F0A4F850B10D490E4840F2D242F5
:1034E0000EF0B3FD40F2D24109480EF0A7FD0A49A3
:1034F0003A46002C14BF20460846334612F098FC8A
:10350000044618B1691D0C3006F014F82046F8BDC9
:1035100045A10200558D020048280020F8B5044658
:103520000430D0E8AF3F9B0511D5B4F8A630B4F80D
:10353000A8209A420BD8B4F8AA209A4207D3D4E91B
:103540002B239A4203D16FF4007110F071FC164BDB
:103550001D6875B9154D164FBD4222D9154916483B
:1035600040F2A5520EF071FD40F2A55111480EF047
:1035700065FDEE683EB12046B4F8AE30B4F8AC203C
:10358000B4F8A610B047AD69E3E7EE683EB1204657
:10359000B4F8AE30B4F8AC20B4F8A610B0471C357F
:1035A000DAE7F2D3F8BD00BF503D0020AC7D020049
:1035B000E47D020045A10200558D02002DE9F04195
:1035C000074608460C4610F016FA054618B90025BD
:1035D0002846BDE8F081194B1E687EB9184EDFF809
:1035E0006480464523D91849184840F2ED520EF040
:1035F0002CFD40F2ED5114480EF020FDB3680BB9DC
:10360000B669EAE72146384698470028DFD02046C9
:1036100010F0F1F90028F3D1D9E721463846984750
:103620000028D4D0204610F0E6F920B9CFE7CFD259
:10363000B368002BF1D11C36D3E700BF503D00200A
:10364000AC7D0200E47D020045A10200558D020020
:103650002DE9F041C3780446BBB900F19E06164B34
:1036600004F190071D689DB9144D154F04F19008A1
:10367000BD421DD91349144840F2BC720EF0E5FC5E
:1036800040F2BC710F480EF0D9FC00F19706E6E756
:103690002B691BB13A46314620469847AD69E2E7AF
:1036A0002B691BB142463146204698471C35DFE75F
:1036B000F6D3BDE8F08100BF503D0020AC7D020094
:1036C000E47D020045A10200558D0200F8B5437A61
:1036D00004468372164610F002FD124B1D6875B940
:1036E000114D124FBD421AD91149124840F6280215
:1036F0000EF0ABFC40F628010D480EF09FFC6B6904
:103700001BB132462046617A9847AD69E7E76B699D
:103710001BB132462046617A98471C35E2E7F6D362
:10372000F8BD00BF503D0020AC7D0200E47D0200EA
:1037300045A10200558D020070B506460D460A48A7
:103740000121FFF741FC044660B1067207222946B9
:1037500090300FF0D5FF01236372A372A370034B67
:10376000C4F8A830204670BD203000201800280082
:1037700070B505460A480E46FFF782FD044620B1A3
:103780008378012B04D0FFF79FFD0024204670BDF5
:103790003246294610F0E4FB0028F7D12046F2E734
:1037A00020300020F8B505460E480E461746FFF7B4
:1037B00067FD044620B18378012B03D0FFF784FD19
:1037C00000240DE036B13246294610F0C9FB08B995
:1037D0002046F3E7637BBB42FAD1237AAB42F7D1B1
:1037E0002046F8BD2030002010B5837802460B70CB
:1037F000C3784B70037A8B70437B082B0FD8264C11
:10380000E35C0B770023CB77437A4B7710F072FBA6
:1038100088779378012B0DD06FF0150010BD1F49EC
:103820001F4840F60E120EF010FC40F60E111B4819
:103830000EF004FC02F190038B60137A1948C3EB7D
:10384000C30303444B60D47802F19E0302F1970056
:1038500014B11C4603462046C1E90303B2F8A63062
:103860008B82B2F8AC30CB82B2F8AE300B83D2F898
:10387000C03023B15B7BD80644BF0123CB77D2F89D
:10388000C03013B15B7B9B0601D40020C6E7CB7F21
:1038900043F00203CB77F8E760A2020045A10200E3
:1038A000558D02000020002038B5044608460D461C
:1038B00010F0A1F838B3154B93F8D030990707D41E
:1038C000E37873B129462046BDE8384000F09CBA41
:1038D00094F8B5309A07F3D5231DD3E8AF3F5B05C5
:1038E000EED42946204610F065FB58B92B88A4F881
:1038F000A8306B88A4F8AA30AB88A4F8B030EB8865
:10390000A4F8B23038BD6FF01500FBE700200020AE
:10391000F7B510F8533C0446A0F160065BBB304697
:1039200010F0C5FB304B1D6875B9304D304FBD42AE
:103930001AD93049304840F26C520EF086FB40F202
:103940006C512C480EF07AFB6B681BB1304614F8B2
:10395000541C9847AD69E7E76B681BB1304614F813
:10396000541C98471C35E2E7F6D3304603B0BDE857
:10397000F040FFF7A9BC10F85E3C012B1ED1A0F16E
:103980005C056FF40071284610F052FA830517D5D4
:10399000A36C69460093236D30460193FFF784FFC3
:1039A00020B96FF48071284610F042FAD5E8EF3F55
:1039B00043F08003C5E8E23F002AF7D103B0F0BD31
:1039C0006B460E4A1068516803C369463046FFF7DC
:1039D0006BFF0028EAD1D5E8EF3F43F48073C5E8D8
:1039E000E23F002AE2D0F6E7503D0020AC7D020025
:1039F000E47D020045A10200558D020024800200F2
:103A000001460148FFF760BDE42800202DE9F041A0
:103A100006464FF0FF334FF0FF3200200C46FFF711
:103A2000EFFF737B0546072B4FF0000605D005F02E
:103A300059FE35462846BDE8F081866100F10C0745
:103A40000C4E3846B6F8FC8012F00CFA80450CD2C9
:103A5000B6F8FC6054F80C1F3246384612F00AFAE9
:103A60003146204605F010FFE4E7384612F0FAF937
:103A700086B2EFE70020002070B5437B04465BB9B7
:103A80006FF04001043010F0D3F9430604D520460E
:103A9000BDE87040FFF7C6BA0022002304F13800E9
:103AA00012F0CBF9054658B940F21A3222492348A0
:103AB0000EF0CBFA404080F311884FF0030002DF94
:103AC0001F4E2A8AB6F8FC309A4207D800230222F9
:103AD00029462046FFF7D6F968B905E02946204671
:103AE000FFF794FF014638B90023AE692846AB6161
:103AF00005F0F8FDCEB970BD012300222046FFF786
:103B0000C1F90028F0D02A8AB6F8FC309A4202D8CF
:103B100000230322DCE729462046FFF777FF014612
:103B20000028E1D001231A46E8E731462046BDE8E7
:103B30007040FFF783B900BF45A10200558D020018
:103B4000002000200B4B58B11A6862B902693AB9DB
:103B500002685AB942684AB982683AB942692AB9D0
:103B60001860002070476FF0770070476FF0150005
:103B7000704700BF5C3D002068B10023C360074B65
:103B800000F10C02596819B9C3E9002200207047FE
:103B90000A605A60FAE76FF015007047543D002044
:103BA00010B90248FFF76CBB00207047203000209E
:103BB00010B50C4813F062FD0B490A4813F06BFD79
:103BC0000A49084813F067FD0949064813F063FDE8
:103BD00000F01AFF03F086FF044608B910F0CAFA95
:103BE000204610BDF8270020203D0020303D002059
:103BF000403D002008B502460748036823B9074A3C
